:0900000601000013340031320046
:020000041A00E0
:10000000B8F100202106001A2906001A4100001B41
:100010002D06001A2F06001A3106001A5A5A5A5A8B
:10002000000000000000000000000000F104001AC1
:100030003506001A00000000A905001A0D06001A76
:100040003B06001A3B06001A0562001A0000000079
:100050003B06001A8563001AED4C001B3B06001A94
:100060002D59001B3B06001A3B06001A3B06001ADE
:100070003B06001A3B06001A3B06001A3B06001A14
:100080003B06001A3B06001A2168001A3B06001ABC
:100090003B06001A3B06001A3B06001A3B06001AF4
:1000A0004152001B3B06001A3B06001A3B06001A91
:1000B0003B06001A3B06001A3B06001A3B06001AD4
:1000C0003B06001A3B06001A3B06001A3B06001AC4
:1000D0003B06001A3B06001A3B06001A3B06001AB4
:1000E0003B06001A3B06001A3B06001A8D5F001AF9
:1000F000000000003B06001A3B06001A3B06001AEF
:10010000000000003B06001A3B06001A1138001BD5
:100110003B06001A00000000000000000000000084
:1001200000000000000000000000000000000000CF
:1001300000000000000000000000000000000000BF
:1001400000000000000000000000000000000000AF
:10015000000000000000000000000000000000009F
:10016000000000000000000000000000000000008F
:10017000000000000000000000000000000000007F
:10018000000000000000000000000000000000006F
:10019000000000000000000000000000000000005F
:1001A000000000000000000000000000000000004F
:1001B000000000000000000000000000000000003F
:1001C000000000000000000000000000000000002F
:1001D000000000000000000000000000000000001F
:1001E000000000000000000000000000000000000F
:1001F00000000000000000000000000000000000FF
:1002000000000000000000000000000000000000EE
:1002100000000000000000000000000000000000DE
:1002200000000000000000000000000000000000CE
:1002300000000000000000000000000000000000BE
:1002400000000000000000000000000000000000AE
:10025000000000000000000000000000000000009E
:10026000000000000000000000000000000000008E
:10027000000000000000000000000000000000007E
:10028000000000000000000000000000000000006E
:10029000000000000000000000000000000000005E
:1002A000000000000000000000000000000000004E
:1002B000000000000000000000000000000000003E
:1002C000000000000000000000000000000000002E
:1002D000000000000000000000000000000000001E
:1002E000000000000000000000000000000000000E
:1002F000000000000000000000000000FFFFFFFF02
:1003000000F002F800F0B3F80AA090E8000C824474
:100310008344AAF10107DA4501D100F0A8F8AFF251
:10032000090EBAE80F0013F0010F18BFFB1A43F0D3
:1003300001031847880B0500F80B05000A444FF02D
:10034000000C10F8013B13F0070408BF10F8014B34
:100350001D1108BF10F8015B641E05D010F8016B79
:10036000641E01F8016BF9D113F0080F1EBF10F8DD
:10037000014BAD1C0C1B09D16D1E58BF01F801CB00
:10038000FAD505E014F8016B01F8016B6D1EF9D583
:100390009142D6D370470000103A24BF78C878C184
:1003A000FAD8520724BF30C830C144BF04680C607B
:1003B000704700000023002400250026103A28BFC3
:1003C00078C1FBD8520728BF30C148BF0B607047C7
:1003D0006E2900F05F83702903F01A82662932F0DB
:1003E000BA80652932F0B780672932F0B48061297C
:1003F00003F0138203681B0A28BF41F080016929BA
:1004000000F00C83642900F00983752900F006834D
:100410006F2900F07483782903F00482E92903F03E
:100420000682E42903F00382F52903F00082EF2914
:1004300000F07183F82903F0FF810368DB0928BF0E
:1004400041F08001632901F09583732901F09A83BB
:10045000E32903F0F681F32903F0F88100207047C7
:1004600010B5002001F06DFD03F0F5F910BD03F0AB
:10047000F7F9114603F0F9F90FB403F0FBF90FBCDB
:1004800024F010FF03F0FBF980F309887047EFF3C5
:1004900009807047684680F3098804480078C007DF
:1004A00014BF0220032080F31488704714E4041A58
:1004B000DFF818C0EFF305831B0618BF6047EFF3A2
:1004C0001483DB0708BF604700DF7047A3B1021A3F
:1004D000DFF818C0EFF305831B0618BF6047EFF382
:1004E0001483DB0708BF604700DF704719B3021AA7
:1004F000EFF30980816911F8021CE1BB90E80F104D
:1005000010B5E047BDE81040EFF3098C8CE8070018
:10051000214B93E80600914208BF704741B91EF095
:10052000100F16D11D49086820F00100086010E086
:100530001EF0100F06BF2CED108A0120002081F85C
:1005400025002CE9F00FC1F828C00CB403F09CF989
:100550000CBC1A60D2F828C0BCE8F00F92F8250055
:1005600000280EBF6FF0020E6FF0120EBCEC108A66
:100570008CF30988704710B5094A1268914209D86E
:10058000084C54F8214090E80F10A047EFF3098C75
:100590008CE80F0010BD00000002002034EF00E0E6
:1005A0000C38001A0C38001A10B52AF0E7FFBDE825
:1005B0001040154B93E80600914208BF7047EFF3D7
:1005C000098C1EF0100F06BF2CED108A01200020B0
:1005D00081F825002CE9F00FC1F828C00CB403F015
:1005E00053F90CBC1A60D2F828C0BCE8F00F92F89E
:1005F000250000280EBF6FF0020E6FF0120EBCEC4B
:10060000108A8CF3098870470002002010B52BF087
:1006100047F9CCE710B52AF06FFB2BF041F9C6E79C
:100620000948804709480047FEE7FEE7FEE7FEE786
:10063000FEE7FEE7FEE7FEE7FEE7FEE704480549C2
:10064000054A064B704700005573001A0103001A53
:1006500000080028B8F100200088FF29B8EF00202A
:1006600000487047D8EE00200B3020F0070070479C
:100670002DE9F04117460E460446FFF7F5FFA0426C
:10068000054633D9002F1CBF06F10C0003F001F919
:1006900030467468F4B12168A94217D305F1080205
:1006A00091423CBF6168416007D3626861194A604A
:1006B0002268521B0A6041602560002F1CBF06F1B2
:1006C0000C0021F00FFF201DBDE8F081204664687A
:1006D000002CE0D12946304603F0E0F80028D7D1BD
:1006E000002F1CBF06F10C0021F0FCFE0020BDE82D
:1006F000F08110B5044600F011FE01682046BDE807
:1007000010400122B4E70B3020F0070070472DE9BC
:10071000F0410F460546041F00F000FE0668F7B1E1
:10072000384615B3FFF7EFFFB84205463CBF00203F
:10073000BDE8F08106F10C0003F0ABF82268AA4294
:1007400038BF314615D3511B082931D36019002217
:1007500040F8041B3146256003F0A5F828E0284640
:1007600003F0A6F80020BDE8F081BDE8F041FFF7F6
:10077000C0BF4868002818BFA04238BF0146F8D360
:10078000131983421BD103681A44954217D8531B8F
:10079000082B0AD343686219536023680068184421
:1007A000401B106025604A6002E02260406848609B
:1007B00006F10C0021F096FE201DBDE8F08100221C
:1007C0003146281FFFF754FF05000AD02068211D7D
:1007D000021F284603F071F800223146201D03F065
:1007E00062F806F10C0021F07DFE2846BDE8F0819C
:1007F00053EA020C00F069802DE9F04B4FF000063F
:10080000002B1FBFB3FA83F503FA05F424FA05F6AB
:100810005E4012BF1643B2FA82F502FA05F4C5F142
:1008200020051EBF22FA05FC44EA0C04203556EAD6
:10083000044C4FEA144418BF641C4FF000084FF0FA
:100840000009904271EB030C39D3002919BFB1FAAA
:1008500081F701FA07F6B0FA80F700FA07F6C7F158
:1008600020071EBF20FA07FC46EA0C062037B6FB1D
:10087000F4FCA7EB0507103F07F01F0BCBF1200698
:100880000CFA0BFB2CFA06F644BFB3460026202FC9
:10089000A4BF5E464FF0000B5BEA060C08BF4FF0AA
:1008A000010B19EB0B09ABFB027C48EB0608C01BE4
:1008B00006FB02CC0BFB03CC71EB0C01C1E70B4632
:1008C000024641464846BDE8F08B13B54FF00000A4
:1008D0004FF00001AFF30080BDE81C407047B2F15B
:1008E00020030AD5C2F1200301FA02F120FA03F332
:1008F00000FA02F041EA0301704700FA03F14FF0F9
:10090000000070470FB4014610B504AA039802F026
:10091000D9FF10BC5DF814FB0FB41CB5084B06AA38
:100920007B4469460090059801F007F904460020D1
:10093000694602F0CCFF20461CBC5DF814FB0000A9
:10094000110100010FB47CB50C0009AA009001D080
:100950002044401E084B7B4469460190089801F0F2
:10096000ECF805461CB10020694602F0B0FF2846AD
:100970007CBC5DF814FB0000E500000170B5044686
:1009800085690068C10601D5302600E02026C00731
:1009900007D070BDD4E9012130469047206A401C41
:1009A00020626D1EF6D570BD70B50446856900786D
:1009B000C00707D170BDD4E9012120209047206AEB
:1009C000401C20626D1EF6D570BD70B50C46054604
:1009D000012A05D02878800600D5EA69002302E0C4
:1009E000012305E05B1C934202D2E05C0028F9D1B0
:1009F000A869E618C01AA861286A1844286228461F
:100A0000FFF7BCFF04E0D5E9012114F8010B904782
:100A1000B442F8D32846FFF7C7FF70BD2DE9F04177
:100A20000646002410687529314616A510D002F03C
:100A300053FF002802DA404213A507E031688A0715
:100A400001D512A502E0490704D511A5012401E052
:100A500002F047FF00210A2206F1240709E0B0FB5B
:100A6000F2FCB0FBF2F302FB1C0030307854184665
:100A7000491C0028F3D123462A463046BDE8F04100
:100A800000F072BC000000002D0000002B000000F0
:100A90002000000011680268006A530501D5087043
:100AA0000AE0D30501D5088006E0130603D5C21776
:100AB000C1E9000200E008600120704730B4002165
:100AC00000F1240408E002F00705D208303542EABC
:100AD0004372DB086554491C52EA0305F3D10468EC
:100AE000002310A2250707D5A40600D421B1C469AC
:100AF00001230DA2641EC46130BC00F035BC10B5EA
:100B000004462146106802F0ECFE02462046BDE88D
:100B100010400023D2E7D21D22F00701D1E90023C3
:100B2000CCE7000000000000300000002DE9F05F7D
:100B3000894604464FF0000ADFF874B1FB44C0F860
:100B400020A02046E1688847002874D0252806D0D8
:100B5000D4E901219047206A401C2062F1E7002679
:100B60005F462046E16888472028054607DB312D8F
:100B700005D2781910F8200C08B10643F1E7B00748
:100B800001D526F00406C4F81CA00027C4F818A05C
:100B90002A2D09D0284602F0A9FE38B304EB8708B5
:100BA000303DC8F8185019E059F8041B204604EBF2
:100BB00087029161E1688847012F054618D1E069F5
:100BC000002820DA26F020061DE0D8F8180000EBF7
:100BD000800005EB40003038C8F818002046E16876
:100BE0008847054602F082FE0028EED1012F0AD088
:100BF0002E2D08D12046E16888477F1C0546022F2C
:100C000046F02006C4DBA069002803DA404246F023
:100C10000106A061F00701D026F010066C2D0BD064
:100C2000682D09D04C2D39D06A2D35D0742D35D092
:100C30007A2D33D016E038E0E1682F462046884709
:100C4000B842054609D16C2F26D04FF48060E16888
:100C5000064320468847054604E06C2F1AD04FF41F
:100C6000807006430DB3A5F14100192802D8203544
:100C700046F400664A462946204626604E46FFF75F
:100C8000A7FB80B101280BD0F61D26F0070000F16C
:100C9000080956E74020E4E78020D8E70020D6E79F
:100CA00006F104094DE7284652E7206ABDE8F09FA7
:100CB0007CE104012DE9FF5F1D464FF0FF3B9146AB
:100CC0004FF000085F46D5E90146A96901987F1CED
:100CD0008847296A824688470028F6D1BAF1FF3F43
:100CE0000CD0002E24F4C06419DD600614D5BAF1CE
:100CF0002B0F09D0BAF12D0F0ED103E0584604B0E6
:100D0000BDE8F09F44F48064A96901987F1C88477E
:100D1000761E8246002E02DDBAF1300F03D0B9F103
:100D2000000F26D032E0A969761E01987F1C44F49A
:100D300000748847002E824605DDBAF1780F06D090
:100D4000BAF1580F03D0B9F1000F10D01EE0B9F17D
:100D5000000F02D0B9F1100F18D1A969761E0198C1
:100D60007F1C24F4007488478246102002E008208B
:100D700000E00A20814609E0A96908FB0908761EFF
:100D800001987F1C44F4007488478246002E05DDDC
:100D90004946504602F0AFFD0028EDDAE9690198B6
:100DA0008847A00502D46FF00100A8E7E00725D12D
:100DB000600613D5600502D5C8F1000000E040468A
:100DC00029680A1D2A600968220501D5087015E006
:100DD000220701D5088011E008600FE02868011D96
:100DE00029600068210502D580F8008006E021070F
:100DF00002D5A0F8008001E0C0F8008038467EE708
:100E000070B5064602F07CFD0468054630460A22AD
:100E1000002102F07AFD2C6070BD00002DE9F04148
:100E2000044616460D464769007B80072ED038469B
:100E300002F070FD50BB3EB3012E02D0022E25D130
:100E400004E0204602F06BFD05441DE0384602F048
:100E50006BFDE168002841F01001E16005DA2046F1
:100E600000F0BCFF0120BDE8F081C9030BD562682A
:100E7000E16A914200D81146A26911442269891A97
:100E8000814200DD08460544002D01DA0220EAE730
:100E9000E16A6068E268814206D29103E06203D5AC
:100EA00022F4003141F01002A6690027AE4213DCA3
:100EB000E16A814201D90B4600E0034603EB060CD0
:100EC0002369ACEB030CAC4506DD814201D98C46AD
:100ED00000E084469C4505D1A760276042F02000D1
:100EE000A5620DE0AD1BE669AE1B8142A66000D98C
:100EF0000846C01A281A20605819606022F02000A5
:100F000003490840E060002084F84870ABE7000027
:100F1000BFCFD7FF00F0DABF70B50C46064601F12F
:100F20004C05284602F0B5FC2146304602F001FD92
:100F30000446284621F0D6FA204670BD70B5044616
:100F400000F14C05284602F0A4FC204602F0E7FC24
:100F50000446284621F0C6FA204670BD70B5044606
:100F600000F14C05284602F094FC207B00F0400480
:100F7000284621F0B7FA204670BD00002DE9F04761
:100F800016468846814602F14C07384602F081FC3D
:100F9000304602F0D3FC18F8010B61280AD0722801
:100FA00002D077283FD102E00125002405E0022588
:100FB000042402E0082448F2020518F8010B2B284B
:100FC00006D0622809D018F8010C74280AD00BE06A
:100FD00045F0030544F00204EFE745F0040544F052
:100FE0000104EAE744F010044846214602F0ABFC55
:100FF000411C18D00021316171604FF40071F5601F
:10100000F1617061200704D5304602220021FFF70C
:1010100005FF306D40F001003065384621F062FA7E
:101020003046BDE8F0870026F7E72DE9F041154688
:101030000E460746204C204602F02BFC2A4631463D
:101040003846FFF79BFF0546204621F04BFA28461D
:10105000BDE8F0812DE9F0410E468046164D284648
:1010600002F017FC154C206DC10704D0410804D0D4
:1010700020F00104F7E7224612E05420FFF739FB85
:10108000070017D0206D47F0010108435421206567
:10109000384602F05DFC07F14C0002F05EFC3A4677
:1010A00031464046FFF76AFF0446284621F01AFA07
:1010B0002046CDE70024F8E720020020A0650010BC
:1010C000014A00F067BF00004002001030B505463D
:1010D0000B462A4613F8014B12F8010B08B1A04247
:1010E000F8D01CB1002802D06D1CF1E7284630BDB5
:1010F00040EA010310B59B070FD1042A0DD310C895
:1011000008C9121F9C42F8D020BA19BA884201D9E6
:10111000012010BD4FF0FF3010BD1AB1D30703D02E
:10112000521C07E0002010BD10F8013B11F8014BE4
:101130001B1B07D110F8013B11F8014B1B1B01D100
:10114000921EF1D1184610BD40EA0103024630B5A7
:101150009B0710D14FF0013400E008C208C91D1BE5
:101160009D4315EAC41FF8D013F0FF0102F8011BDC
:101170000DD01B0AF8E711F8013B002B02F8013BE8
:1011800005D011F8013B002B02F8013BF3D130BD33
:101190002DE9F041054690460E460020044600E049
:1011A000641C44450BD2285D02F0DCFB0746305D31
:1011B00002F0D8FB381A02D1295D0029F0D1BDE830
:1011C000F081002101E0801C491C0288002AFAD12C
:1011D0000846704740EA010370B59B072ED14FF0D7
:1011E0000136042A2AD308C810C99D1B9D43121F2B
:1011F00015EAC61517D0D8B2E1B2401A50EA056117
:1012000010D198B2A1B2401A50EA05410AD123F098
:101210007F4024F07F41401A50EA052102D1180E88
:10122000A0EB146070BDA342DBD018BA21BA88428B
:1012300001D9012070BD4FF0FF3070BD0AB9002008
:1012400070BD10F8013B11F8014B63B1A3420AD104
:10125000521E08D010F8013B11F8014B1BB1A342FC
:1012600001D1521EEDD1181B70BD421E12F8013F74
:10127000002BFBD111F8013B002B02F8013BF9D107
:10128000704700004FF0013C50F8042B51F8043B2C
:101290009A4221D1A2EB0C03934313EACC1317D14A
:1012A00050F8042B51F8043B9A4215D1A2EB0C03E1
:1012B000934313EACC130BD150F8042B51F8043BA1
:1012C0009A4209D1A2EB0C03934313EACC13DBD06F
:1012D0004FF00000704700BFD01A01BAB1FA81F197
:1012E00001F0180122FA01F0CB40C1F12001DBB27C
:1012F000C0B2C01A2CFA01F3D11A914311EAC311FA
:10130000E6D17047704770477047000010B502F093
:101310002EFB001D10BD00BF51B1020010B5FFF73C
:101320009FF9083010BD10B5FFF79AF9383010BD9D
:10133000704770477CB51D4616460C00009001D0E2
:101340002044401E074B7B442A46694601903046A4
:1013500000F0F3FB05461CB10020694602F0B7FA25
:1013600028467CBDF5F6FF002DE9F0470D4699466D
:101370009246044600F124080168880604D5E06915
:1013800021F01001216000E00120A84201DD471B8F
:1013900000E00027A1697A1902EB0900081AA06190
:1013A0002078C00602D42046FFF7E8FA002608E0BD
:1013B000D4E901211AF806009047206A401C761CE7
:1013C00020624E45F4DB2078C0060AD52046FFF7A0
:1013D000D5FA06E0D4E9012130209047206A401C6C
:1013E0002062381EA7F10107F4DC07E0D4E90121EF
:1013F00018F805009047206A401C2062281EA5F1BD
:101400000105F3DC2046FFF7CFFA2078000602D56D
:101410000220BDE8F0870120FBE770472DE9FF4F70
:101420000C461E464FF0FF378BB0D2E90001DDF8C5
:1014300060800A908A46C1F30A5505B93D460021ED
:1014400008464FF00000BAF1000F00F4400005DA42
:1014500000EB80004FF4400101EA50004FEA905940
:10146000B9F1010F00DDB9460A9850EA4A000ED0E2
:1014700044F61050A5F2FF3545432F14B8F1000F84
:101480001ED07542291E1EDDC9F100021CE0B8F114
:10149000010F4FF0000001D0302103E0F24305E0DE
:1014A0002154401CB042FBDB304600220021215475
:1014B0000B99C1F80880C1E900200FB0BDE8F08F9A
:1014C000BD1B6D1CDEE74A4600DA694206A802F041
:1014D00053FA06AB93E8070003AB83E807005046D6
:1014E0000A9901F055FF8DE80700A0F500501F385C
:1014F00000900398002D09DD42F21F014A4608447E
:1015000003A90390684602F059F908E0A0F50050DD
:101510004A461F3803A90390684602F032FA8DE864
:1015200007000004000C03D04FF0FF30410800E03A
:101530001046B8F1000F03D00022009215461EE0BD
:10154000751E05D400F08CFD303262556D1EF9D544
:10155000B3460122084302D000227F1C04E0207819
:10156000302801D100227F1E002A099786D01DE075
:10157000112D07DA00F074FD303262556D1C50EA0F
:101580000102F5D1084302D00098C8B10EE0002155
:10159000681E05E0235C625C63542254401E491CB3
:1015A0008142F7DBAB46A81B401E0990002004F8DF
:1015B0000B000B98099AC0F80880C0E9002B7CE763
:1015C00011264FF0000859E72DE9F04F88460446F0
:1015D000D21D22F0070191B0D1E90001CDE90A0145
:1015E0001EF062F902460B98C00F01D02D2007E0D3
:1015F0002068810701D52B2002E0202101EAC000EC
:10160000032A099001D0072A05DB034641462046FC
:1016100002F0BCF90BE12078800601D5E06900E01A
:101620000620B8F1650F814606D0B8F1660F18D0D4
:10163000B8F1670F70D131E00020B9F1110F0090BF
:1016400001DB112301E009F101030AAA01A90CA899
:10165000FFF7E4FEDDE90C70002609F10105834681
:1016600047E001204B4600904FF000470AAA01A92D
:101670000CA8FFF7D3FEDDE90DB00C995D460026FE
:1016800010B909F101000D18B9EB050003D4C0F140
:10169000FF3609F10105A5EB09002BE0B9F1010FB7
:1016A00001DA4FF001090020B9F1110F009048460E
:1016B00001DD112300E003460AAA01A90CA8FFF7E7
:1016C000ADFEDDE90C704D4600268346207800070C
:1016D0000AD4AB4500DA5D4601A8012D04DD4119AD
:1016E00011F8011C302907D04F4502DA17F1040F19
:1016F00004DA012082460FE06D1EEEE7002F02DCC7
:10170000ED1B3E4403E0781CA84200DD7D1CB81BA5
:1017100000F1010A4FF000472078000703D4AA45E2
:1017200001DB4FF0FF3A0021B7F1004F0DF1430804
:101730008DF8431024D002202B23002F01DA7F42A2
:101740002D230A21021EA0F1010000DC5FB197FBEE
:10175000F1FC97FBF1F201FB1C7C17460CF1300CFD
:1017600008F801CDEEE7A8F1010003702188090512
:1017700001D5452100E06521A0F1010800F8011C18
:1017800009980FA9A1EB0807FF1D00B1012041191D
:1017900001EBEA70A1693844081A401EA061207864
:1017A000C00602D42046FFF7E9F8099828B1D4E929
:1017B00001219047206A401C20622078C00622D573
:1017C0002046FFF7DBF81EE0002E04DBB34502DD08
:1017D00001A8805D00E03020D4E901219047206A13
:1017E000401C2062761CAAF101005FEA000A0AD1BF
:1017F00002F0BDF8C0680168405CD4E9012190475F
:10180000206A401C2062281EA5F10105DCDC07E0EF
:10181000D4E9012118F8010B9047206A401C20628E
:10182000381EA7F10107F3DC2046FFF7BDF80320BF
:1018300011B043E62DE9F04F04460D46D21D22F0CB
:10184000070089B0D0E90097484639461EF02CF8C9
:101850000246F80F01D02D2307E02068810701D54B
:101860002B2302E0202101EAC0038DF820300BB1C8
:10187000012000E00020032A824601D0072A04DB71
:101880002946204602F082F83FE12078800601D404
:101890000D2500E0E569C7F30A560D2D49DA002150
:1018A0004FEA175B08464FF00000002F00F440009D
:1018B00007DA00EB80004FF4400100EBD07001EA42
:1018C00060008115012901DD4FF0FF3100224FEA50
:1018D000850CBCF1180F06D31346ACF118004FF07D
:1018E0008052C24003E04FF4801323FA0CF30CF152
:1018F0000C0CBCF1200F04D3ACF1200C09FA0CF055
:1019000001E007FA0CF000294FF0004801DD18B99A
:101910000FE00ED140450CD319EB02095F4121B90C
:10192000404502D19F4329EA0209BBEB175F00D073
:10193000761C2088000502D57B48784402E07A486E
:101940007844193808AA302302F80A30037C0AF1D7
:101950000101002E0AF1020A53546A4602DC4FF0DC
:10196000300101E04FF031014FF001088DF8001017
:1019700002D0A6F2FF3603E059EA470100D06B4ED1
:10198000002D02DC2178090704D54FF002082E2132
:101990008DF80110C44600210BE0C7F303433F015B
:1019A000C35C491C6D1E02F80830052908F10108C6
:1019B00001DA002DF1DC00210CE000EB1973491C69
:1019C0001B786D1E082902F808304FEA091908F142
:1019D000010801DA002DF0DC21688B0602D516E043
:1019E000A8F10108E04505DD02EB080313F8013C0E
:1019F000302BF5D0B8F1000F09DD02EB080313F826
:101A0000013C2E2B03D1090701D4A8F10108002DB8
:101A100005DD3E2102F808106D1E08F10108407C2A
:101A2000002E02F8080008F1010804DA2D207642A1
:101A300002F8080002E02B2002F808000A214FF407
:101A40007A70864208F101080BDB96FBF0F3303325
:101A500002F8083096FBF0F308F1010800FB13666A
:101A600001E0642E0CDB642096FBF0F3303302F8C7
:101A7000083096FBF0F308F1010800FB136601E063
:101A80000A2E06DB96FBF1F0303002F8080008F170
:101A9000010896FBF1F001FB1060303002F80800FD
:101AA000A16908F1010808EB050202EB0A00081A17
:101AB000A0612078C00602D42046FEF75FFF216AAD
:101AC00008AE01EB0A00206204E0D4E9012116F817
:101AD000010B9047BAF1010AF7D22078C00602D56F
:101AE0002046FEF74BFF6E4609E016F8010B3E2834
:101AF0000FD0D4E901219047206A401C2062B8F140
:101B00000108F2D22046FEF74FFF09B00320BDE8DE
:101B1000F08F206A2844206203E0D4E901213020BC
:101B200090476D1EEBD3F8E76DD5040102FCFFFF73
:101B300001694A1C02610878704700B58FB0CDE991
:101B400001310021059105497944CDE90310114681
:101B50006846FEF7EBFF0FB000BD0000E5FFFFFF9A
:101B600010B5436913B1AFF3008001E0FEF72DFF1C
:101B7000012010BD127800F124010A7000224A7081
:101B80000122EDE711684FF0FF32E9E7D1E90023C8
:101B90009A4202D2931C0B60108070470FB400B5BC
:101BA0008DB010A9099000910B904FF0FF300A9072
:101BB00000200C90064878440690064878446A460F
:101BC00007900F9909A800F00DF80DB05DF814FB0F
:101BD0008BEFFF00A3EFFF00026811441378016050
:101BE00018467047D16005497944516104497944E8
:101BF000116200211161114600F078BAEDFFFFFF7C
:101C00006BF2FF002DE9F04705460C46C86820F44A
:101C1000201040F48000C860800602D5084600F01D
:101C200034F9E06841F282014FF0FF3901400229A6
:101C300003D0204600F0D2F8B5E000F42041B1F521
:101C4000004F0FD1C00306D56168E06A884200D812
:101C50000846606006E02069E0626060606901F04B
:101C600063FEA061A0680022EEB200280DDAE168F0
:101C70008B050AD4C043A06041F490302260E0603C
:101C80006068411C61600670A5E0E06890462260D3
:101C900040F40050E060206968BB606901F03AFEE2
:101CA000012704F12405A0B1A08910F4407F08D0D9
:101CB000E069FEF71EFD206118B1E06840F40060A5
:101CC00016E0E7612561E06820F4407040F4806030
:101CD0000EE0E069FEF70DFD00282061F1D0E0681C
:101CE00040F4006010F4407FE06002D140F4807066
:101CF000E06020696060E06825696FF0010AC10555
:101D00001FD56168E06A884200D80846411B04D0AC
:101D10002246284600F06CF8F0BBE068010203D5CB
:101D2000E562C4E9015854E0691CE1626160E1695F
:101D300040F48030491EC4E9021030462E70BDE8E0
:101D4000F087010202D500F480320AE06068411C8D
:101D500061600670E0680A2E40F48030E06006D0D2
:101D60000022E16A6068814203D90B4602E0012249
:101D7000F7E70346A7895B1B7F0503D4E7699F420A
:101D800000DDE2B1814200D80146E5620F1AC4E9E4
:101D90000158002B09DD00E005E0224619462846DF
:101DA00000F026F808B14846C9E747B1A069E562E6
:101DB0006560C01BA061E06840F01000E060E06872
:101DC000000208D56168A069E562491B08446560A6
:101DD000A0615046B3E73046B1E70000C16821F486
:101DE000001141F08001C1600021816001607047F5
:101DF0002DE9F047814614460E464FF0FF38324831
:101E0000D5685769054209D03846A16920F08DFB95
:101E1000002811DB2C48C0430540E5602B463246C4
:101E20004946384620F09BFBA16920F00042B21AD7
:101E300011440028A16103D02046FFF7CFFF4046A0
:101E4000BDE8F08770B504460569C06A61688842DC
:101E500000D80846E16821F42011E160C90312D5D9
:101E6000A84208D02246411B2846FFF7C1FF10B107
:101E70004FF0FF3070BD0020E562C4E90150E0681A
:101E800020F48030E060002070BD10B50446C068CA
:101E900020F02000E060A16AA06988420DD02046B1
:101EA000FFF7D0FFE06820F4405040F01000E06001
:101EB000A06AA0612069E062606044F24001E068CD
:101EC0008843E06010BD00001000020070B50446B9
:101ED00000F14C05284601F0DCFC204622F02CFAEB
:101EE0000446284620F0FEFA204670BD70B516461E
:101EF0000C460546FFF70AFA036893F8010101282A
:101F000006D0FF2C0FD8185D68B101202C7070BD71
:101F1000D3F807013246214603F20713034428464B
:101F2000BDE8704018474FF0FF3070BD10B500207D
:101F300000F0ACFCFEF794FABDE81040012000F080
:101F400089B82DE9F0410646FFF7EDF98046454690
:101F500013E016B1E068B0420ED120682860D4E9E1
:101F60000101D8F800708847204601F0A1FCD8F89C
:101F70000000B842EBD100E025462C68002CE8D1E7
:101F8000BDE8F08110B501F006FDBDE8104001F09C
:101F900007BD00002DE9F04115460E46040002D1B0
:101FA0002C6804B90BA4204601F0FFFC04442078FF
:101FB00070B127463146384600F076FC044420785C
:101FC00010B1002004F8010B38462C60BDE8F08108
:101FD0000027F9E700000000431A28BF9A4241F2A7
:101FE0006C84104410F0030F11441EBF11F8013D22
:101FF000521E00F8013D10F0030F7FF4F6AF103AC7
:10200000C0F00A8010B531E91850103A20E9185094
:10201000BFF4F9AFBDE81040530724BF31E9081001
:1020200020E9081044BF51F8043D40F8043D12F087
:10203000030F08BF7047D20728BF31F8023D48BFE1
:1020400011F8012C28BF20F8023D48BF00F8012CF0
:102050007047000001491820ABBEFEE726000200D1
:1020600030B5B0F10A024FEA900E71F100034EEA6A
:10207000817EB0EB0E0061EB91014FEA101E4EEA3B
:10208000017E10EB0E0041EB11114FEA102E4EEACB
:10209000016E10EB0E0041EB11214FEA104E4EEA9B
:1020A000014E10EB0E0041EB1141401841F10001CF
:1020B0004FEAD00040EA41704FEAD10110EB8005B1
:1020C0004FEA810444EA907444EB01046D1944EB37
:1020D0000404521BA3414FF0000348BF0A3200D54D
:1020E00030BD401C41F1000130BD00002DE9F34F2F
:1020F0004FF0000A0C4656468DB001200C9001F1BD
:102100000C000B9062690B9801219047051E2DD0A1
:10211000252D2CD0216A8847C0B162690B98012116
:102120009047216A88470028F7D16269411E0B98C1
:10213000904700E0761CA1690D988847216A88477E
:102140000028F7D1E1690D988847DBE7A1690D9870
:102150008847A842074601D1761CD3E7E1690D986C
:1021600088477F1C02D1BAF1000F6FD06BE1626922
:102170000B9800273D46394690472A2804D16269CA
:102180000B98012190470125DFF8D08262690B98F6
:1021900001219047A0F130010A290AD24745E5DC28
:1021A00007EB870100EB4107303FDFD445F0100516
:1021B000ECE7E90601D46FF000476C280AD04C2800
:1021C00014D0682815D06A280DD074281CD07A281D
:1021D0001AD01DE062690B98012190476C2802D04B
:1021E00045F0040514E045F002050DE045F020053A
:1021F0000AE062690B9801219047682802D045F0F7
:10220000080505E045F4006562690B9801219047D7
:10221000C4E9015765283DD019DC58287AD00CDC78
:10222000452837D004DC252826D041289ED131E02E
:1022300046282FD0472899D12CE05B2877D06128F9
:1022400028D063287CD0642823D15AE0F6E06F2898
:1022500048D008DC66281DD067281BD0692821D00B
:102260006E2816D127E0702845D0732868D07528CD
:1022700047D078280DD14DE0A1690D9888472528D1
:1022800005463FF469AFE1690D9888476D1C3FF43E
:102290006AAFD8E00D9923466A466FF0010030F02E
:1022A0008EF9C5E045F0400023464FF00002606023
:1022B000A80736D43EE0E8077FF447AF2068011D49
:1022C00021600068290501D506701BE7290701D5A3
:1022D000068017E7A90703D5F117C0E9006111E7E8
:1022E00006600FE745F0400023464FF008026060AB
:1022F000A80716D41EE040F60E0125EA0100606032
:1023000016E045F0400023464FF00A026060A8073F
:1023100007D40FE045F040006060A80708D52346C9
:1023200010220D996FF0010001F044FB80E007E0FE
:10233000102223460D996FF00100FEF7BBFC77E0F9
:102340004FF0000963284F46C8464B46CB4602D0A3
:102350005B2806D038E0E80601D40120A060012700
:1023600032E06269D4F80CB00B98012190475E28E6
:1023700007D14FF0010949466269D4F80CB00B98B7
:102380009047216939B900210A4603AB43F821205F
:10239000491C0829FADBD8B3216949B308F10108BF
:1023A00062690B98012190475D28F4D1B9F1000FC3
:1023B00009D0002003A951F82020D24341F8202061
:1023C000401C0828F7DB03AB2069002820794FEA7E
:1023D00040701ED05B462246CDF80080CDE90197C3
:1023E0000D9900286FF0010020DA00F0A9F81FE035
:1023F000C11703AA00EBD1614B1121F01F0102EBC1
:102400008302411A13680120884003431360C7E721
:1024100019E00D99224600286FF00100009702DABA
:1024200001F0CDFA04E000F01BF801E001F0CCFA75
:1024300000280ADA401C06D10C9820B14FF0FF307A
:102440000FB0BDE8F08F5046FAE7E90701D10AF175
:10245000010A064400200C9054E60000CCCCCC0CC1
:102460002DE9FF5F4FF000089946144646469169F2
:10247000D2E901A7DDF838B001988847054659EA46
:102480000B0005D009E0A1690198761C8847054634
:10249000216A284688470028F5D1681C03D05FEAE6
:1024A000CA7005D015E04FF0FF3004B0BDE8F09FD2
:1024B0002068011D2160D0F800800AE05FEACA7040
:1024C00001D108F8015BA169761C01987F1E88473D
:1024D0000546002F1ADD681C18D0B9F1000F0DD089
:1024E000E81705EBD060421120F01F0059F82210C8
:1024F0002A1A012090400142E0D107E0BBF1000F11
:10250000DCD12846216A88470028D7D0E1690198A4
:102510008847BBF1000F07D1002E05DD5FEACA70C6
:1025200002D1002188F80010A068B84203DDBBF199
:10253000000F03D017B16FF00100B6E73046B4E7E3
:102540002DE9FF5F9B46144600273D469169D2E97D
:102550000196DDF840A00198884780465BEA0A00B2
:1025600005D009E0A16901986D1C88478046216A61
:10257000404688470028F5D1B8F1FF3F03D05FEA15
:10258000C97005D014E04FF0FF3004B0BDE8F09FF3
:102590002068011D216007680AE05FEAC97001D167
:1025A00027F8028BA1696D1C0198761E884780462A
:1025B000002E15DDB8F1FF3F12D0BBF1000007D0AF
:1025C0004346DDE90E1201F004FA0028E5D107E0E8
:1025D000BAF1000FE1D14046216A88470028DCD0DB
:1025E000E16901988847BAF1000F05D1002D03DD9C
:1025F0005FEAC97000D13880A068B04203DDBAF14B
:10260000000F03D016B16FF00100BEE72846BCE70B
:1026100070B50D4601461446D36850692A4601F04C
:10262000DDF9002807DA411C07D0E16820F00040FE
:1026300041F48041E160281A70BD2046FFF7CEFBCF
:102640004FF0FF3070BDC1680022026021F480515C
:1026500041F0400111F4C06FC16001D08260704749
:1026600002694168891AC269891A816070472DE937
:10267000F0470446C06840F48000E060010312D5D2
:1026800020F40020E060810606D4E26A61688A4294
:1026900000D80A46511A216040F40010E06094F816
:1026A0002500BDE8F08720F40010E060800602D528
:1026B0002046FFF7EAFBE06842F281014FF0FF3964
:1026C0000140012903D02046FFF788FBB6E02168CE
:1026D000002600290ADAC94340F480502160C4E989
:1026E00002606068411C61600078DAE744F24001F2
:1026F00008420CD020F4A04040F040002660E0608A
:1027000021696068401AE169401AA06096E0216979
:1027100091B9C00310D4E069FDF7EBFF2061B0B1BF
:10272000E06840F4006010F4407FE06002D140F4C3
:102730008070E06020696060E068D4F814A0C10691
:102740001AD5C0030ED52046FFF77CFB14E004F138
:10275000240020610120E061E06820F4407040F432
:102760008060E6E721696068401AA169014450462B
:102770001FF0DBFE0028A6DBE068C0032AD56168F5
:10278000E06A884200D808462169451AE069471B7B
:102790001BD02046D4F81880FFF754FB08EB050146
:1027A0005046C4F818801FF0C0FE00288BDBE0689C
:1027B00040F40030E060000202D5A0692844A06126
:1027C000E1692069C91B45180DE02046FFF73AFB77
:1027D000E769F5E725696168D4E90607491BE56201
:1027E00008446560A061E06820F0100010F4C06F3C
:1027F000E06002D0204600F0F3FAE06840F4805038
:10280000C4E90260000205D52069E06260606FF0F3
:10281000010046E7224639462846FFF7F9FE411CEB
:102820000CD02918E16258B1401E2060681C60601D
:10283000E06840F40030E060287832E7484630E74E
:1028400065602046FFF7FFFEF8E7000070B504461C
:102850000D4D284601F01DF803E001F06AF8401C18
:102860000ED0094914F8010B4C390028F5D10A2083
:1028700001F05FF8044628461FF034FE204670BD84
:102880004FF0FF34F7E7000084EF002010B501F0AF
:10289000AAF8BDE8104001F083B810B500F006FBBF
:1028A000BDE8104001F07CB830B503461D781DB17D
:1028B0000A4603E0AC4201D1181A30BD12F8014BB0
:1028C000002CF7D15B1CF1E710B501F091F801691C
:1028D00019B100220261884701E080688047FFF754
:1028E00025FB00002DE9FF4F064689B00878FF2838
:1028F00006D0491C2D2805D000244FF0000908E01F
:1029000000200CE00124F8E709EB8903491C00EBE7
:1029100043090878FF28F7D114B1C9F100008146B6
:10292000107800252C46AA4629462D2801D02B28B0
:1029300004D1521C2D2813D0002082468B461078DB
:10294000FF280FD04FF0000C0A21521CA5FB017884
:1029500004FB018105FB0C11C5194BEB0104EEE7EB
:102960000120EAE7002108464FF00000BAF1000F0D
:1029700002D000EB80004008C0F38158B8F1010F8D
:1029800001DD4FF0FF380C9809EB000755EA040011
:1029900009D04FF0020917F5FA7F0BDA4FEACA7037
:1029A000C6E900B012E04FEACA70C6E900B00DB047
:1029B000BDE8F08FB7F5FA7F0DDDF0487844D0E937
:1029C0000010C6E9001040EACA70706000F098FF7D
:1029D000C0F80090EBE7391E02DAC8F1000200E00F
:1029E000424600DA794206A800F0C6FF06AB93E83B
:1029F000070003AB83E8070044F23E005BEA0401F2
:102A00000090584604D144F21E012C465D460091C8
:102A1000210C0904014306D10099240444EA154419
:102A20002D041039009104F07F41014306D1009933
:102A3000240244EA15642D020839009104F0704123
:102A4000014306D10099240144EA15742D01091FA0
:102A5000009104F04041014306D10099A40044EAEA
:102A60009574AD00891E009104F00041084304D123
:102A700000986D196441401E009042466846002F40
:102A8000CDE9014503A902DD00F0B7FF01E000F048
:102A9000A9FEBAF1000F04460D4601D084F00044AF
:102AA00040F2FF7724F00040284303D0C4F30A50DB
:102AB000B84212D100F024FFC0F80090C4F30A50CD
:102AC000B8420AD1AE487844D0E90010C6E90010F7
:102AD00004F000410843706069E7C6E9005466E706
:102AE0002DE9FF4F1F464FF0000A4FF0FF384546D3
:102AF00091B0D7E90146CDF83CA000F038FFC0689E
:102B00000168405C1090B96912986D1C8847396A59
:102B1000814688470028F6D1B9F1FF3F0AD0002E40
:102B200024F4D06411DDB9F12B0F08D0B9F12D0FC9
:102B30000BD102E0404615B03AE744F48064B9692D
:102B400012986D1C8847761E8146600504A901D540
:102B50002D2000E02B20002E01F1010B0DF130089B
:102B60008DF810003FDDB9F1690F08D0B9F1490FB8
:102B700005D0B9F16E0F02D0B9F14E0F1CD13B4612
:102B800001A8009580E85002DDE912126FF0020002
:102B900000F038FFC11CCED10EE0B96912986D1C4F
:102BA000884781461398761E44F4007405600F9898
:102BB000401C002E0F9016DDB9F1300FEDD0B9F1A9
:102BC000780F02D0B9F1580F0DD10F9801280AD112
:102BD0003B46CDE90054DDE91212001F029600F0D9
:102BE00016FFC11CA7D1109989453ED144F080043D
:102BF00006E01399681CAAF1010A44F40074086005
:102C0000B9696D1C1298761E884730288146F0D02D
:102C10002BE01099894505D1200603D4761E44F097
:102C2000800418E0484600F061FE08B3761E0DF1FE
:102C300023018B4544F4007408D2A9F130000BF84D
:102C4000010B200607D5AAF1010003E0200602D4FB
:102C50000AF101008246A00502D51399681C08609C
:102C6000B96912986D1C88478146002ED1DC53E06B
:102C7000002E51DDB9F1650F02D0B9F1450F4BD1EE
:102C8000A00549D5B9696D1C1298761E24F44074CC
:102C90008847002E81460CDD2B2804D0B9F12D0F7A
:102CA00007D144F48074B96912986D1C8847761E68
:102CB0008146E00501D52D2100E02B2108F8011BFC
:102CC000CDF8008021E0761E0DF13901884544F4ED
:102CD00000740CD2A9F1300010F0FF0088F8000059
:102CE00002D10099884509D908F1010806E0E005FC
:102CF00001D5244801E042F20F708246B96912986A
:102D00006D1C8847814613980560002E04DD4846F7
:102D100000F0ECFD0028D6D1F96912988847FF2011
:102D200053468BF8000088F8000000200A900B90B2
:102D300004AA0CA90AA8FFF7D5FDA00502D46FF0DC
:102D40000100F8E614F0240F0AD0E00714D1386827
:102D5000DDE90A12031D3B600068C0E900120BE0C8
:102D60000AA968461EF080FDE00705D13868009A80
:102D7000011D3960006802602846DCE610DB0401B2
:102D800006DA0401F1D8FFFF2DE9F04104461746A9
:102D90000D4602F14C00804600F07BFD012D2646D9
:102DA00016DD384621F0C8FA411C0FD0C0B20A28FF
:102DB00004F8010B02D06D1E012DF2DC0020207002
:102DC00040461FF08FFB3046BDE8F081B44201D190
:102DD0000026F5E7387B0006F0D50026EEE7000078
:102DE0002DE9F04707461348814600F052FD124C8A
:102DF00040F2022817E094F85000C00710D0BC42FF
:102E00000ED004F14C05284600F043FDE668284644
:102E10001FF068FB38EA060002D1204600F0FCFDF6
:102E2000206D20F00104002CE5D148461FF05AFB2C
:102E3000BDE8F08720020020A065001070B516469E
:102E40000C460546FEF762FA036893F80101012873
:102E500004D0185D68B101202C8070BDD3F8030147
:102E60003246214603F2031303442846BDE870406E
:102E700018474FF0FF3070BD10B5014602A000F0BA
:102E8000D0FD012010BD0000534947525452454423
:102E90003A2052656469726563743A2063616E27F3
:102EA00074206F70656E3A200000000010B5012894
:102EB00005D0002103A000F0B4FD012010BD09A140
:102EC000F8E7000053494752544D454D3A204F759D
:102ED00074206F662068656170206D656D6F727912
:102EE000000000003A2048656170206D656D6F72CA
:102EF0007920636F727275707465640000DE2DE96D
:102F0000F04117460E46054633B107FB0354E41B58
:102F10002046B047A542FAD1A5F10800BDE8F081EE
:102F20002DE9FF4F1F464FF03C0987B04FF000429C
:102F3000DDE9141001F10108DDF858A002EA405063
:102F40000390002005908346054604460490B96925
:102F5000461E08988847AAF1010A0290BAF1000FAC
:102F60003BDD02982E2815D0102100F0C4FC00286B
:102F70002EDB4FF0010B0599014317D0B9F1000F7B
:102F80000BDB4A46C117FDF7AAFC05430C43A9F128
:102F9000040905E0012004900BE008B145F00105AB
:102FA00001200590049820B9361D02E0049800B174
:102FB000361FB969089808F101088847BBF1000F6E
:102FC000AAF1010A0290C9D00999C1F80080C5E7A9
:102FD0000298702808D0502806D0F96908988847C8
:102FE000BBF1000F14D04FE0002002900120BBF194
:102FF000000F049009D0B969089808F101088847C2
:10300000AAF10109B9F1000F07DCF96908988847AE
:103010006FF001000BB0BDE8F08F2B2804D02D28F5
:103020000CD14FF0FF300490B969089808F10108FD
:103030008847A9F10109B9F1000FE6DD411CE4D090
:103040000A2100F058FC0028DFDB029908F1010892
:1030500001EB810100EB41000290B96908988847B3
:103060000A2100F048FC099AA9F10109B9F1000F01
:10307000C2F8008001DD0028E7DAF969089888477E
:103080000499029800FB016655EA040004D004F09C
:103090004041090002D006E0039898E0A40044EA09
:1030A0009574AD00B61E04F00041080002D16D1900
:1030B0006441761E159810F0240F03D04FF00B09D1
:1030C0005C4803E04FF028096FF07D0082465645CA
:1030D00007DAAAEB06018944B9F1410F01DD4FF08F
:1030E000410901200021A9F10102FDF7F8FB024688
:1030F00028400B462140084301D0012100E0002177
:10310000501E029143F1FF3128402140084301D075
:10311000012000E000200299834651EA0B014FD0C4
:10312000002108464FF00000039900F4400039B137
:1031300000EB80004FF4400100EBD07001EA60002A
:103140008015012802DD4FF0FF3000E013D0401C55
:1031500036D0029860B3BBF1000F0CD14A46012073
:103160000021FDF7BCFB28402140084301D001208D
:1031700000E00020E0B101204A460021FDF7AFFB4E
:10318000034640190A4661412D1A8C4111D3B9F109
:10319000400F09DD159810F0240F02D0AAF1340673
:1031A00003E0AAF1170600E0761C00254FF000446A
:1031B00006E05B1E42F1FF3220EA030521EA020429
:1031C000CAF10100B04206DA1B4903980843019096
:1031D000002000900EE0039AC4F3D321E80A0A43CA
:1031E000164940EA44500A433146CDE90002684698
:1031F0001FF03EF8159810F0240F0BD01598C0075B
:1032000015D13868DDE90012031D3B600068C0E994
:1032100000120CE002A869461EF026FB1598C007B4
:1032200005D13868029A011D396000680260404685
:10323000F0E6000002FCFFFF0000F07F0000F03F1E
:103240002DE9FF4F92461D4685B04FF00041DDE964
:10325000124BDDE914727F1E01EA4B50414940F0E8
:10326000FF4940EA0108002122F02000492804918A
:1032700002D04E2828D04CE03BA0012607C88DE89C
:103280000700A9690698641C88477F1E014606D47A
:103290001DF8060018B121F0200181420BD0E96928
:1032A00006988847032E34D0082E32D06FF00100E4
:1032B00009B0BDE8F08F761C032E01D0082EE0D1B6
:1032C000601CCAF80000DCE7A9690698641C8847FE
:1032D0007F1E2AD420F02000412826D1A969069813
:1032E000641C88477F1E20D420F020004E281CD16B
:1032F000A9690698641C88477F1E48F4002849F491
:103300008009CAF8004001D4282806D0E969069847
:1033100088475FEACB7012D022E0A9690698641C46
:1033200088477F1E01D4002803DAE9690698884798
:10333000BCE72928F1D1641CCAF80040E9E71BF07A
:10334000240F07D028680499031D2B600068C0E98A
:10335000001805E02868021D2A600068C0F8009087
:103360002046A5E70000F07F494E46494E49545992
:10337000000000002DE9F04116461F460C46851B53
:1033800002E02846B847AD1B641EFAD2BDE8F081C2
:103390005FEA400C08BF91F0000F4FEA8C234FEA20
:1033A000C12243EA51514FEA1C5018BF00F5F040CA
:1033B0004FEA300018BF41F000415FEA6C5C00F05A
:1033C0000680BCF1FF3F08BF40F08040704711F01D
:1033D000004F08BF704731F0004100F027830B0C0D
:1033E00006BF09044FF0100C4FF0000C0B0E04BF89
:1033F00009020CF1080C0B0F04BF09010CF1040CBD
:103400008B0F04BF89000CF1020CCB0F04BF4900E5
:103410000CF1010CCCF12003A0EB0C0022FA03F319
:1034200002FA0CF241EA030100F10100704720F0BA
:103430007F4C80EA030023F07F47ACEB070303F5E2
:103440007C5300F0004003F1FF032DE980494FEA6F
:10345000154B09B44FEA144325EA0B4E24EA0348FE
:103460000FF2042606EB132749083E785FEA320282
:1034700003FB0667C7F5000707FB06F64FEA54375C
:103480004FEAD64606F1020607FB066CCCF1005C5B
:103490004FEA1C472CEA074C07FB06F40CFB06F529
:1034A00004EB15464FEA961634BF00204FF000405B
:1034B0004FEAD13706FB07FC4FEA1C4C0CFB0BF71D
:1034C000D21B03FB0CF761EB07010CFB0EF7B0EB13
:1034D000074072EB17420CFB08F734BFA2EB074220
:1034E000B2EB074261EB17414FEA0C444FEA9107F8
:1034F00006FB07FC4FEA1C4C0CFB0BF7B0EBC7407C
:1035000072EB573203FB0CF734BFA2EBC742B2EBAE
:10351000C74261EB57310CFB0EF7B0EBC70072EB03
:1035200057720CFB08F734BFA2EBC702B2EBC7021D
:1035300061EB5771039F4FEA816141EA921104EBFD
:10354000CC044FEAD1374FEA826206FB07FC42EA1D
:1035500090124FEA80604FEA1C4C0CFB0BF7D21B19
:1035600003FB0CF761EB07010CFB0EF7B0EB074018
:1035700072EB17420CFB08F734BFA2EB0742B2EB29
:10358000074261EB17414FEA8C554FEA910704EB74
:103590009C2406FB07FC4FEA1C4C0CFB0BF7B0EB22
:1035A000C74072EB573203FB0CF734BFA2EBC742A4
:1035B000B2EBC74261EB57310CFB0EF7B0EBC70023
:1035C00072EB57720CFB08F734BFA2EBC702B2EBE9
:1035D000C70261EB577115EB4C254FEA816141EA57
:1035E00092114FEA82624FEAD13742EA901206FB0B
:1035F00007FC44F100044FEA80604FEA1C4C0CFBCE
:103600000BF7D21B03FB0CF761EB07010CFB0EF76A
:10361000B0EB074072EB17420CFB08F734BFA2EB8C
:103620000742B2EB074261EB174115EB1C154FEA5D
:10363000813141EA92414FEA823242EA90424FEAB6
:1036400080304FEA0C7644F1000448EA03434EEA26
:103650000B484FF0000EB2EB080C71EB030724BFD0
:10366000624639464EEB0E0E4FF0000B00185241E9
:1036700049414BEB0B0BB2EB080C71EB03077BF1F1
:10368000000B24BF624639464EEB0E0E4FF0000B86
:103690000018524149414BEB0B0BB2EB080C71EB9C
:1036A00003077BF1000B24BF624639464EEB0E0E3A
:1036B00051EA020718BF46F0010616EB0E7655F1E7
:1036C000000254F1000103D5BDE88901BDE800887E
:1036D000BDE88901BDE80048B619524141EB01013E
:1036E000A3F10103704780807F7E7D7C7B7A7978AF
:1036F000777676757473727171706F6E6E6D6C6CB7
:103700006B6A6A6968686766666564646363626158
:103710006160605F5F5E5E5D5D5C5C5B5B5A5A59D9
:103720005958585757565655555554545353525245
:103730005251515050504F4F4F4E4E4D4D4D4C4C9D
:103740004C4B4B4B4A4A4A494949484848474747E6
:103750004746464645454544444444434343434223
:10376000424242414141000046EA0646A3F57053F9
:103770004FEA164646EA42564FEAD22242EA415200
:1037800010B54FEAD121A3F1010300F054F920F064
:10379000004000F1010C00F0004701EB0050114621
:1037A000BCF5006F40EA070000D210BD02484FF0A0
:1037B000000140EA070010BD0000F07F2DE9C0487D
:1037C000934630B491E8380007C831EA400C48BF4E
:1037D00034EA430C03D5FFF72AFE00F02CF9F0BCC5
:1037E000BDE800882DE9C048934630B491E8380020
:1037F00007C831EA400C48BF34EA430C03D5FFF751
:1038000016FEFFF7B1FFF0BCBDE800880000000025
:1038100040F2373CC1F6003C60474AF6D95CC1F63D
:10382000013C604740F20F3CC1F6003C604740F667
:10383000AD2CC1F6003C604740F22B3CC1F6003C89
:10384000604740F6952CC1F6003C604740F6A52C39
:10385000C1F6003C604740F6155CC1F6003C60478D
:1038600041F2675CC1F6003C604740F2010CC1F6D2
:10387000003C604740F2490CC1F6003C604740F212
:10388000F55CC1F6003C604747F2AD5CC1F6013C17
:10389000604741F6C95CC1F6013C604740F6731CC5
:1038A000C1F6003C604740F2990CC1F6003C60470D
:1038B00040F2FB0CC1F6003C604740F2E37CC1F6ED
:1038C000003C604740F6F16CC1F6003C604740F6B2
:1038D000352CC1F6003C604740F2D91CC1F6003CD3
:1038E000604740F2EB1CC1F6003C604741F6BB5C10
:1038F000C1F6013C604740F6293CC1F6003C6047F8
:1039000040F26D0CC1F6003C604740F2893CC1F6C4
:10391000003C604741F63F6CC1F6013C604740F215
:10392000F93CC1F6003C604741F6156CC1F6013C1C
:10393000604743F6153CC1F6013C604740F23F4CFE
:10394000C1F6003C604741F6656CC1F6013C60473A
:1039500040F69B0CC1F6003C604741F6E95CC1F6BD
:10396000013C604740F2351CC1F6003C604740F620
:10397000156CC1F6003C604741F2852CC1F6003C55
:10398000604741F6652CC1F6003C604740F6716C1B
:10399000C1F6003C604741F2C14CC1F6003C6047B3
:1039A00041F2A94CC1F6003C604741F2F14CC1F62E
:1039B000003C604740F6317CC1F6003C604741F274
:1039C000870CC1F6003C604741F29B1CC1F6003CED
:1039D000604741F2BB5CC1F6003C604741F6D16CE8
:1039E000C1F6013C604741F6ED0CC1F6003C604772
:1039F00041F21B5CC1F6003C604741F68D2CC1F6DC
:103A0000003C60474AF63D6CC1F6013C60474AF60F
:103A1000396CC1F6013C604740F2ED4CC1F6003C08
:103A2000604741F6B90CC1F6003C604741F6591CAD
:103A3000C1F6003C604741F69F1CC1F6003C604760
:103A400049F6D97CC1F6013C604743F2C93CC1F656
:103A5000003C604743F28D5CC1F6003C604743F296
:103A6000996CC1F6003C604743F6816CC1F6003C9E
:103A7000604744F6C54CC1F6003C604741F2F12C6A
:103A8000C1F6013C604741F20D3CC1F6013C604784
:103A900043F6491CC1F6003C604740F6570CC1F69E
:103AA000003C604743F69D1CC1F6003C604741F274
:103AB000D52CC1F6013C604746F6556CC1F6013C79
:103AC000604746F6956CC1F6013C604744F2111C14
:103AD000C1F6003C604744F2752CC1F6003C6047DB
:103AE00044F27D2CC1F6003C604744F2495CC1F6CB
:103AF000003C604744F6850CC1F6003C604744F644
:103B0000954CC1F6003C604741F2273CC1F6013CB0
:103B1000604746F68D3CC1F6013C604744F2250CF7
:103B2000C1F6013C604744F28D0CC1F6013C604790
:103B300042F2897CC1F6013C604745F2AD2CC1F6EA
:103B4000003C604745F2113CC1F6003C604745F23D
:103B5000455CC1F6003C604745F6590CC1F6003C97
:103B6000604743F6355CC1F6003C604743F6655C50
:103B7000C1F6003C604745F2497CC1F6003C604715
:103B800043F6316CC1F6003C604746F29D7CC1F6BD
:103B9000003C604746F2A50CC1F6003C604745F684
:103BA000414CC1F6003C604740F2D56CC1F6003C88
:103BB000604747F6612CC1F6003C604746F2E53CA1
:103BC000C1F6003C604746F2695CC1F6003C6047C4
:103BD00046F6491CC1F6003C604747F26D0CC1F641
:103BE000003C604746F6D13CC1F6013C604747F2D5
:103BF000450CC1F6003C604746F6091CC1F6003C86
:103C0000604746F6453CC1F6003C604740F2911CD7
:103C1000C1F6003C604747F6512CC1F6003C6047B6
:103C200047F6452CC1F6003C604746F6054CC1F608
:103C3000003C604746F25D7CC1F6003C604747F6B9
:103C40000F2CC1F6003C604746F6E92CC1F6003C5B
:103C5000604747F6052CC1F6003C604746F6635CBA
:103C6000C1F6003C604747F2D97CC1F6003C604792
:103C700047F6510CC1F6003C604746F6397CC1F668
:103C8000003C604746F66F5CC1F6003C604746F674
:103C9000755CC1F6003C604745F6074CC1F6003C38
:103CA000604746F2BD1CC1F6003C604746F20D2C51
:103CB000C1F6003C604746F2752CC1F6003C6047F7
:103CC00046F6951CC1F6003C604745F6295CC1F6F6
:103CD000003C604746F6695CC1F6003C604747F22D
:103CE000411CC1F6003C604746F6615CC1F6003CF1
:103CF000604746F6417CC1F6003C604746F2A92C7D
:103D0000C1F6003C604746F6914CC1F6003C604766
:103D100046F64D4CC1F6013C604746F67D4CC1F677
:103D2000013C604744F6794CC1F6003C604748F2DC
:103D3000793CC1F6003C604749F20B2CC1F6003CCF
:103D4000604747F64D5CC1F6003C604747F6215C92
:103D5000C1F6003C604748F2DD1CC1F6003C6047FC
:103D600047F61D4CC1F6003C604749F2312CC1F6C4
:103D7000003C604747F6095CC1F6003C604748F2EA
:103D8000850CC1F6003C604747F6655CC1F6003C17
:103D9000604748F6613CC1F6003C604748F6515C1C
:103DA000C1F6003C604748F6415CC1F6003C604704
:103DB00048F6F96CC1F6003C604748F6193CC1F67C
:103DC000003C604748F2455CC1F6003C60474EF25B
:103DD000153CC1F6003C604748F27F6CC1F6003CE0
:103DE000604748F6E16CC1F6003C604740F2791C40
:103DF000C1F6003C604746F2217CC1F6003C6047BA
:103E00004DF61D3CC1F6003C60474EF2411CC1F628
:103E1000003C604749F2BF5CC1F6003C604749F294
:103E2000A55CC1F6003C60474BF2690CC1F6003C52
:103E300060474BF2BB0CC1F6003C604749F6D30C1F
:103E4000C1F6013C60474BF2510CC1F6003C6047A3
:103E500049F6412CC1F6013C604748F2954CC1F649
:103E6000013C604749F27D6CC1F6003C604749F275
:103E7000756CC1F6003C604743F2B12CC1F6003CC2
:103E8000604748F6692CC1F6003C60474BF2F74C9E
:103E9000C1F6003C60474BF2CF3CC1F6003C6047A6
:103EA0004BF2C93CC1F6003C60474BF2075CC1F6DF
:103EB000003C60474BF2D53CC1F6003C604747F6FA
:103EC000A14CC1F6003C604749F2912CC1F6003C80
:103ED000604748F6F11CC1F6003C60474DF68D3C4A
:103EE000C1F6003C604741F2C93CC1F6003C604766
:103EF0004DF64D3CC1F6003C60474DF6490CC1F60D
:103F0000003C60474DF6850CC1F6003C60474DF61D
:103F10002D0CC1F6003C604747F6D17CC1F6003C51
:103F2000604740F6E90CC1F6003C60474DF2F57C75
:103F3000C1F6003C604740F28D4CC1F6003C604742
:103F400041F2B50CC1F6013C60474DF60D0CC1F6CF
:103F5000003C604749F2A54CC1F6003C60474AF678
:103F6000090CC1F6003C604749F2495CC1F6003CCF
:103F7000604740F6470CC1F6013C60474AF2CD7CF1
:103F8000C1F6013C60474EF2091CC1F6003C604797
:103F90004DF6256CC1F6003C604740F2857CC1F6C9
:103FA000013C60474DF6997CC1F6003C604740F209
:103FB000D17CC1F6013C604740F6510CC1F6013C92
:103FC000604749F2C75CC1F6003C60474EF6FD7C95
:103FD000C1F6003C60474DF6A97CC1F6003C604745
:103FE0004CF69D7CC1F6003C604740F63B0CC1F6A8
:103FF000013C604746F6D94CC1F6013C604748F2A7
:104000004D3CC1F6003C60474EF2CD0CC1F6003C81
:10401000604748F2D97CC1F6003C60474BF2E54C62
:10402000C1F6003C60474BF2910CC1F6003C604782
:1040300049F6A32CC1F6003C60474AF6DD7CC1F688
:10404000003C604749F2695CC1F6003C60474CF2B5
:10405000755CC1F6003C604749F64D2CC1F6003C4A
:1040600060474BF68D3CC1F6003C604740F2F57C62
:10407000C1F6013C604745F2BD2CC1F6013C6047EA
:1040800040F6B12CC1F6013C604740F64D2CC1F61C
:10409000013C60474AF23F5CC1F6003C604741F298
:1040A000553CC1F6013C604749F60D0CC1F6003C99
:1040B000604749F6453CC1F6003C604748F22D3C5C
:1040C000C1F6003C60474CF6490CC1F6003C604725
:1040D00049F69D4CC1F6013C60474EF2910CC1F689
:1040E000003C604749F2815CC1F6003C60474AF2FF
:1040F000795CC1F6013C604740F2FD7CC1F6013CB1
:1041000060474DF65D7CC1F6003C604740F6F92CF7
:10411000C1F6013C604740F6613CC1F6013C604796
:1041200048F2193CC1F6013C604748F27D2CC1F6CB
:10413000013C604741F2BD0CC1F6013C60474CF6C2
:10414000214CC1F6003C604749F2774CC1F6003C77
:10415000604749F68D4CC1F6003C604749F6E52CB6
:10416000C1F6003C60474EF2F10CC1F6003C6047DE
:1041700049F6CB0CC1F6013C60474EF27D2CC1F6EE
:10418000003C60474EF2F52CC1F6003C60474EF211
:10419000513CC1F6003C60474AF2435CC1F6003C2A
:1041A000604749F6DF3CC1F6013C604748F27D4C70
:1041B000C1F6013C604740F6B92CC1F6013C6047AE
:1041C00048F2092CC1F6013C604748F2691CC1F66F
:1041D000013C60474AF2310CC1F6003C604740F2B6
:1041E000496CC1F6003C604740F2976CC1F6003C58
:1041F00060474AF2590CC1F6003C604740F2657CCA
:10420000C1F6013C604749F6711CC1F6013C6047AC
:1042100049F6311CC1F6013C604749F6891CC1F6DC
:10422000013C60474AF2E73CC1F6003C60474AF275
:10423000853CC1F6003C604740F26D7CC1F6013C14
:1042400060474AF21B2CC1F6003C60474EF2E91C65
:10425000C1F6003C60474AF2430CC1F6003C60479F
:1042600040F6233CC1F6013C60474BF6B53CC1F635
:10427000003C604749F6ED7CC1F6003C60474AF2DD
:10428000F91CC1F6003C60474AF6A51CC1F6003C8B
:10429000604749F6BF0CC1F6003C604749F63D7CDB
:1042A000C1F6003C604749F2A17CC1F6003C604782
:1042B00048F2F17CC1F6003C60474AF20B5CC1F663
:1042C000003C604740F6710CC1F6013C604740F687
:1042D000ED1CC1F6013C604740F6C90CC1F6013C3B
:1042E00060474AF2792CC1F6003C604749F63D3CF4
:1042F000C1F6003C604749F6793CC1F6013C604795
:104300004AF6853CC1F6003C604740F27D7CC1F630
:10431000013C604740F6192CC1F6013C60474BF662
:10432000B10CC1F6003C60474CF6BD3CC1F6003C08
:1043300060474AF2594CC1F6003C60474AF6AD3C32
:10434000C1F6003C60474AF6E13CC1F6003C6047DC
:104350004AF6ED5CC1F6003C604740F6470CC1F6FA
:10436000003C60474AF6BD4CC1F6003C604749F648
:10437000932CC1F6013C604749F6752CC1F6013C0F
:10438000604749F6072CC1F6013C604748F22D5CB6
:10439000C1F6013C604749F6DB0CC1F6013C6047C1
:1043A0004AF2E97CC1F6013C60474DF6ED7CC1F66E
:1043B000003C60474DF6DD7CC1F6003C60474DF6A1
:1043C000697CC1F6003C60474DF6757CC1F6003C47
:1043D00060474BF2E30CC1F6003C604749F6B72C4E
:1043E000C1F6003C60474AF6396CC1F6003C6047B4
:1043F00040F6330CC1F6013C604746F6C14CC1F6AD
:10440000013C60474DF2935CC1F6003C60474BF2C3
:10441000413CC1F6003C60474DF2695CC1F6003C8E
:1044200060474BF24F3CC1F6003C60474BF2C53C45
:10443000C1F6003C604740F25D7CC1F6013C60473C
:104440004AF2E10CC1F6013C604749F6813CC1F6F5
:10445000013C60474AF22D0CC1F6013C604741F235
:10446000CD4CC1F6013C60474BF2D17CC1F6003C1B
:10447000604740F2356CC1F6003C604746F64B7C25
:10448000C1F6013C604740F27D5CC1F6003C6047EC
:1044900048F62F5CC1F6013C604748F6E94CC1F68E
:1044A000013C60474BF2553CC1F6003C60474BF283
:1044B000993CC1F6003C60474CF2452CC1F6003CEB
:1044C00060474BF6391CC1F6003C60474BF6EF3CA9
:1044D000C1F6003C60474BF6651CC1F6003C6047E6
:1044E0004BF6C31CC1F6003C60474BF6D91CC1F625
:1044F000003C60474BF6DD1CC1F6003C60474BF6C4
:10450000F31CC1F6003C60474BF6F71CC1F6003CBB
:1045100060474BF6472CC1F6003C604745F2A31CB0
:10452000C1F6013C60474BF6A12CC1F6003C604748
:104530004BF64D3CC1F6003C60474BF6E95CC1F6DA
:10454000003C604749F6AB4CC1F6013C604749F678
:10455000654CC1F6013C60474AF2DF4CC1F6013CB4
:1045600060474DF6A16CC1F6003C604740F2995C93
:10457000C1F6013C60474AF2F74CC1F6013C604786
:104580004AF2E74CC1F6013C604749F65F0CC1F6C0
:10459000013C60474AF2AB5CC1F6013C604740F227
:1045A000996CC1F6013C604749F22F3CC1F6013CD1
:1045B000604749F21D3CC1F6013C604749F2A14CFD
:1045C000C1F6013C604749F6B34CC1F6013C604777
:1045D0004CF2652CC1F6003C604743F6CD1CC1F699
:1045E000013C60474CF69D0CC1F6003C604743F629
:1045F000615CC1F6013C604743F6215CC1F6013CB9
:1046000060474CF6611CC1F6003C604743F6751CE0
:10461000C1F6013C604743F63D2CC1F6013C6047C2
:104620004CF2752CC1F6003C60474AF2571CC1F6AB
:10463000013C60474AF2432CC1F6013C604749F215
:10464000397CC1F6013C60474CF6BD5CC1F6003CCC
:1046500060474AF2F92CC1F6013C60474AF2A32CAC
:10466000C1F6013C60474AF24B2CC1F6013C604761
:104670004AF2AB2CC1F6013C604748F2BD3CC1F6A2
:10468000013C60474CF6415CC1F6003C604749F292
:10469000A90CC1F6013C60474DF28B5CC1F6003CB1
:1046A00060474DF28F5CC1F6003C60474DF2E57CFF
:1046B000C1F6003C604749F2FB1CC1F6003C604774
:1046C00049F2C52CC1F6003C604741F2AD0CC1F681
:1046D000013C604748F6613CC1F6013C604741F24D
:1046E000994CC1F6003C60474AF63D0CC1F6013CCE
:1046F000604749F6E30CC1F6013C604747F6E17CB0
:10470000C1F6013C604748F22F0CC1F6013C6047FE
:104710004EF69D0CC1F6003C60474EF6DD3CC1F6FE
:10472000003C60474EF6AF1CC1F6003C60474EF6B9
:10473000716CC1F6003C60474EF6E12CC1F6003CBE
:1047400060474EF6C52CC1F6003C60474EF6573C1C
:10475000C1F6003C604740F2D92CC2F6000C60471D
:1047600040F28D1CC2F6000C60474FF6851CC1F666
:10477000003C604740F26D6CC1F6003C604748F277
:10478000D51CC1F6013C604749F6930CC1F6013CCB
:10479000604740F23B4CC1F6003C60474FF67D2C31
:1047A000C1F6003C60474AF2372CC1F6003C604736
:1047B0004AF2DB1CC1F6003C60474EF2112CC1F6F8
:1047C000003C604740F2710CC1F6003C60474EF27D
:1047D000393CC1F6003C60474DF6836CC1F6003CA5
:1047E000604741F2D95CC1F6003C60474EF67B6CF5
:1047F000C1F6003C60474EF6F12CC1F6003C604724
:104800004EF6DD4CC1F6003C60474EF63D3CC1F62D
:10481000003C60474BF6393CC1F6003C60474BF624
:104820004D2CC1F6003C604749F2951CC1F6003C96
:10483000604740F22D1CC1F6013C604740F2B50CC8
:10484000C1F6013C604740F2312CC1F6013C6047A3
:1048500040F2C51CC1F6013C604748F2D15CC1F68C
:10486000013C60474AF67D3CC1F6003C604740F29F
:104870009B4CC1F6013C604740F2796CC1F6013CAB
:10488000604740F2356CC1F6013C604741F27D3C27
:10489000C1F6013C604741F24F1CC1F6013C604744
:1048A00040F6073CC1F6013C604749F2D91CC1F60D
:1048B000003C604741F23D0CC1F6013C60474DF6BB
:1048C000755CC1F6003C604741F2090CC1F6013C41
:1048D000604748F6FB2CC1F6013C60474DF60D4C95
:1048E000C1F6003C604740F6E97CC1F6013C6047F8
:1048F00049F6A17CC1F6013C604740F6A15CC1F6D7
:10490000013C604740F65F4CC1F6013C604740F611
:10491000B96CC1F6013C60474DF2FD5CC1F6003C4C
:1049200060474DF2A35CC1F6003C604740F6F56C71
:10493000C1F6013C604740F6651CC1F6003C60478B
:1049400040F6152CC1F6003C604741F2976CC1F669
:10495000013C604747F6CD0CC1F6013C604741F28F
:10496000F97CC1F6013C60474AF2FB7CC1F6013C90
:1049700060474AF6ED2CC1F6013C60474AF6DD5C23
:10498000C1F6013C604741F2D97CC1F6013C604769
:1049900041F2C17CC1F6013C604741F2917CC1F615
:1049A000013C604741F6010CC1F6013C60474AF604
:1049B000795CC1F6013C604741F6110CC1F6013C3F
:1049C000604743F6314CC1F6013C604740F2076C4A
:1049D000C1F6003C604749F6695CC1F6003C60479F
:1049E00048F26D6CC1F6013C604746F6A53CC1F645
:1049F000013C60474CF6A14CC1F6003C604746F6CE
:104A0000214CC1F6013C60474EF6191CC1F6003C32
:104A1000604740F2D52CC1F6013C60474AF60D2CA8
:104A2000C1F6003C60474FF6517CC1F6003C604740
:104A300043F2010CC1F6013C604743F6B55CC1F698
:104A4000013C604743F2F53CC1F6013C604742F649
:104A5000915CC1F6013C604743F2D15CC1F6013C78
:104A6000604743F2211CC1F6013C604742F68D5C71
:104A7000C1F6013C604741F6055CC1F6013C604768
:104A800048F2D14CC1F6003C604748F2AD4CC1F64B
:104A9000003C604741F65D7CC1F6013C604741F651
:104AA000F97CC1F6013C604746F2E51CC1F6013CC9
:104AB000604742F6C51CC1F6013C604745F6E91C5B
:104AC000C1F6013C604742F23D7CC1F6013C6047C3
:104AD00042F6CF5CC1F6013C604743F6E92CC1F6D3
:104AE000013C604745F2755CC1F6013C604746F207
:104AF000D56CC1F6013C604742F2CD6CC1F6013C79
:104B0000604745F2A11CC1F6013C604746F6611CB6
:104B1000C1F6013C604743F6E10CC1F6013C604739
:104B200042F2014CC1F6013C604743F66D6CC1F6A0
:104B3000013C604743F2CD4CC1F6013C604742F670
:104B4000A75CC1F6013C604743F6F57CC1F6013C29
:104B5000604744F23B2CC1F6013C604744F2050C2F
:104B6000C1F6013C604744F20F0CC1F6013C6047BE
:104B700042F24D3CC1F6013C604743F6F15CC1F6A0
:104B8000013C604746F6D16CC1F6013C604746F6F1
:104B90007D5CC1F6013C604746F6AF5CC1F6013C66
:104BA000604744F69F1CC1F6013C604743F6D93C80
:104BB000C1F6013C604744F26B2CC1F6013C6047F2
:104BC00044F2F52CC1F6013C604743F2053CC1F6C6
:104BD000013C604742F6B35CC1F6013C604742F6D7
:104BE000136CC1F6013C604744F2F92CC1F6013C5C
:104BF000604747F6850CC1F6013C604742F6AF5C62
:104C0000C1F6013C604744F2D52CC1F6013C604737
:104C100042F6A35CC1F6013C604743F6195CC1F65D
:104C2000013C604743F6C55CC1F6013C604743F672
:104C3000BD4CC1F6013C604745F2653CC1F6013C04
:104C4000604744F2711CC1F6013C604747F20D1CFD
:104C5000C1F6013C604747F2754CC1F6013C604724
:104C600044F2C71CC1F6013C604744F2FF1CC1F688
:104C7000013C604749F6CF0CC1F6003C604749F65D
:104C8000615CC1F6003C604749F27B5CC1F6003CC8
:104C9000604749F6472CC1F6003C60474BF2F10CE7
:104CA000C1F6003C60474DF2497CC1F6003C6047CC
:104CB00047F2B54CC1F6003C60474EF2551CC1F6B8
:104CC000003C604749F6594CC1F6003C604746F647
:104CD000954CC1F6013C60474EF6AD6CC1F6003C08
:104CE000604747F62D4CC1F6003C60474AF6690C18
:104CF000C1F6003C60474CF2CD4CC1F6003C604729
:104D000049F2C90CC1F6003C604745F2093CC1F6C6
:104D1000013C604746F2457CC1F6003C604747F6DF
:104D2000852CC1F6003C604745F2253CC1F6013CAC
:104D3000604745F23D3CC1F6013C604744F2014CFE
:104D4000C1F6013C604744F2875CC1F6013C604714
:104D500044F2A35CC1F6013C604744F6510CC1F635
:104D6000013C604744F2CB6CC1F6013C604743F61E
:104D7000E55CC1F6013C604744F6810CC1F6013C9C
:104D8000604744F6970CC1F6013C604744F2FD6C65
:104D9000C1F6013C604744F6D50CC1F6013C6047C2
:104DA00044F2C93CC1F6013C604744F2A57CC1F61F
:104DB000013C604744F2DD7CC1F6013C604746F6A9
:104DC000E93CC1F6013C604742F26B6CC1F6013C24
:104DD000604745F2754CC1F6013C604745F2310C25
:104DE000C1F6013C604746F6654CC1F6013C6047A0
:104DF00046F2297CC1F6013C604742F6E16CC1F6FF
:104E0000013C604742F6797CC1F6013C604742F6BE
:104E1000416CC1F6013C604745F62D1CC1F6013CD2
:104E2000604746F2F16CC1F6013C604745F2813CB7
:104E3000C1F6013C604740F2650CC1F6003C60479A
:104E400046F2093CC1F6013C604746F2137CC1F6CC
:104E5000013C604746F6FD4CC1F6013C604746F216
:104E6000357CC1F6013C604740F24D3CC1F6003C48
:104E7000604742F2991CC1F6013C604742F2D50CF2
:104E8000C1F6013C604742F2A52CC1F6013C6047E7
:104E900042F2D91CC1F6013C604745F6E10CC1F66F
:104EA000013C604745F6F10CC1F6013C604740F219
:104EB0006D1CC1F6003C604745F2312CC1F6013C47
:104EC000604745F28D6CC1F6013C604746F2B93C43
:104ED000C1F6013C604745F2157CC1F6013C6047D4
:104EE00045F6792CC1F6013C604745F2B15CC1F64C
:104EF000013C604745F6596CC1F6013C604746F2FB
:104F0000C55CC1F6013C604746F6A51CC1F6013CF4
:104F1000604742F6F16CC1F6013C604742F60F7CF7
:104F2000C1F6013C604746F2414CC1F6013C604786
:104F300042F63D7CC1F6013C604745F6056CC1F682
:104F4000013C604742F6B94CC1F6013C604746F26D
:104F5000ED0CC1F6013C604745F6A97CC1F6013C69
:104F6000604745F2E94CC1F6013C604746F2F90C56
:104F7000C1F6013C604742F6E93CC1F6013C60479E
:104F800045F67D4CC1F6013C604744F2F90CC1F690
:104F9000013C604745F6514CC1F6013C604745F283
:104FA0009D4CC1F6013C604745F2155CC1F6013CE1
:104FB000604744F6C95CC1F6013C604744F6B55C05
:104FC000C1F6013C604744F6397CC1F6013C6047BC
:104FD00045F26D0CC1F6013C604744F6C56CC1F664
:104FE000013C604742F6D10CC1F6013C604747F6F0
:104FF000294CC1F6013C604747F6855CC1F6013C8F
:10500000604747F6816CC1F6013C604747F6257C56
:10501000C1F6013C604747F6656CC1F6013C60474C
:1050200045F28F5CC1F6013C604745F2815CC1F6F8
:10503000013C604742F69D2CC1F6013C604747F6B3
:10504000272CC1F6013C604744F24D1CC1F6013CDF
:10505000604747F6893CC1F6013C604744F6D12CD5
:10506000C1F6013C604744F6EB0CC1F6013C6047D9
:1050700044F6A91CC1F6013C604743F62F3CC1F63B
:10508000013C604742F2AD7CC1F6013C604742F60C
:10509000AB5CC1F6013C604745F6252CC1F6013CEE
:1050A000604747F2954CC1F6013C604747F2A90CB6
:1050B000C1F6013C604747F2DD4CC1F6013C604758
:1050C00047F2F14CC1F6013C604747F20D5CC1F676
:1050D000013C604746F6D57CC1F6013C604747F28B
:1050E000311CC1F6013C604742F6C10CC1F6013CDF
:1050F000604742F6910CC1F6013C604741F6755C91
:10510000C1F6013C604747F2F50CC1F6013C60472F
:1051100046F6455CC1F6013C604746F65D7CC1F64B
:10512000013C604747F6CD3CC1F6013C604747F281
:10513000D90CC1F6013C604747F6CD1CC1F6013CD5
:10514000604747F61D3CC1F6013C604747F2212C01
:10515000C1F6013C604747F2D10CC1F6013C604703
:1051600047F2652CC1F6013C604747F2253CC1F689
:10517000013C604747F2015CC1F6013C604747F2E1
:105180006D5CC1F6013C604747F2250CC1F6013C5D
:10519000604747F6090CC1F6013C604747F28D6C49
:1051A000C1F6013C604747F2810CC1F6013C604703
:1051B00047F2D15CC1F6013C604742F2D55CC1F6D2
:1051C000013C604743F6CD6CC1F6013C604749F6AF
:1051D000C91CC1F6013C604746F6014CC1F6013CD2
:1051E000604748F6DD2CC1F6013C604748F6D52CF7
:1051F000C1F6013C604748F6F52CC1F6013C60471A
:1052000048F6ED2CC1F6013C604740F67B4CC1F6F8
:10521000013C604741F2413CC1F6013C604740F629
:10522000076CC1F6003C604748F6B12CC1F6013C62
:10523000604748F6B92CC1F6013C604748F6C12CDE
:10524000C1F6013C60474DF6694CC1F6003C604731
:1052500048F6B93CC1F6013C604748F6A72CC1F6B8
:10526000013C604749F6150CC1F6013C604748F621
:10527000F90CC1F6013C604748F6C33CC1F6013C5D
:10528000604749F6313CC1F6013C604749F63D3C78
:10529000C1F6013C604748F63F4CC1F6013C60470F
:1052A00048F6495CC1F6013C604748F6750CC1F60A
:1052B000013C604748F6753CC1F6013C604748F642
:1052C000D16CC1F6013C604748F6C72CC1F6013CE1
:1052D000604748F6CF2CC1F6013C604748F6A15C18
:1052E000C1F6013C604749F6270CC1F6013C604716
:1052F00048F6E51CC1F6013C604748F6AB5CC1F6D8
:10530000013C604749F6493CC1F6013C604748F61C
:10531000276CC1F6013C604748F6815CC1F6013C50
:10532000604748F63D7CC1F6013C604749F2710C8C
:10533000C1F6013C604749F64B0CC1F6013C6047A1
:1053400049F2B92CC1F6013C604749F2931CC1F601
:10535000013C604749F6553CC1F6013C604749F2C3
:105360000F2CC1F6013C604749F2531CC1F6013CC9
:10537000604749F2051CC1F6013C604749F6CB3C49
:10538000C1F6013C604749F2891CC1F6013C604707
:1053900049F2056CC1F6013C604740F6954CC1F6F8
:1053A000013C604749F6613CC1F6013C604749F663
:1053B0006D3CC1F6013C604748F6E32CC1F6013C68
:1053C000604749F6390CC1F6013C604749F2496C27
:1053D000C1F6013C60474AF6653CC1F6013C6047B6
:1053E00041F25D6CC1F6013C604749F6893CC1F66B
:1053F000013C604740F62B4CC1F6013C604740F64B
:105400000B4CC1F6013C604749F6E97CC1F6013C12
:10541000604749F6E56CC1F6013C604749F67D5CA2
:10542000C1F6013C604749F6597CC1F6013C604732
:1054300048F6610CC1F6013C604748F6577CC1F65E
:10544000013C60474AF2D50CC1F6013C60474AF284
:10545000270CC1F6013C60474AF2A70CC1F6013C9B
:1054600060474AF2731CC1F6013C604749F6075C8D
:10547000C1F6013C604749F6F34CC1F6013C604778
:105480004AF27B1CC1F6013C60474AF21D2CC1F672
:10549000013C60474AF2350CC1F6013C604749F6D1
:1054A000A13CC1F6013C60474AF2470CC1F6013C01
:1054B000604749F69B3CC1F6013C60474AF2730CD9
:1054C000C1F6013C60474AF28F1CC1F6013C6047BF
:1054D00049F60F4CC1F6013C604749F6EF3CC1F676
:1054E000013C604749F6D94CC1F6013C60474AF29D
:1054F000312CC1F6013C604749F6C54CC1F6013C70
:10550000604749F6074CC1F6013C604749F6234C19
:10551000C1F6013C604748F6892CC1F6013C604762
:105520004AF2497CC1F6013C604749F61B4CC1F682
:10553000013C604749F6594CC1F6013C604749F6C9
:105540003B4CC1F6013C604749F63F5CC1F6013C6B
:10555000604749F62D5CC1F6013C60474AF2EF2CEA
:10556000C1F6013C60474AF2757CC1F6013C6047D8
:105570004AF2DD2CC1F6013C604749F6195CC1F6E0
:10558000013C604749F6514CC1F6013C604749F681
:10559000675CC1F6013C60474AF2C93CC1F6013C78
:1055A00060474AF66F5CC1F6013C60474AF6BF3C73
:1055B000C1F6013C60474AF6250CC1F6013C604744
:1055C00038B504466846AFF3008001462046FEF732
:1055D00037FA38BD1E48007D00F0040010B94FF0C6
:1055E000FF3070474FF04020006820F010004FF06F
:1055F000402108600846006840F00700086040F25B
:105600003730144908604FF6FF704FF0402148646E
:105610000F48406820F001000D4948600846406886
:1056200020F0080048600846406820F040004860CC
:105630000846406820F0800048604FF04020006835
:1056400040F010004FF0402108600020C9E7000042
:10565000B88608108C40004070B504460D46002204
:1056600029462046FEF7F1F970BD000001480068A8
:10567000704700004487041AF8B504460D461646E4
:105680001F4600203B463246294600902046FEF742
:10569000E1F9F8BD70B504460D46002229462046C2
:1056A00000F0E8F970BDF8B504460D4616461F46F1
:1056B00000203B463246294600902046FEF7CFF9AF
:1056C000F8BD10B504460021204600F06FFA10BD69
:1056D00010B5002000F036FC10BD00000148406805
:1056E000704700004487041A70B504460D46012235
:1056F0002946204600F092F870BDF8B504460D46E4
:1057000016461F4601203B46324629460090204659
:1057100000F0BAF8F8BD18B504460121204600F0A3
:1057200031FA009018BD10B504460121204600F062
:105730003DFA10BD70B504460D46164601233246AB
:105740002946204600F0ECFA70BD10B50920FEF79E
:105750008BF910BD0246114B53F8210000BF036ABC
:1057600003F40043002BFAD110234362531C03625D
:1057700000BF036A03F40043002BFAD1836B23F4C8
:105780008073836390234362531C036200BF036AE8
:1057900003F40043002BFAD1704700005087041A2D
:1057A00030B502461A4C54F822000024194DAC546E
:1057B000012404600AB1202400E0202423460021B3
:1057C00021E000BF046A04F40044002CFAD1A024B4
:1057D0004462002444634C1C046200BF046A04F465
:1057E0000044002CFAD1082444624C1C046200BF1F
:1057F000046A04F40044002CFAD1074D05EB42156D
:105800006C544C1CE1B29942DBDB0024446030BD97
:105810005087041AA4000010B3BB002070B50646E0
:105820000D461446022C02D34FF0FF3070BD1348D2
:10583000005D08B10020F9E7114840F824601148E4
:1058400040F8245054B9522201210320FEF711F9E7
:10585000122202210320FEF70CF909E05622092149
:105860000420FEF706F9162208210420FEF701F9AC
:105870000120024908550020D8E70000A2000010CE
:10588000A8000010B00000102DE9FE4F05460E469E
:1058900017469846DDF83090B9F1020F03D34FF068
:1058A000FF30BDE8FE8FB9F1000F01D0202000E0ED
:1058B0002020A84202D86FF00400F2E76A4810F8EE
:1058C000090010B94FF0FF30EBE7684800EB4910D2
:1058D000405D022801D1C01EE3E7654850F8294029
:1058E000206A00F4004010B16FF00100D9E73420C5
:1058F0006062681C206200BF206A00F4004000283B
:10590000FAD1D4F838A0206B0290D4F834B05748BC
:1059100000EB4910405D012815D1306800F00040CF
:1059200040B1308880B202903068C0F30C4040F43F
:10593000404B08E00020029041F6FF71306801EA18
:10594000800040F4004B494800EB4910405D0528B9
:1059500036D2DFE800F00307041D220000BF4FF03D
:10596000FF309EE7307900F0010010B94BF4005B86
:1059700002E03079C0F30318B8F1080F01D94FF0F5
:1059800008082AF00F0040F4807040EA080A1AE084
:105990002AF00F0040EA080A15E0307900F0010013
:1059A00010B13079C0F30318B8F1080F01D94FF0E6
:1059B00008082AF00F0040F4807040EA080A02E06C
:1059C0004FF0FF306DE700BFB020606202982063A7
:1059D000C4F834B0C4F838A0244800EB4910405D46
:1059E00004281ED03878797840EA0120E063B8783E
:1059F000F97840EA01202064606A40F002006062A9
:105A0000B8F1040F0DDD3879797940EA012060643E
:105A1000B879F97940EA0120A064606A40F0010099
:105A20006062681C206200BF206A00F40040002809
:105A3000FAD101904FF6FF70009000BF2946204632
:105A400026F04CFC30B90198411C01914FF6FF71D2
:105A50008842F3D34FF6FF710198884202D34FF08A
:105A6000FF301EE740461CE7A0000010B3BB00203B
:105A70005087041A10B503460C46022A02D34FF091
:105A8000FF3010BD0AB1202000E02020984202D84B
:105A90006FF00400F5E73848805C10B94FF0FF3034
:105AA000EFE7364850F82210086A00F4004010B1C1
:105AB0006FF00100E5E770204862581C086200BFE3
:105AC000086A00F400400028FAD1F0204862052C52
:105AD00040D2DFE804F0030713232F0000204863BF
:105AE00088633AE0C86A40F48040C862486B40F47A
:105AF000204048634FF4086088632EE0C86A40F491
:105B00008040C862486B20F400504863486B40F402
:105B10000040486341F2884088631EE0C86A20F470
:105B20008040C862486B40F4204048634FF4D45032
:105B3000886312E0C86A20F48040C862486B20F491
:105B400000504863486B40F4004048634FF4A45051
:105B5000886302E04FF0FF3093E700BF084800EB96
:105B60004210C454581C086200BF086A00F4004088
:105B70000028FAD100BF84E7A00000105087041A63
:105B8000B3BB002008B50246022905D209B1202086
:105B900000E02020904203D800200090009808BD2B
:105BA00001480068FBE700004C87041A70B5054601
:105BB0000C46022C02D34FF0FF3070BD15B1022D00
:105BC00072D153E0002050490855A4B93320FDF7A5
:105BD00055FF4E484E4908604E48D0F8280140F025
:105BE00001004D49086000BF4B48006800F001000B
:105BF0000028F9D016E02B20FDF740FF4348444928
:105C0000091F08604348D0F8200240F001004249D3
:105C1000F831086000BF4048F830006800F001002B
:105C20000028F8D02046FFF7BBFD74B93A48006859
:105C300020F001003749C1F8280100BF364800684C
:105C400000F001000028F9D10FE03348F830006877
:105C500020F001002F49C1F8200200BF2E48F83083
:105C6000006800F001000028F8D14AE02B48005DF0
:105C700010B94FF0FF30A0E72348005D08B10020C5
:105C80009BE794B92148224908602248D0F82801AE
:105C900040F001002049086000BF1F48006800F084
:105CA00001000028F9D014E028E018481849091F1D
:105CB00008601848D0F8200240F001001649F83179
:105CC000086000BF1448F830006800F001000028A8
:105CD000F8D02046FFF764FD01200B49085534B980
:105CE000332019F00DFE3320FDF7CDFE05E02B200B
:105CF00019F006FE2B20FDF7C6FE02E06FF0030050
:105D00005BE700BF002058E7A00000100008000972
:105D1000840005400010054028110540A200001035
:105D20002DE9FF4F85B0884692460898022804D393
:105D30004FF0FF3009B0BDE8F08F059810B16FF05B
:105D40000600F7E751490898085C10B94FF0FF309A
:105D5000F0E70AF0FF0BCAF307200290CAF30740EE
:105D60000190CAF30460039002985844022803D3B8
:105D700002985844102802D96FF00800DAE7019819
:105D800010B10198082802D96FF00A00D2E70398F1
:105D900010B10398042802D96FF00B00CAE73C4900
:105DA000089851F820600BF1010002990144019814
:105DB00001EB00090920FDF757FE0546012414E018
:105DC000102C02D14FF0FF30B4E7B5FBF4F03149AD
:105DD000884209D8B5FBF4F109FB08F0B1FBF0F2F9
:105DE00000FB121000B901E0641CE9E700BF09FBE9
:105DF00008F06043B5FBF0F7B7F5806F02D96FF09C
:105E0000070097E707FB09F000FB08F06043A84292
:105E10000CD807FB09F000FB08F000FB14500F2121
:105E2000B1EB802F0FD26FF0070083E707FB09F07B
:105E300000FB08F06043401B0F21B1EB802F02D222
:105E40006FF0070076E730680490049800F0410096
:105E5000412801D0412030600398411E781E61F333
:105E60009F1002995944491E40EA01210198401EA1
:105E700041EA0030F060781E8009B061601EC6F80B
:105E8000800104983060002054E70000A00000105A
:105E90005087041A80F0FA0270B506460C46022CB0
:105EA00002D34FF0FF3070BD2348005D10B94FF0B2
:105EB000FF30F8E7214850F82450062E35D2DFE8AD
:105EC00006F0030B1316202A012028601C4850F806
:105ED0002410042088472BE00E202860184850F832
:105EE00024100120884723E06FF00300DBE78620C1
:105EF000286008206861124850F824100320884761
:105F000016E08E202860182068610D4850F8241093
:105F1000032088470CE08E20286010206861084824
:105F200050F824100320884702E06FF00400BAE71D
:105F300000BF0020B7E70000A00000105087041A3F
:105F4000A800001010B50446022C02D34FF0FF3019
:105F500010BD54B9002201210320FDF78AFD002263
:105F600002210320FDF785FD09E00022092104201C
:105F7000FDF77FFD002208210420FDF77AFD0020B7
:105F80000149085500BFE3E7A200001070B5494879
:105F9000446849484078604000F0E00060B34648FB
:105FA00040786040204000F0800020B143484168C4
:105FB000042088471EE0404840786040204000F0C0
:105FC000200020B13D4841680320884712E03A484C
:105FD00040786040204000F0400020B137484168E0
:105FE0000220884706E004F0E00018B13348416819
:105FF0000120884730494C7058E02E480069C5B2EE
:1060000005B954E0002D51D0202D4FD81C2029492E
:10601000843108602748C0F8805000BF2548803090
:10602000006800F400400028F8D16D1E2448405D4F
:10603000052839D2DFE800F003040A1B210034E010
:10604000204801214268284690472EE01D48022141
:1060500042682846904717489830006800F480400E
:1060600020B1184804214268284690471DE0154891
:10607000012142682846904717E00E489830006892
:1060800000F4004078B10F4802214268284690474A
:1060900008489830006800F4804020B10948042185
:1060A00042682846904700E000BF00BFA5E700BF58
:1060B00070BD000000400A40A4000010A8000010BD
:1060C000D3BB0020B000001001461448007D00F052
:1060D000020010B94FF0FF30704701F00F000128A7
:1060E00002D0022814D109E04FF04020406820F08F
:1060F00001004FF0402250600020EDE74FF04020BB
:10610000406840F001004FF0402250600020E3E77B
:1061100000BF00BF6FF00300DEE70000B886081084
:10612000F0B50446C1680320B1FBF0F789B0002642
:106130005FE000BFA16806EB46000D18D4E900013E
:1061400001228368681C9847002855D0694620467C
:10615000FDF79EFCF0B3D4E9000101228368A81C7E
:106160009847002848D020690099884202D3401CF3
:1061700008D139B9E81CC4E90410781E864201D15F
:10618000A0686061204604A9FDF782FC18B104995B
:10619000009888422CD0D4E9000101228368284667
:1061A0009847002828D0226861680298D3680122A5
:1061B0009847002820D0039830B1D4E90021D36853
:1061C00001229847002817D04FF400716068FDF74E
:1061D00064FC00E00CE0D4E900010122C368681C03
:1061E0009847002808D0607E40F00400607602E006
:1061F000761CBE429ED3012009B0F0BD02466FF06E
:106200000300704770B50024B2E05B4801680120CC
:10621000A0400140002975D0584800EB441556486D
:1062200040680121A140084000287DD00120A04005
:106230005149886004EB8400514901EB8000C0683B
:1062400004EB84014E4A02EB8101896888425AD0EE
:1062500004EB8400114601EB8000806804EB8401AC
:1062600002EB8101C968461AB6F5805F01D340F69A
:10627000FF7604EB8400424901EB8000C0683044A3
:1062800004EB84013E4A02EB8101C860E86800F03B
:10629000806098B104EB8400114651F8200028601A
:1062A00004EB840051F82010E868C0F3814006FA3E
:1062B00000F0084404EB840142F82100E86800F093
:1062C0000060B8B104EB84002D4901EB8000406808
:1062D000686004EB840001EB80004168E868C0F36B
:1062E000415006FA00F0084404EB8401244A02EB12
:1062F00081014860E86866F30B00E860286940F0B7
:106300000100286133E0E0B2FDF7CCFB04EB840030
:106310001B4901EB8000006948B304EB84000A4686
:1063200002EB8000016900E002E0012088471EE0E6
:106330001148C0680121A1400840C0B10020286177
:10634000E860E0B2FDF7AEFB0120A0400A49086119
:1063500004EB84000A4901EB8000006938B104EBCA
:1063600084000A4602EB8000016902208847641C11
:10637000082CFFF44AAF70BD00200040002100400F
:106380005031001070B50024124845691248284069
:106390001049486105F0010008B144F0020405F01D
:1063A000400008B144F001040C48856B05F008007A
:1063B00030B10A48C06A00F0200008B144F004047B
:1063C00034B10748006818B105480168204688477D
:1063D00070BD0000001001404100010000000140BC
:1063E000B40C00102DE9F05F0446884691461E4625
:1063F000DDE90BAB0A9F082C03DB4FF0FF30BDE853
:10640000F09F204600F0C0FE401C10B94FF0FF3056
:10641000F5E704EB84002D4901EB8000C0F810B0D3
:106420002B4800EB441500202861E8600120A040C3
:10643000284988600120A04008610020A860012050
:10644000086300BF2348006B00F001000028F9D06A
:1064500004EB84001D4901EB80008660B6F5805F87
:1064600001D340F6FF76384666F30B000746C5F8C1
:106470000080C5F8049007F0806020B1C7F3814028
:1064800006FA00F0804407F0006020B1C7F34150E5
:1064900006FA00F0814404EB84000C4941F82080A6
:1064A00004EB840001EB8000C0F8049004EB84004E
:1064B00001EB8000C660EF60C5F810A00AF0010093
:1064C00010B92046FDF7EEFA002098E75031001091
:1064D000002100400020004010B50446082C02DBDB
:1064E0004FF0FF3010BD2046FDF7DCFA054800EB09
:1064F0004410006920F00101024800EB44100161E2
:106500000020EFE70021004010B51348006810B9E3
:106510004FF0FF3010BD10480068401E0E49086063
:106520000846006808B10020F4E70C48006820F035
:1065300001000A4908600220002807DB00F01F0262
:1065400001219140064A430942F8231000BF02206E
:10655000FDF7ADFA0020DDE75001081040140540BA
:1065600080E100E00246054850F8220001238B40FC
:10657000184008B1012070470020FCE700610F407F
:1065800010B52AB101238B40054C44F8203005E0BA
:1065900001238B40024C803444F8203010BD0000B1
:1065A00000620F4070B10F49096841F003010D4AC4
:1065B000116000BF0B49091D096801F001010029A4
:1065C000F8D00DE00749096821F00301054A116080
:1065D00000BF0449091D096801F001010029F8D133
:1065E000704700001014054010B54AB1094B53F82C
:1065F000203001248C402343064C44F8203008E02E
:10660000044B53F8203001248C40A343014C44F840
:10661000203010BD00600F4002464FF0FF33112ABA
:1066200044D2DFE802F00E090A0B0C431923262995
:10663000434334373A3D400000BF00BF00BF10461F
:1066400070471F48406800F00A00022802D04FF04F
:10665000FF30F5E70020F3E71A48806900F00100F9
:1066600010B14FF0FF30EBE70620E9E71548016A6B
:106670001EE01448016B1BE01248006C00F00100A2
:1066800010B11048406C00E00020014610E00D48B9
:10669000816C0DE00B48C16C0AE00A48016D07E00F
:1066A0000848416D04E00748816D01E01846C7E7DE
:1066B00000BF01F0010008B9C1F304631846BFE749
:1066C000003004400000054038B500200090084824
:1066D000807A00F0020028B105486A46012103686B
:1066E00008469847BDF80000C0F38004204638BD36
:1066F000443100100148406870470000B886081017
:1067000001466FF00300704704461AA0FDF7D4F964
:106710001E4802681EA12348FAF7FEF82148FDF73B
:10672000CBF91A48006800F08040B8B11EA0FDF710
:10673000C3F91648001F026820A11A48FAF7ECF8BE
:106740001848FDF7B9F91148001F006820490840B2
:1067500020B10E49091F0868FDF7B3F91DA11148C2
:106760006269FAF7D9F81FA12248A269FAF7D4F8AA
:1067700000BFFEE7496E2048617264204661756C77
:10678000742048616E646C65720A00002CED00E0B4
:106790005343422D3E48465352203D203078253009
:1067A00038780A00B8B80020466F726365642048E4
:1067B000617264204661756C740A00005343422D77
:1067C0003E43465352203D203078253038780A0029
:1067D00000000F036C72203D203078253038780A95
:1067E000000000007063203D203078253038780AA2
:1067F0000000000008B9002070B504460D46034AA9
:1068000029462046FDF762F970BD00006CE4041AC9
:1068100010B50248FDF75FF910BD00006CE4041AE2
:1068200010B50248FDF75CF910BD00006CE4041AD5
:10683000F8B504460D4616461F4604483B46324608
:1068400029460090204600F05BF8F8BD6CE4041A7D
:1068500010B5044602492046FDF747F910BD000077
:106860006CE4041A70B504460D46034A29462046D6
:10687000FDF740F970BD00006CE4041A014800689F
:106880007047000068E4041A08B5024800680090E8
:1068900008BD000064E4041A014688694068704736
:1068A00070B505460C46A069007A00F0010008B1F9
:1068B000002070BD10492068884204D140F60800CD
:1068C000FDF71DF90DE00D492068884209D14122EC
:1068D00004210220FDF7CDF8412203210220FDF71B
:1068E000C8F82421A069FDF733F8A06905600120EC
:1068F000A16908720020DCE700100A4000000E4089
:106900002DE9F04105460E4617469846069C16B1FD
:106910000FB17F2D03D96FF00400BDE8F081A069AD
:10692000007A00F0040010B94FF0FF30F5E7A069DD
:10693000007900F0010020B9A069C07A00F00600DB
:1069400010B16FF00100E8E794F9040018F0F4FFCB
:10695000012000EB4500A1694872A06980F80A8017
:10696000A0694661A06987614FF0FF30A1690861A5
:10697000A069406820F00100401CA1694860A0693E
:10698000406820F00200801CA1694860A06940684E
:1069900020F00400A1694860A069406820F0100060
:1069A000A1694860A069406820F02000A1694860A2
:1069B000A069C07A28B9A069007B40F02000216856
:1069C000086094F90400FDF79FF80020A5E770B572
:1069D00005460E46144605B116B96FF0040070BDA9
:1069E000A069007900F0010020B9A069C07A00F028
:1069F000030010B16FF00100F1E794F9040018F002
:106A00009BFFA069007A40F00800A1690872A069A4
:106A1000C561A06906624FF0FF30A1690861A069F5
:106A2000406820F00800A1694860A069406820F033
:106A30002000A169486094F90400FDF765F8002082
:106A4000CDE7000010B504460020A16908720C498A
:106A50002068884203D10020FDF751F80DE0094974
:106A60002068884209D1002204210220FDF701F8A4
:106A7000002203210220FCF7FCFF002010BD0000D3
:106A800000100A4000000E402DE9F04106460F4676
:106A900014461CB96FF00400BDE8F0811D48007970
:106AA00000F0020010B94FF0FF30F5E71948C07947
:106AB00040F0010040EAC62040EA8710164908610C
:106AC000FDF727F8054600BF1348006900F00100F4
:106AD00020B91148406920800020DDE7FDF719F852
:106AE000421B0E480088C82148430D490988C82325
:106AF000594300EB21408242E6D30748006900F089
:106B0000010020B90448406920800020C4E76FF0EC
:106B10000200C1E7B40C0010000001400CE4041AAC
:106B20000EE4041A70B5054625B1012D2AD0022DB8
:106B300077D12AE00520002807DB00F01F020121A1
:106B400091406A4A430942F8231000BF6848006830
:106B5000C04340F480006749C1F8000100BF6448A9
:106B6000006800F480000028F9D06348006820F035
:106B70000100614908606148007920F002005F4926
:106B80000871AFE06FF0030070BD5C48007900F061
:106B9000010010B94FF0FF30F6E75848007900F0D7
:106BA000020008B10020EFE75348006840F00300FE
:106BB0005149086000BF5048001D006800F0010006
:106BC0000028F8D04E48006820F00700001D4D490D
:106BD000C1F82C0146480068C04340F48000454994
:106BE000C1F8000100BF4248006800F4800000289E
:106BF000F9D04548006840F001004349086000BFF3
:106C00004148006800F001000028F9D10920FCF794
:106C10002BFF04463D48844204D310203749C871F5
:106C20001FE05CE03A48844203D304203349C87132
:106C300017E03848844203D300203049C87110E07F
:106C40003548844203D30C202C49C87109E03348ED
:106C5000844203D308202949C87102E06FF0030081
:106C600092E72648C0792E4908614FF42040086019
:106C700020204860802088610020086448644FF428
:106C80000270C863FCF74AFFFCF74DFF4FF0FF307E
:106C90001D4948612348C8610520002807DB00F032
:106CA0001F0201219140204A430942F8231000BFEE
:106CB0000520002809DB00F01F0201219140420954
:106CC000920002F1E022C2F8001100BF00200B493F
:106CD00088600846007940F00200087102E06FF019
:106CE000030051E700BF00204EE7000080E100E014
:106CF000503105400030054020140540B40C001010
:106D00002C310440003004400010014080D1F008D4
:106D100000E1F50500879303C00E160240787D015F
:106D2000000001404100010080E200E010B5014692
:106D300011B102297ED148E00620002807DB00F0CF
:106D40001F0301229A40624B440943F8242000BFEC
:106D50006048007D20F002005E4A107510464068D1
:106D600020F0010050601046406820F002005060A2
:106D70001046406820F0040050601046406820F043
:106D8000080050601046406820F010005060104627
:106D9000406820F0200050601046406820F040001D
:106DA00050601046406820F0800050604A480068FB
:106DB000C04340F48010494AC2F8000100BF0020DF
:106DC000474A1060474A10607EE04248007D00F06C
:106DD000010010B94FF0FF3010BD3E48007D00F0BB
:106DE000020008B10020F7E700203A4A9060002234
:106DF000384802613B48006840F00300394A10609F
:106E000000BF3848006800F001000028F9D034487D
:106E1000006840F00300324A106000BF304800684C
:106E200000F001000028F9D007204FF04022106048
:106E300000BF00E045E04FF04020006800F0070090
:106E40000028F6D10120284A106000BF26480068BB
:106E500000F001000028F9D11420234A10321060FC
:106E60004AF2CF304FF04022506220481060204854
:106E7000D0648020C2F880001E481B4A083210608F
:106E80000620002807DB00F01F0301229A401A4B5E
:106E9000440943F8242000BF0620002809DB00F045
:106EA0001F0301229A4043099B0003F1E023C3F82A
:106EB000002100BF0748007D40F00200054A107520
:106EC00002E06FF0030087E700BF002084E70000C6
:106ED00080E100E0B88608105031054000300540E0
:106EE0000028054038140540804000401000000292
:106EF0000F000E007886081080E200E070B50646AC
:106F00000C461EB914B16FF0040070BD1D48007925
:106F100000F0020010B94FF0FF30F6E71A48406861
:106F200040F2044188431849486000208860C860E6
:106F300004B9EAE71AE006213046FCF7F9FD850EB0
:106F400005F0200048B11048806805F01F020121BB
:106F5000914008430C49886006E00B48C068012155
:106F6000A94008430849C860B61D641E002CE2D140
:106F70000548406840F20441084303494860002046
:106F8000C3E70000B40C00100000014030B51F241E
:106F9000604D2C60604C614DEC660024AC6140F2A9
:106FA000DC5100E0491E0029FCD15C4C646C44F0CB
:106FB00001045A4D6C645A4C6C6400BF574C246CED
:106FC00004F00104002CF9D0564C544DEC6640F20C
:106FD0001A4100E0491E0029FCD1534C4F4D6C640E
:106FE00000BF4E4C246C04F00104002CF9D04D4C31
:106FF0004A4DEC662C46246A44F001042C624FF49E
:107000008040142424B1012C05D0022C07D104E0C7
:107010004FF0FF3012E0454810E045480EE01421E3
:1070200008E080EA500404F00104C0F34D0545EA8D
:107030008430491CB1F5004FF3D900BF00BF0B22CB
:107040001823540444EA83540443344D6C62802072
:10705000012424B1012C05D0022C09D105E04FF008
:10706000FF3018E040F2023015E040F2022012E05A
:1070700001210CE080EA900484EAD00484EA101430
:1070800004F00104C0F3460545EAC410491CB1F5FB
:10709000807FEFD900BF00BF0403204DAC621020F9
:1070A000012424B1012C05D0022C07D104E04FF0BB
:1070B000FF3012E0622010E042200EE0012108E0E3
:1070C00080EA900404F00104C0F3430545EA04108B
:1070D000491CB1F5007FF3D900BF00BF0F4CA46A73
:1070E00004430E4DAC62134C2C6200BF0B4CE469A0
:1070F00004F00104002CF9D00A4C0834074DAC64AC
:107100000D4CEC64044C2C656C65064C8434AC6509
:1071100030BD00000C520040000800010000054096
:107120000000130600080009000813060380010090
:10713000030001001C08000604080003014611B901
:107140006FF0040070470E48007900F0020010B99B
:107150004FF0FF30F6E708794A7940EA0220094A01
:107160001064C87800068A7840EA02404A7840EA0B
:1071700002200A781043034A50640020E2E700002E
:10718000B40C00100000014010B5014600BF0B48D0
:1071900050E8002F01208840104020B1BFF32F8F0E
:1071A0004FF0FF3010BD012088401043034C44E8ED
:1071B0000003002BEBD10020F4E700004C01081085
:1071C00070B50B4600213EE04468B4F5F05F02D98B
:1071D0004FF4F05400E0446822464FF000442A4D3A
:1071E00005EB01152C60284C04EB01146260264D60
:1071F00005EB01150468AC6004681444224D05EBEE
:107200000115EC600468144404604468A41A4460E6
:107210004468B4F5F05F02D94FF4F05400E04468DC
:1072200022467AB1184C04EB0114646844EA4234F3
:10723000154D05EB01156C60046814440460446846
:10724000A41A4460491C042902D24468002CBBD112
:1072500044685CB94C1E0C4D05EB0414246844F0E2
:1072600004054C1E084E06EB041425602BB1064C99
:10727000246844F00804044D2C60034C246B44F053
:107280002004014D2C6370BD788608102DE9F04173
:1072900005460F4614461E460DB107B11CB96FF0E6
:1072A0000400BDE8F0812248007D00F0040010B920
:1072B0004FF0FF30F5E71E480079C0F3C00010B171
:1072C0006FF00100EDE706F0010030B11848007DD5
:1072D00040F008001649087505E01548007D20F0CB
:1072E00008001349087506F0020030B11048007D0F
:1072F00040F010000E49087505E00D48007D20F0B3
:1073000010000B4908750A48C56007FB04F00849DE
:1073100008614FF04020C461084600694FF04021E9
:107320000862012102480C30FFF74AFF0020B8E74D
:10733000B886081010B50548C06EC0F30464204636
:10734000FCF792FB0249086010BD000000000540F8
:107350001402001010B50F48006840F470000D4989
:1073600008604FF080700C4908604FF0E020006921
:1073700020F003004FF0E021086108486FF313008C
:10738000044980390860FFF701FEFFF7D3FF00F0E2
:1073900007F810BD88ED00E0043105400000001A38
:1073A0002DE9F04385B00720F949086000BFF8488F
:1073B000001D006800F001000028F8D0F5480068C2
:1073C000F549884203D20020F449086003E047F2FF
:1073D0007770F2490860F220F1490860F04980397D
:1073E000C1F88400EE4908310860F320091D0860E7
:1073F000091D0860091D0860091D0860091D086055
:10740000091D0860091D0860091D0860091D086044
:10741000091D0860091D0860091D0860F220E04987
:1074200080310860091D0860091D0860DC49983139
:107430000860F320091D0860091D0860091D086027
:10744000091D0860091D0860091D0860091D086004
:10745000F220D4490860091D0860091D0860091D53
:107460000860091D0860091D0860091D0860091DE4
:107470000860F120CB4984310860091D0860F320C1
:10748000091D0860091D0860091D0860F120091D1B
:107490000860091D0860091D0860F320091D0860C7
:1074A000091D0860091D0860091D0860BE490860C3
:1074B000F220BE490860091D0860091D0860091D09
:1074C0000860091D0860091D0860091D0860091D84
:1074D0000860091D0860091D0860091D0860091D74
:1074E0000860091D0860091D0860091D0860091D64
:1074F0000860091D0860F320AC4980310860091D4F
:107500000860091D0860091D0860091D0860091D43
:107510000860091D0860091D0860091D0860091D33
:107520000860091D0860091D0860091D0860091D23
:107530000860091D0860091D086001209C49086059
:10754000002088608146934800689A4988422CD977
:107550004FF0010900240DE0A00000F18050006808
:107560004DF82400944850F82410A00000F18050F9
:107570000160641C052CEFD300BF00BF00BFBFF348
:107580006F8F00BF00BF00BF2722814948318B4861
:107590008B4B9847002406E05DF82410A00000F112
:1075A00080500160641C052CF6D3F02085490860EA
:1075B000091D0860091D0860091D086081208249B5
:1075C000086000207A49C1F804027F490831086048
:1075D0000620091D08600020091D08600220091D01
:1075E00008600020091D08604FF489407749086051
:1075F00040F20330091D086001206D4988621421A2
:107600006448026809F10100B2FBF0F0A1FB0050F0
:1076100001466F4A00232846F9F7EAF864490863EF
:107620002D215C48026809F10100B2FBF0F0A1FBDA
:107630000051674A00232846F9F7DAF85C494863A5
:1076400046215448026809F10100B2FBF0F0A1FBA9
:10765000005001465E4A00232846F9F7C9F854490C
:1076600088630520C86308640E214A48026809F14E
:107670000100B2FBF0F0A1FB00500146544A002388
:107680002846F9F7B5F84A49486444214148026858
:1076900009F10100B2FBF0F0A1FB005001464C4A99
:1076A00000232846F9F7A4F8414988644421394861
:1076B000026809F10100B2FBF0F0A1FB0051444A5D
:1076C00000232846F9F794F83949C864462131481F
:1076D000026809F10100B2FBF0F0A1FB00513C4A45
:1076E00000232846F9F784F8314908650E21294816
:1076F000026809F10100B2FBF0F0A1FB0051344A2D
:1077000000232846F9F774F829494865022088655E
:10771000642002F0D5FF40F2831025490862C8209A
:1077200002F0CEFF40F2031021490862022408460D
:107730004462C82002F0C4FF43F6095115480268AC
:1077400009F10100B2FBF0F0A1FB00700146204AF4
:1077500000233846F9F74CF8054610220023F9F7C4
:1077600047F8441C124844624FF0830010490862F5
:10777000184800684FF0000008620846D0F8000181
:1077800040F400201149086005B0BDE8F083000016
:10779000301405401402001000B4C404006D084009
:1077A000806008408062084010650840806608409C
:1077B00000500040000E27075CEA041B2C310440F7
:1077C00001000010006C08400052004000510040D1
:1077D00000CA9A3B0040062870B504460D46034A8D
:1077E0002946204600F03AF870BD000018E6041A59
:1077F00008B50248FCF7A1F9009008BD18E6041A84
:1078000010B5024800F039FC10BD000018E6041A5B
:1078100010B50248FCF796F910BD000018E6041AEE
:1078200010B5044602492046FCF791F910BD00004E
:1078300018E6041A70B504460D46034A2946204648
:1078400000F0DEFC70BD000018E6041A10B5024816
:10785000FCF782F910BD000018E6041A2DE9FE4F6E
:1078600081460E461446206E90F82D0000F002006E
:1078700018B94FF0FF30BDE8FE8F00200290019054
:1078800000270090804609F0FF001538062870D2C6
:10789000DFE800F0034299B8DDFE06B3206E90F8F1
:1078A0002C0006280CD0E06850B1E3681B7903F087
:1078B000070343F08002E36859781878FCF7D9F899
:1078C000206E90F82D0040F00800216E81F82D0008
:1078D0006068C06D40F001006168C8651AE0206E04
:1078E00090F82D0020F00800216E81F82D006068CE
:1078F000C06D20F001006168C865206E90F82C0012
:10790000062807D0E06828B1E26851781078802214
:10791000FCF7AFF80020AEE766B3206E90F82C00BD
:10792000062811D0206E90F82C0004280CD0206975
:1079300050B123691B7903F0070343F0C0022369A8
:1079400059781878FCF795F8206E90F82D0040F0E3
:107950001000216E81F82D006068C06C20F00200DC
:107960006168C8646068406840F00400616848600D
:1079700027E0C1E0FFE7206E90F82D0020F0100016
:10798000216E81F82D006068C06C40F002006168D3
:10799000C8646068406820F0040061684860206E38
:1079A00090F82C0006280CD0206E90F82C000428AB
:1079B00007D0206928B12269517810788022FCF71D
:1079C00058F8002057E78EB1206E90F8260010B1CD
:1079D0006FF001004FE76068C06840F040006168E8
:1079E000C8600121206E80F8261009E06068C06838
:1079F00020F040006168C8600021206E80F82610E9
:107A0000002038E76068406820F002006168486044
:107A100094F8540000F0C000451CE06D08B9A06D5A
:107A200008B145F0080545F0040560688560A06D63
:107A300038B1206E90F8260018B1A16D0878FEF7D5
:107A40004BFD0021206E80F82610002013E76068AF
:107A5000406820F001006168486094F8540000F02C
:107A6000C000451CE06D08B9A06D08B145F00805DF
:107A700045F0020560688560E06D30B1206E0079E8
:107A800018B1E16D0878FEF727FD0020216E00E0B7
:107A900001E00871EFE66068406820F0030061686B
:107AA0004860A06D38B1206E90F8260018B1A16D25
:107AB0000878FEF711FDE06D30B1206E007918B145
:107AC000E16D0878FEF708FD94F8540000F0C0005E
:107AD000451CE06D08B9A06D08B145F0080545F0FA
:107AE0000605606885600020216E08710021206E07
:107AF00080F826100020BEE600BF00BF09F0FF009E
:107B000015286FD2DFE800F0FC0B0E1B282D39FC86
:107B1000FCFCFCFCFCFCFCFC464BA1BCE4004FF074
:107B2000010AF0E02078C0F3400010B10320029079
:107B300002E06FF006009EE64FF0020AE3E02078D4
:107B4000C0F3800010B10120029002E06FF0060047
:107B500091E64FF0030AD6E0012001904FF0040AAD
:107B6000D1E02078C0F3001008B1012702E06FF0E7
:107B7000060080E64FF0050AC5E02078C0F340100B
:107B800010B10120009002E06FF0060073E64FF0A4
:107B9000060AB8E0206E80F8246000206BE62078AA
:107BA000C0F3001088B336B96068406A20F0020064
:107BB0006168486247E0216C0968C1F30460FBF723
:107BC00053FFFE49B1FBF0F56068406A20F03807CA
:107BD0006800B04200D32EE0A800B04203D347F0C3
:107BE000080728E08CE0E800B04202D347F0100715
:107BF00021E02801B04202D347F018071BE06801DA
:107C0000B04203D347F0200715E019E0A801B042C5
:107C100002D347F028070EE0E801B04202D347F054
:107C2000300708E02802B04202D347F0380702E0EC
:107C30004FF0FF301FE647F002006168486202E043
:107C40004FF0FF3017E6002015E62078C0F3401013
:107C500088B1FF2E02D94FF0FF300CE66068806CCF
:107C600020F47F40616888646068806C40EA062088
:107C70006168886402E04FF0FF30FCE50020FAE51F
:107C80002078C0F3401010B94FF0FF30F3E50EB983
:107C90000020F0E52078C0F38010A0B1206E90EDB8
:107CA0000C0AB8EE400AD4ED190A60EE200A00EE84
:107CB000106AB8EE400AF4EE400AF1EE10FA05D070
:107CC0004FF0FF30D7E54FF0FF30D4E50020D2E58C
:107CD0002078C0F3401070B136B16068806C20F03D
:107CE00002006168886409E06068806C40F002000E
:107CF0006168886402E04FF0FF30BCE50020BAE51F
:107D00006FF00300B7E500BF206E007918B9206E50
:107D100090F8260010B16FF00100ACE509F4E060C6
:107D200088B1B0F5A06F06D0B0F5C06F05D0B0F542
:107D3000E06F0BD104E000BF0BE048F0010808E061
:107D400048F0020805E048F0030802E06FF0080080
:107D500091E500BF09F4405030B1B0F5805F04D028
:107D6000B0F5005F07D103E008E048F0180805E02F
:107D700048F0080802E06FF009007CE500BF09F454
:107D8000404018B1B0F5804F04D100E005E048F064
:107D9000040802E06FF00A006DE500BFA06890B330
:107DA000A068006920F0C00B09F4403048B1B0F57C
:107DB000803F07D0B0F5003F0FD0B0F5403F27D14E
:107DC00016E028E02078C0F3C01010B14BF0400B53
:107DD00002E06FF00B004EE51DE02088C0F30020AC
:107DE00010B14BF0800B02E06FF00B0043E512E0A6
:107DF0002078C0F3C01038B12088C0F3002018B13B
:107E00004BF0C00B03E007E06FF00B0033E502E03E
:107E10006FF00B002FE500BFBAF1020F02D0BAF1EC
:107E2000030F0DD109F4802010B16FF00C0022E592
:107E300009F40020B0F5002F02D06FF00D001AE514
:107E40002146304600F0AAFA401C10B96FF0070036
:107E500011E5216E81F82CA08025206E90F82C0071
:107E6000062805D1E068007900F0070005430DE021
:107E7000206E90F82D0000F0080028B1E06800792D
:107E800000F00700054300E000BF00BF00BFE0684E
:107E900028B1E268517810782A46FBF7EAFD802580
:107EA000206E90F82C00042802D0062803D100E0B0
:107EB00000BF00BF0FE0206E90F82D0000F0100012
:107EC00038B12069007900F0070040F04000054318
:107ED00000E000BF00BF00BF206928B122695178CF
:107EE00010782A46FBF7C5FD606910B38025206E27
:107EF00090F82C00022804D0032808D006280ED1C0
:107F000000BF6069007900F0070005430AE060697E
:107F1000007900F0070040F04000054302E045F022
:107F2000400500BF00BF6269517810782A46FBF710
:107F3000A0FD2078C0F3400018B92078C0F380007D
:107F400020B1029840F02400616888652078C0F371
:107F5000C00010B10198616808642078C0F3001077
:107F600030B16068406A20F00100384361684862BF
:107F70002078C0F3401038B16068806C20F00100B8
:107F80000099084361688864A06838B1A0680069F6
:107F900020F0C00040EA0B00A16808616068C0687A
:107FA00000F0C00040EA08006168C860206E90F8E8
:107FB0002D0040F00400216E02E0000000CA9A3B50
:107FC00081F82D00002056E408B501468868002895
:107FD00041D0086E90F82D0000F0040000283AD03F
:107FE000886882690888C0F3003028B113090098B6
:107FF00063F30000009003E0009820F0010000907F
:108000000888C0F3803028B15309009863F3410019
:10801000009003E0009820F0020000900868C0F390
:10802000004028B19309009863F3C300009003E077
:10803000009820F0080000900888C0F3C03028B1F4
:10804000D309009863F38200009014E0009820F0B8
:10805000040000900FE0009820F0010000900098CC
:1080600020F002000090009820F008000090009896
:1080700020F004000090009808BD70B50446E06D43
:1080800028B1E16D0878FBF76CFD054601E0206E34
:10809000C569284670BD70B505460C46206E90F83F
:1080A0002D0000F0010008B1002070BD206E0560B9
:1080B0000020216E08710021206E4171206E8171B7
:1080C000206EC171206E0172206E80F82610206E25
:1080D00080F824102088C0F3003050B1A3691B79C8
:1080E00003F0070343F0C002A36959781878FBF73F
:1080F000C0FC2088C0F3C02040B1E3691B7903F0C5
:108100000702E36959781878FBF7B3FC2088C0F3BD
:10811000C03050B1236A1B7903F0070343F0C0025B
:10812000236A59781878FBF7A4FC2088C0F38030C4
:1081300050B1636A1B7903F0070343F0C002636A1E
:1081400059781878FBF795FC2088C0F3403040B18F
:10815000A36A1B7903F00702A36A59781878FBF722
:1081600088FC2068C0F3004050B1E36A1B7903F03B
:10817000070343F0C002E36A59781878FBF779FCEB
:10818000A06D08B9E06D08B1FBF7F0FC0120216E8D
:1081900081F82D00002088E710B5014600204B68CB
:1081A0005B6903F01E0202F002037BB101240B6E37
:1081B0005C7140F020000B6E93F82C30032B05D13E
:1081C0000B6E93F826300BB140F0100002F0040360
:1081D00023B101240B6E1C7240F4007002F01003F6
:1081E0002BB101240B6E9C7140F0800007E002F07F
:1081F000080323B101240B6EDC7140F4807010BDC4
:108200002DE9FE4305460E46144605B11EB96FF032
:108210000400BDE8FE83206E90F82D0000F00400FD
:1082200010B94FF0FF30F4E7206E90F8260010B13F
:108230006FF00100EDE70121206E80F826104FF06D
:108240008069206E90F82C00022804D0206E90F8EF
:108250002C0003281AD1206E90F8270078B901214C
:10826000206E80F82710216E01F12500224631464C
:10827000FBF781FC07464FB14FF0FF30C9E7206E96
:1082800090F82700022801D14FF00009206E856187
:10829000206E06610021206E0162A06D08B3A26D00
:1082A00091785078FBF76CFCA06D4068A16D49781F
:1082B0004FF4F86202EA811141F44841491C49F047
:1082C0000342CDE900210290A16D0878334629468A
:1082D0006268FEF787F80746781C00285CD1401ECC
:1082E00097E76068406900F0200018B10021206E17
:1082F00080F8281011E0206E026A501C216E08627E
:10830000206E8069805C61680860206E90F82800AB
:10831000401CC1B2206E80F82810206E90F8280012
:10832000102804D2206E016A00698142E3D1206ED8
:10833000016A0069814229D10021206E80F826104F
:108340008846206E90F82C00022804D0206E90F809
:108350002C0003280DD1206E90F8270001280AD1A7
:10836000206E90F82D0000F0100020B94FF00108A9
:1083700001E04FF00108206E006830B1B8F1000F45
:108380000AD0206E01684046884705E06068406872
:1083900040F002006168486000203AE72DE9F34FA1
:1083A0008BB08946D9F840100968C1F30460FBF727
:1083B0005BFB059000210903059841EA1051000379
:1083C000CDE9000100230B9AF8F712FA04464FF0AA
:1083D000FF30039000200890D9F8600090F82C003E
:1083E000062845D199ED190ABCEEC00A10EE100A14
:1083F0001FFA80FA4FF0000836E0C74830F828002E
:10840000B4FBF0F0B0FBFAF6B6F5803F00D329E0FC
:108410000020069022E0032E01D2761C1BE0BE480D
:1084200030F828007043B0FBFAF7BC4202D9E01BD9
:10843000049001E0381B0490DDE90310884208D263
:1084400004980390B44800EB880090F802B0B0B2F2
:108450000790761C00BF0698401C069006980228DC
:10846000D9D300BF08F10108B8F1480FC5D315E111
:10847000B4F54C3F4FD3260CB4EB064F0DD100BFE3
:108480004FF48030B0EB161F07D9002003908346CD
:10849000B0B207904FF0100A00E14FF0000836E04C
:1084A0009D4830F82800B4FBF0F00609B6F5803F8F
:1084B00000D32AE00020069023E0032E01D2761C90
:1084C0001CE0954830F8280070430701BC4202D9EF
:1084D000E01B049001E0381B0490DDE903108842A2
:1084E0000AD2049803908C4800EB880090F802B000
:1084F000B0B207904FF0100A761C00BF0698401CDF
:10850000069006980228D8D300BF08F10108B8F1F8
:10851000480FC5D3C2E0D9F8080020B14FF0FF30B2
:108520000DB0BDE8F08F4CF6CC4084427ED9B4F556
:10853000403F01D90F2532E0B4F5343F01D90E2573
:108540002DE0B4F5283F01D90D2528E0B4F5183FFA
:1085500001D90C2523E0B4F50C3F01D90B251EE011
:10856000B4F5003F01D90A2519E0B4F5E83F01D977
:10857000092514E0B4F5D03F01D908250FE0B4F582
:10858000B83F01D907250AE0B4F5983F01D906257F
:1085900005E0B4F5803F01D9052500E00425B4FBD2
:1085A000F5F7C7F30B0038B9002003908346C7F3F3
:1085B0000F300790AA4623E003264FF000081CE086
:1085C000554830F82800704300FB05F7BC4202D93B
:1085D000E01B049001E0381B0490DDE903108842A1
:1085E00009D2049803904C4800EB880090F802B040
:1085F000B0B20790AA4608F10108B8F1480FDFD3DE
:108600000BF00F010A914FEA2B100990DDE90901E7
:1086100008440799484300FB0AF00103099891FBBD
:10862000F0F7C7F30B00C8BB102500E013E000BF54
:10863000B7FBF5F0C0F30B0040B9B7FBF5F74FF00F
:10864000000BC7F30F300790AA4603E0681E85B2FF
:10865000042DEDD222E04FF4007002904FF450450B
:1086600000BFAC4202D9601B049001E0281B0490BB
:10867000DDE90310884206D2049803904FF0000B06
:1086800001200790AA460298281A85B2B5F5804FB6
:10869000E7D2CAF3422008904FEA2A3A64210398AD
:1086A0004843B0FBF4F0032802D94FF0FF3037E71E
:1086B000D9F80400C06840F08000D9F80410C86000
:1086C0000798000AD9F8041048600798C0B2D9F892
:1086D00004100860D9F80400C06820F08000D9F8C0
:1086E0000410C8600BF0F0000BF00F010843D9F83C
:1086F00004108862D9F8080040B9AAF1010001010C
:10870000089841EA4000D9F80410C8620B98D9F8DB
:1087100060100863002003E7F8E4041A0246086EBC
:1087200090F82D0000F0040010B94FF0FF307047B2
:10873000886810B96FF00300F9E76AB90888C0F3D8
:10874000C02030B18868006920F002008B68186191
:1087500002E06FF00300EAE7012A0DD10888C0F3B8
:10876000C02030B18868006940F002008B68186151
:1087700002E06FF00300DAE7022A0DD10888C0F3A7
:10878000403030B18868006920F001008B681861C2
:1087900002E06FF00300CAE7032A0DD10888C0F396
:1087A000403030B18868006940F001008B68186182
:1087B00002E06FF00300BAE70020B8E72DE9F041CE
:1087C00080460E4617461C46B8F1000F01D006B190
:1087D0001FB96FF00400BDE8F081206E90F82D0005
:1087E00000F0040010B94FF0FF30F4E7206E90F86D
:1087F0002C00022804D0206E90F82C00032815D1FC
:108800000321206E80F82710224639463046FBF7B8
:10881000B2F905460DB12846DDE722463946404605
:10882000FFF7EEFC054625B12846D4E74FF0FF30B0
:10883000D1E70020CFE7000010B50022042101207D
:10884000FBF717F9002203210120FBF712F9074873
:108850000078012808D100220721FBF70AF900223D
:1088600005210120FBF705F910BD000030010810BB
:108870000020FBF78AF910B504462146002001F0DC
:1088800077FE10BD00200149087070477400002079
:1088900001460120704770470146012070470020C3
:1088A000FBF778B901460020704702460020704768
:1088B000014600207047014600207047704770470E
:1088C0000146002070470146002070470146002005
:1088D000704701460020704770477047002070477E
:1088E0002DE9FC410646002400F0E0F808BB1248E0
:1088F000124950F82600C568007C2A3551F820003E
:1089000087680F4850F8261099B1684688470400D8
:108910000FD000982860BDF80400A8809DF80600DC
:10892000A87100983860BDF80400B8809DF8060072
:10893000B8712046BDE8FC8184EA041A90E9041A63
:10894000DCEA041A00207047002070477CB5064618
:10895000002400F0ABF808BB1148124950F826007B
:10896000C568007C2A3551F820000F49806851F80D
:10897000261099B1026800928288ADF804208079AF
:108980008DF8060068468847040007D000982860E4
:10899000BDF80400A8809DF80600A87120467CBDA3
:1089A00084EA041A90E9041AD8EA041A08B50122E4
:1089B000694600F015F8012802D04FF0FF3008BDDD
:1089C0009DF8000008BD13B5012201A9FBF7E7F8E7
:1089D000012802D04FF0FF301CBD01981CBD0000E3
:1089E0002DE9F05F14468A46834600F05FF810B127
:1089F0004042BDE8F09F2A4951F82B602949307C5C
:108A0000F56851F82000296AC06890F8350006EB37
:108A10004000B0F82090A869401A29D0844200D9BB
:108A20000446E9697068738B0A1AA3EB0900801A7F
:108A30008046274644450CD302465046FBF7B4F81F
:108A40007068E861296AC24401EB0800A7EB0807D7
:108A5000286257B13A465046E969FBF7A5F8E8693C
:108A60003844E861286A38442862A87810B115E0D3
:108A70000024FAE7296AA869401A718B091AB1EB38
:108A8000490F0BD30220A870B07D074A4FF4007144
:108A900041EA003152F82B0001F09EFD2046A8E784
:108AA00084EA041A90E9041ABC0100200D490978EF
:108AB000884212D20C4951F8200070B1C16861B1EE
:108AC0000A49007C0978884209D2094951F82000F6
:108AD00028B1C06818B100207047272070472120B6
:108AE0007047000040EA041A84EA041A8CE9041A68
:108AF00090E9041A2DE9F0410E460746FFF7D6FF2C
:108B0000002818D10D484FF0000850F82740A07DEC
:108B1000E568B04208D185F80280607C20B9084839
:108B200050F8270000B18047607D40F08000B042DF
:108B300001D185F80080BDE8F081000084EA041AC4
:108B4000FCEA041A70B50446FFF7B0FF050029D10E
:108B5000154850F82400407C01280AD0134800BF73
:108B600050F8240000B18047114E56F8240010B18F
:108B70000AE01048F4E71048214650F82400FBF7BB
:108B800018F846F8240060B10C4E56F8240048B995
:108B90000B48214650F82400FBF70BF846F8240058
:108BA00000B91025284670BD84EA041AECEA041ABC
:108BB000B8010020CCEA041A38EA041ABC010020EB
:108BC0003CEA041A2DE9F04116460F4605460024FA
:108BD000FFF76CFF38B9054850F825201AB1314627
:108BE0003846904704462046BDE8F08110EB041A51
:108BF00070B50E4605460024FFF758FF30B904480B
:108C000050F8252012B1304690470446204670BDEA
:108C100030EB041A70B50E4605460024FFF746FFF8
:108C200030B9044850F8252012B130469047044628
:108C3000204670BD20EB041A70B50E460546002490
:108C4000FFF734FF30B9044850F8252012B1304600
:108C500090470446204670BD14EB041A70B50D46CB
:108C600006460024FFF722FF68B9084850F826108E
:108C700049B128468847040005D0054850F8260029
:108C8000C06880F83250204670BD00003CEB041AEA
:108C900084EA041A70B50E4605460024FFF706FF65
:108CA00060B9074850F8251041B1304688470400A4
:108CB00004D0044850F82500C0688686204670BD60
:108CC00034EB041A84EA041A70B50E4605460024F3
:108CD000FFF7ECFE30B9044850F8252012B13046B9
:108CE00090470446204670BD1CEB041A07490978DA
:108CF000884209D2064951F8200028B1C16819B14B
:108D0000006808B100207047212070478CE9041AE0
:108D100090E9041A2DE9F05FDFF86C910546002018
:108D200059F82510002929D0584951F82510CC6848
:108D300094F84010C1F34112012A1FD1DFF850A16D
:108D4000544F11F01F0107D0012919D002293ED03C
:108D5000032913D1002692E000260CE05AF82610D1
:108D60000978A94205D159F82610E06C88470028F7
:108D700004D1761CF6B239788E42EFD3BDE8F09F6D
:108D80000026BB461EE000BF5AF8268098F8001067
:108D9000A94215D15FF00007C7EBC70108EB4101FD
:108DA0000A794AB1B4F8442049798A4204D159F881
:108DB0002610E06C884718B97F1CFFB2042FEBD354
:108DC000761CF6B29BF800108E42DDD3D6E7002663
:108DD000BB4642E05AF8268098F80010A9423AD1E2
:108DE0005FF00007C7EBC70108EB41010A7972B3D6
:108DF0008A7922B1B4F84420CB799A4222D00A7AF7
:108E000022B1B4F844304A7A93421BD08A7A22B114
:108E1000B4F84430CA7A934214D00A7B22B1B4F831
:108E200044304A7B93420DD08A7B22B1B4F844206F
:108E3000CB7B9A4206D00A7C4AB1B4F84420497CE4
:108E40008A4204D159F82610E06C884718B97F1C73
:108E5000FFB2042FC6D3761CF6B29BF800108E42E8
:108E6000B8D38BE75AF826100978A94205D159F8EA
:108E70002610E06C8847002880D1761CF6B239783D
:108E80008E42EFD37AE70000B8EA041A90E9041A98
:108E900014EA041AD4E9041A2DE9F84FDFF87491A2
:108EA000054659F8250000282DD05B4850F82500CC
:108EB000C46894F84000C0F34111012923D1DFF8C0
:108EC0005CA1DFF85C8110F01F0009D001281CD0E4
:108ED000022843D0032816D100265746403494E098
:108EE0000026574640340AE057F826000078A8428A
:108EF00003D159F8261020468847761CF6B298F818
:108F000000008642F0D3BDE8F88FCB4604F1400064
:108F10000026C14600901CE05AF8268098F8000010
:108F2000A84214D15FF00007C7EBC70108EB41006E
:108F3000017941B1B4F844104079814203D15BF822
:108F40002610009888477F1CFFB2042FECD3761CB4
:108F5000F6B299F800008642DED3D4E70026C34675
:108F600043E000BF5AF8268098F80000A8423AD1A2
:108F70005FF00007C7EBC70108EB4100017971B34F
:108F8000817921B1B4F84410C279914222D0017A9A
:108F900021B1B4F84420417A8A421BD0817A21B1B0
:108FA000B4F84410C27A914214D0017B21B1B4F8D4
:108FB0004410427B91420DD0817B21B1B4F8441022
:108FC000C27B914206D0017C49B1B4F84410407C88
:108FD000814204D159F8261004F1400088477F1CD3
:108FE000FFB2042FC6D3761CF6B29BF8000086426F
:108FF000B8D388E757F826000078A84203D159F87B
:10900000261020468847761CF6B298F80000864263
:10901000F0D378E7B0EA041A90E9041A14EA041AC3
:10902000D4E9041A70B504462E4E0D46C80704D084
:1090300056F8241009B101208847A80707D556F82B
:10904000241009B100208847204601F07BFA680708
:1090500021D5204601F076FA234850F8240006680E
:10906000F078B38800F00302B178204600F080FA6F
:1090700048B9F078B38800F00302B07840F080017E
:10908000204600F075FA204601F02EFA174850F8F5
:10909000240000B1804728070BD51549012051F85D
:1090A0002410C96881F83500124850F8240000B136
:1090B0008047E80604D5104850F8240000B18047E6
:1090C000A80604D50D4850F8240000B18047280AAE
:1090D000400705D029122046BDE8704000F07EBB55
:1090E00070BD000050EB041AFC01002054EB041A80
:1090F00090E9041A58EB041A5CEB041A60EB041AAA
:1091000010B504460B480C4950F824000978C06893
:109110008C4201D3002010BD0028FCD00749C06C50
:1091200051F8241088470028F5D12046BDE81040AA
:10913000FAF744BD90E9041A8CE9041A78EB041A92
:1091400010B504460A480B4950F824000978C06855
:109150008C420BD2002809D00749403051F8241026
:1091600088472046BDE81040FFF796BE10BD0000BE
:1091700090E9041A8CE9041A74EB041A10B5044639
:109180000D480E4950F824000978C0688C4201D37C
:10919000002010BD0028FCD0094900F14C0251F814
:1091A0002430111F403098470028F2D12046BDE8F6
:1091B0001040FAF708BD000090E9041A8CE9041A7F
:1091C00070EB041A10B504460020FAF701FD10BD3B
:1091D00010B504460020FAF7FBFC10BD0146002044
:1091E0007047017801F01F0121B1012903D0022944
:1091F00003D101E002E001E000E000BF00BF7047E2
:1092000070B5054605F0020078B301210020FAF799
:10921000E4FC16490968C1F800024FF0FF3400BFB2
:10922000124A1168124A506A2246FAF7DBFC08B962
:10923000012000E0002006460D48806A38B136B1B2
:109240000B48806A0068401C0949896A086000BFB1
:10925000084823F016FD054908604FF400730846DE
:10926000012102680020FAF7C2FC70BD0000001066
:1092700098060020641C00207047704710B5044613
:10928000204600F001F810BD10B50446012C03D1B2
:109290000121002000F093FC10BD704770B50D4611
:1092A0000446FAF7A9FC002808D1054850F8242004
:1092B000002A03D02846BDE87040104770BD00006A
:1092C000A8EA041A10B50446FAF796FC002807D15C
:1092D000044850F82400002802D0BDE810400047A0
:1092E00010BD0000A0EA041A70B51149002551F81C
:1092F0002010CC68E36B5BB18021A26BFAF781FC94
:10930000002804D1D4E90E121144C4E90E1570BD31
:1093100094F8361049B100231A468021FAF771FCFF
:109320000028F4D184F8365070BD222070BD0000B2
:1093300090E9041A094910B551F82010CC680021B1
:10934000D4E90E23FAF75DFC002805D1D4E90E011B
:109350000844A0630020E06310BD000090E9041AF7
:10936000704770470178C1F3411131B1012905D02F
:10937000022904D0032904D102E002E001E000E068
:1093800000BF00BF704700002DE9F84304460E46B9
:1093900017462078C0F3411030B1012847D0022889
:1093A00046D0032846D144E020780121B1EBD01FFC
:1093B0003CD1207800F01F00B8BB6078062835D17A
:1093C00060880321B1EB202F30D1A07803282DD164
:1093D000A08840F20941884228D1032017494870EB
:1093E00000BF0020009069460E2011F08BFA144A4D
:1093F00016211448009BFAF709FC124880464046A3
:10940000F7F7DFFE45002A4641460C48801CFAF774
:10941000CBFBA81C0949087008463060A81C3860BE
:10942000012009490870BDE8F883FFE702E001E088
:1094300000E000BF00BF0020F5E7000058B90020A1
:1094400062FC041AF4BB00200000002070470000FA
:1094500000200149087070470000002010B5FFF798
:10946000F5FF10BD704770470848007800F0020013
:1094700010B94FF0FF3070470548006840F0010018
:109480000449C1F840010020F5E70000310108104F
:10949000406100400060004008B5002000900D4889
:1094A000007800F0020008B9009808BD0A48016879
:1094B0000A480068009001F0010020B101F080002E
:1094C00008B9012200E00022009862F3C300009076
:1094D0000098EAE731010810846100403C0108105F
:1094E0000B48007800F0020010B94FF0FF307047D1
:1094F0000848006820F400000749C1F884010846C4
:10950000D0F8840140F04000C1F884010020EEE76B
:1095100031010810846100400060004070B50546CC
:109520000324114E09E000BF56F825006421FAF724
:1095300072FB28B90A20FAF773FB641EE4B2F3D277
:109540006CB10A4850F8250000684069804704461D
:1095500056F8250001F03AF81CB1222070BD2320F6
:1095600070BD002070BD0000AC00002090E9041A1E
:109570002DE9F05F9346884606461022DFF8789082
:1095800001F00F0102EAD8000D1859F826009A469A
:10959000C16805F11400085C20B141463046FAF775
:1095A00044FB08BB1548022400EBC617642157F89A
:1095B0002500FAF730FB28B90A20FAF731FB641EC0
:1095C000E4B2F3D2ACB159F82600524659460068CD
:1095D000C36A40469847044657F8250000F0F6FF56
:1095E00014F1020F05D014B12220BDE8F09F002035
:1095F000FBE72320F9E7000090E9041A90E400203B
:109600002DE9F0479246884606461022DFF874900E
:1096100001F00F0102EAD8000D1859F82600C168C0
:1096200005F11400085C20B141463046FAF7FDFA16
:1096300008BB1548022400EBC61700BF57F82500E9
:109640006421FAF7E8FA28B90A20FAF7E9FA641E61
:10965000E4B2F3D2A4B159F8260051460068426B37
:1096600040469047044657F8250000F0AFFF14F13C
:10967000020F05D014B12220BDE8F0870020FBE7DF
:109680002320F9E790E9041A90E400202DE9F0473F
:10969000884606461022DFF8749001F00F0102EAB6
:1096A000D8000D1859F82600C16805F11400085CAF
:1096B00020B141463046FAF7B8FAF8B91448022406
:1096C00000EBC617642157F82500FAF7A4FA28B969
:1096D0000A20FAF7A5FA641EE4B2F3D29CB159F855
:1096E00026000068016B40468847044657F825006D
:1096F00000F06CFF14F1020F05D014B12220BDE878
:10970000F0870020FBE72320F9E7000090E9041A26
:1097100090E40020024951F82000006840680047AA
:1097200090E9041A2DE9F0411746884605460324BE
:10973000114E08E056F825006421FAF76CFA28B9B2
:109740000A20FAF76DFA641EE4B2F3D284B10B4832
:10975000394650F825000068826840469047044624
:1097600056F8250000F032FF24B12220BDE8F08138
:109770002320FBE70020F9E7AC00002090E9041A61
:109780002DE9F0410F4605460324124E09E000BFC3
:1097900056F825006421FAF73EFA28B90A20FAF7AC
:1097A0003FFA641EE4B2F3D27CB10B4850F82500B6
:1097B0000068816A38468847044656F8250000F05C
:1097C00005FF24B12220BDE8F0812320FBE7002023
:1097D000F9E70000AC00002090E9041A2DE9F047F9
:1097E000DFF8D49205460E4659F8257048074FF029
:1097F0000008FC6828D594F84000000618D5E06BF6
:1098000010B994F8360018B12846FFF76DFD1BE03B
:1098100094F83700012817D184F837802846FAF7E2
:1098200009FA08B101287DD1284600F0A9FE0BE015
:109830002846FAF704FAA078010605D500F07F0162
:10984000A1702846FAF700FAB00746D594F8400010
:1098500001063FD4E16B19B12846FFF76BFD3CE0F0
:1098600094F83710012905D0C0F3411151B30129F3
:1098700028D10BE084F837802846FFF741FC08B177
:1098800001281FD12846FAF7E4F913E010F01F0071
:1098900018D0012802D0022814D10FE0284600F089
:1098A00085F938B92846FAF7D9F918B9284600F0E9
:1098B00009F938B12846FFF743FC0EE0284600F0CE
:1098C000FDF8F6E7012280212846FFF799FEC4F84B
:1098D0003C8002E0284600F059FEF00776D028468A
:1098E0004E4659F82010C9684031FFF749FF00285B
:1098F0006CD12846FFF742FC012150B3012811D159
:10990000B4F84620C2B1A06CA063E06CE06384F8B8
:10991000371094F840301B067ED5904207D27A7DEE
:10992000521E00E08AE0104201D184F83610284629
:10993000BDE8F047FFF7D8BC94F840000006284681
:1099400003D4BDE8F047FAF784B9BDE8F04700F06A
:1099500017BEB868A063B4F84600E06394F840000E
:10996000C0F3411111B1012968D15FE094F84100C1
:109970000C2863D2DFE800F006118717871C2B87BD
:10998000303A3E552846FAF76EF923E02846FFF7AD
:10999000ABFC284600F0F4FD61E0002104E028461D
:1099A000FAF757F95BE00121284600F07DFB3BE028
:1099B00056F82500C06890F8401011F01F0F62D1D2
:1099C00090F8421041F080018170E8E771E028468C
:1099D00000F0D0FA90B3D9E756F82500C06890F8A7
:1099E000401011F01F0F4ED1C11C18E0284600F0A6
:1099F000D7FB19E056F82510C86890F8402002F00F
:109A00001F02012A3FD1C278C2B1B0F8442090F8B9
:109A100034309A4237D200E02CE049681144816327
:109A2000B4E72846FAF724F940B1B8E710F01F0070
:109A300029D0012803D0022825D120E023E02846A0
:109A400000F0BAF858B92846FAF717F938B9284695
:109A5000FAF718F918B92846FAF719F998B128460B
:109A6000FFF76EFB94F84000000622D4B4F84600DD
:109A700000281ED02846BDE8F047FFF75BBC28460B
:109A800000F097F8EAE794F84000000605D4B4F82F
:109A9000460010B10122002106E0012200212846E3
:109AA000FFF7AEFD012280212846FFF7A9FDC4F88B
:109AB0003C80BDE8F087000090E9041A01460020D0
:109AC000704700002DE9F041074635480024DFF8D3
:109AD000D48050F82750EE6833E0334850F8240023
:109AE000017CB9422BD1B6F84410827C914202D05D
:109AF000C07C814223D196F84100412833D007DC55
:109B000068B1022814D0202822D0402817D123E0A1
:109B1000822831D0862834D0882810D138E02046D9
:109B2000FAF7BAF809E03846FAF793F878B306E09E
:109B3000B6F842102046FEF707FF0028F3D1641C58
:109B4000E4B298F800008442C7D30020BDE8F08159
:109B50002046FEF7FBFEF0E7B6F842202046A96853
:109B6000FAF79FF8E9E7B6F84630B6F84210204613
:109B7000AA68FAF79BF8E0E72046A968FFF7A4F87F
:109B8000DBE7A86801682046FAF795F8D5E705E015
:109B9000A86801882046FFF77DF8CEE70120D5E7C9
:109BA00090E9041A40EA041A84EA041A01460020E3
:109BB000704701460020704701460020704770B58D
:109BC0000C460546FFF792F8002805D121462846A5
:109BD000BDE87040FAF729B870BD00002DE9F041EA
:109BE00007460E460024A8E06C4850F824000028E0
:109BF0007ED06A4850F824000078B84278D1002519
:109C000096E0664850F82400001DC5EBC50110F829
:109C1000110000286DD0614850F82400001DC5EBEC
:109C2000C50100EB4100807850B15C4850F8240039
:109C3000001DC5EBC50100EB4100C078B04271D0FA
:109C4000564850F82400001DC5EBC50100EB41004B
:109C5000007960B1514850F82400001DC5EBC501E2
:109C600000EB4100407940F08000B0425AD04B48B0
:109C700050F82400001DC5EBC50100EB41008079C0
:109C800050B1464850F82400001DC5EBC50100EB5B
:109C90004100C079B04245D0404850F82400001D32
:109CA000C5EBC50100EB4100007A60B13B4850F8BC
:109CB0002400001DC5EBC50100EB4100407A40F0D7
:109CC0008000B0422ED0354850F82400001DC5EB6E
:109CD000C50100EB4100807A68B1304850F824009B
:109CE000001DC5EBC50100EB4100C07AB04201E0A8
:109CF00021E01BE016D0294850F82400001DC5EBD8
:109D0000C50100EB4100007B80B1244850F82400DD
:109D1000001DC5EBC50100EB4100407B40F0800019
:109D2000B04203D131462046F9F7CAFF681CC5B2DC
:109D3000042DFFF466AF601CC4B2012CFFF654AFD3
:109D4000002426E0164850F82400C068F8B11448F2
:109D500050F82400007CB84219D1114850F8240072
:109D6000007D40F08000B0420DD00D4850F8240036
:109D7000407D40F08000B04205D0094850F82400F2
:109D8000807DB04203D131462046F9F79EFF601C2A
:109D9000C4B2012CD6DBBDE8F081000014EA041A3D
:109DA00084EA041A2DE9F041044604F00F06052E5A
:109DB00003D94FF0FF30BDE8F0811B48007800F078
:109DC000020010B94FF0FF30F5E72007C00E00EB9E
:109DD000D410164901EB801504F00F01E00901EBE6
:109DE0000011012000FA01F7E0094FEA00182046AF
:109DF00000F04CF80E4807600E4901EB8600D0F8E1
:109E0000C001402101FA08F108430A4A02EB860129
:109E1000C1F8C001E86820F0FF00E860002085F884
:109E20003F0000BFC7E700003101081000C8002054
:109E3000BC61004000600040014601F00F000528B1
:109E400001D9002070470807C00E00EBD110024A6C
:109E500002EB8010806BF5E700C800200548007811
:109E600000F0020008B90020704703480068C0F302
:109E7000CA00F9E7310108104C61004008B50248FA
:109E80000068009008BD00000CEA041B00F00F03FE
:109E9000C20903EB0213012202FA03F1044A116022
:109EA00000BF034A12680A40002AFAD17047000036
:109EB000B46100402DE9F04706463007C00E00EBC4
:109EC000D61A06F00F01F00901EB0011012000FA8B
:109ED00001F9234800EB8A15224800EB4A14A96BCC
:109EE000286B4718D5E90D01A0EB0108B8F5804FA4
:109EF00001D94FF4804800BF1B48006800EA090000
:109F00000028F9D120212046F9F722FD0120206008
:109F1000164901EA084141F4004141F080016068BE
:109F200008436060A76007F58050E06007F50050C7
:109F3000206107F54050606107F58040A061E86846
:109F400020F0FF00E860AC60A5F83C8006480838C7
:109F5000006840EA09000649C1F8B001BDE8F08791
:109F600000C8002000CB0020B86100400000FF7F47
:109F7000006000407CB54A4951F82050EC6894F8E4
:109F8000401011F01F0102D0012960D16FE0B4F838
:109F900042204449130A082B7FD2DFE803F07E04F5
:109FA00018517E7E0A3951F820004068A0631220C3
:109FB0005BE06A7C002A70D094F8352051F82000CC
:109FC0001AB1C068A0630A204FE08068FAE76B7C92
:109FD000002B94F8353007D03BB151F82000406990
:109FE00000900020D2B20BE08BBB51F8200000693A
:109FF000F6E700990B7813B14B8819440091401C87
:10A000008242F6D10098017809B3A06340882CE021
:10A010006B7CE3B194F8353051F8200023B1C0696E
:10A0200000900020D2B208E08069F9E700990B782F
:10A0300013B14B8819440091401C8242F6D1E1E7EC
:10A0400051F82000D1B2006A0090002006E024E020
:10A05000009A13780BB11A440092401C8142F7D148
:10A0600000980178C9B1A0630078019007E001AAC7
:10A070006946F9F72FFE00280ED00098A063E16B27
:10A080000198814207D9E063697D491E084202D1E7
:10A09000012084F8360001207CBD00207CBD00003A
:10A0A00090E9041AFC0100202DE9F04107463948E7
:10A0B00050F82700C46894F8400010F01F0004D046
:10A0C000012856D0022854D117E0B4F842000128E4
:10A0D0004FD141B1304850F8270000B18047208867
:10A0E00040F0020007E02D4850F8270000B18047FB
:10A0F000208820F00200208049E094F844001022DB
:10A1000000F08F0606F00F0002EAD6021044012587
:10A11000E27885406AB332072BD0A2682A4228D061
:10A12000B4F842202ABBC1B1E16829422FD12044B2
:10A13000007D20B131463846F9F777FDC8B90122D4
:10A1400031463846FFF75CFA98B9E0683146284353
:10A15000E0603846F9F7C3FD19E0E068284216D000
:10A160002069284213D1002231463846FFF748FAC9
:10A1700010B10020BDE8F081E0683146A843E060FE
:10A180003846F9F7B1FD31463846FFF727FD012083
:10A19000F0E7000090E9041A68EB041A6CEB041A6B
:10A1A0002DE9FC5F89498046002051F82870FC6841
:10A1B000009094F8400010F01F0F7CD194F84200FA
:10A1C0004FF0000A10F0FF0F4FF0010B4FF48039F1
:10A1D00072D0797C7E48002994F8351004D029B1DA
:10A1E00050F82800456997E00029E6D150F828008A
:10A1F000056991E06878022804D0042863D0052816
:10A200005ED163E0697994F84200814259D1E070EF
:10A21000287984F83400002003E07A6802F800A06E
:10A22000401C798A8142F8D85FF00106A1680BFAD8
:10A2300006F0014212D0A019007D28B131464046F7
:10A24000F9F7F3FC0028B8D131464046FFF71EFA73
:10A25000002830D131464046F9F741FDA16809FA9E
:10A2600006F0014216D0A01990F8240030B146F053
:10A2700080014046F9F7D9FC00281CD146F0800146
:10A2800040460191FFF702FA002814D14046019997
:10A29000F9F725FD761CF6B2102EC7D34FF001104A
:10A2A000C4E9020AC4F810A0E8794006208804D561
:10A2B00040F0010003E05BE033E020F0010020808B
:10A2C00028E0688827E0E878009023E0009808BB41
:10A2D000A878102200F08F0101F00F0002EAD102ED
:10A2E00010440BFA00F62044007D18B14046F9F7FF
:10A2F0009CFCE8BBA0683043A060E878AB8800F025
:10A300000302A9784046FFF733F988BBA978404695
:10A31000FFF764FC28780544287800287FF46AAFAA
:10A320003FE0564684F803A001255F46A06807FA7F
:10A3300005F1084210D06019007D20B12946404641
:10A34000F9F773FCA0B929464046FFF79FF978B9A1
:10A3500029464046F9F7C3FCA16809FA05F0014215
:10A3600016D0601990F8240038B145F0800100E063
:10A3700029E04046F9F759FC28BB45F080018A46A0
:10A380004046FFF783F9F0B951464046F9F7A7FC7C
:10A390006D1CEDB2102DC9D34FF00110C4E90206B7
:10A3A0002661E07894F8421088420CD1E17840466A
:10A3B00000F0DCF8074850F8281009B1E078884729
:10A3C0000120BDE8FC9F0020FBE7000090E9041A93
:10A3D000FC01002064EB041A10B500203B49086022
:10A3E00048603B4908704FF440713A48F9F7B0FAB9
:10A3F0004FF4C0713848F9F7ABFA01240DE0374942
:10A4000001EB8400D0F8C00120F080100A4602EB76
:10A410008401C1F8C001601CC4B2052CEFD94FF013
:10A42000FF302F49086000202C49C1F87C01401EF4
:10A43000C1F844012A4834300068C1F8AC0128480A
:10A440004430006826494431086000BF2448383051
:10A4500000680028FAD1401E21493C31086000BF45
:10A460001F483C3000680028FAD11D483838006881
:10A4700020F47F001949C1F840011A480078C0F360
:10A48000410002280AD1402200210846F9F731FC98
:10A49000402200218020F9F72CFC09E0082200214D
:10A4A0000846F9F726FC082200218020F9F721FC54
:10A4B00008480B49203908600848D0F8A80140F046
:10A4C000080007493031086010BD00004001081045
:10A4D0004801081000C8002000CB002000600040A8
:10A4E000786100403C01081070B5054600240EE07C
:10A4F000124850F8240040B1104850F82400007869
:10A50000A84202D12046FEF7DDFE601CC4B2012C39
:10A51000EEDB00240FE00A4850F82400C06840B188
:10A52000074850F82400007CA84202D12046F9F7E1
:10A53000E5FB601CC4B2012CEDDB70BD14EA041A0B
:10A5400084EA041A70B5084D0446502155F82400D9
:10A55000C068F9F7FDF955F82400017CC068C1F323
:10A560008011018070BD000090E9041A704700005E
:10A57000024A52F8200000F02FB80000A800002086
:10A5800000231A461946F9F73CBB000010B50446F3
:10A590000021F9F7B8FB08B1222010BD064850F899
:10A5A0002400C068007D0028F7D02046BDE8104098
:10A5B0008021F9F73ABB000090E9041A70B504460F
:10A5C0000D462946204620F017FB70BD10B5044605
:10A5D0002046F9F79DFB10BD70B504460D4629468F
:10A5E000204620F02BFB70BD70B504460D46164684
:10A5F00031462846F9F791FB84E8070070BD00005A
:10A6000010B500200C4908710C4C0EE02078102881
:10A6100004D160780021F9F785FB05E061782078A6
:10A620000022F9F726FA00BF083404484830844273
:10A63000ECD1002010BD0000B40C001078E9041B20
:10A6400010B5174817490860002211460C20F9F789
:10A6500010FA00220A210C20F9F70BFA002204213B
:10A660000C20F9F706FA002205210C20F9F701FA6F
:10A67000002206210C20F9F7FCF9002207210C200A
:10A68000F9F7F7F9002208210C20F9F7F2F9002276
:10A6900009210C20F9F7EDF900200349087510BDD8
:10A6A0000008000190000540B8860810002003490A
:10A6B00008604860088188727047000044310010CB
:10A6C0002DE9F04704464FF47A700F490968A0FB62
:10A6D000017001460D4A00233846F6F789F800223A
:10A6E000A0FB045701FB047100FB021104220023AC
:10A6F0002846F6F77DF8814600BFB9F10000A9F1C0
:10A700000109FAD1BDE8F0871402001000CA9A3B93
:10A7100010B5044621460248006814F085F910BDC2
:10A720006800002010B504462146024813F096FE4A
:10A7300010BD000020B1002070B50446264600255B
:10A740003046F5F7D6FF05460DB9002070BD284606
:10A75000FCE700000FB5ADF2FC6D0020CDF8F80667
:10A76000CDF8F406CDF8F006CDF8EC06CDF8E80605
:10A77000CDF8E406CDF8E006CDF8DC06CDF8D80635
:10A78000CDF8D406CDF8D006CDF8CC06B190B09077
:10A79000AF90AE904FF4007127A8F9F7D9F80020D8
:10A7A00020901F901E901C901B900F90F749DDF891
:10A7B00004070860F649DDF808070860DDF80007BF
:10A7C00034287DDDDDF8FC0600784FF07F4101EA9A
:10A7D0000060DDF8FC1649784FF47F0202EA01417F
:10A7E0000843DDF8FC168978121202EA01210843B9
:10A7F000DDF8FC16C9780843CDF8F406DDF8F40658
:10A8000000F0010020902098401CDDF8241708601B
:10A810002098C0001F90DDF8FC060079110401EAC1
:10A820000060DDF8FC164979120202EA0141084392
:10A83000DDF8FC168979121202EA01210843DDF8DD
:10A84000FC16C9790843CDF8F006DDF8FC06007A5D
:10A85000110401EA0060DDF8FC16497A120202EAEE
:10A8600001410843DDF8FC16897A121202EA01213F
:10A870000843DDF8FC16C97A0843CDF8EC061F98AA
:10A88000001DDDF8FC16085C110401EA00611F9848
:10A89000401DDDF8FC26105C4FF47F0202EA004008
:10A8A00008431F99891DDDF8FC26515C4FF47F4257
:10A8B00002EA012108431F99C91DDDF8FC2600E0CA
:10A8C0000AE1515C0843CDF8E8061F981030DDF826
:10A8D000FC16085C4FF07F4101EA00611F981130BF
:10A8E000DDF8FC26105C4FF47F0202EA00400843CA
:10A8F0001F991231DDF8FC26515C4FF47F4202EAC9
:10A90000012108431F991331DDF8FC26515C0843EF
:10A91000CDF8E4061F981430DDF8FC16085C4FF003
:10A920007F4101EA00611F981530DDF8FC26105CBC
:10A930004FF47F0202EA004008431F991631DDF808
:10A94000FC26515C4FF47F4202EA012108431F9923
:10A950001731DDF8FC26515C0843CDF8E0061F985E
:10A960001830DDF8FC16085C4FF07F4101EA006109
:10A970001F981930DDF8FC26105C4FF47F0202EAC4
:10A98000004008431F991A31DDF8FC26515C4FF452
:10A990007F4202EA012108431F991B31DDF8FC26A2
:10A9A000515C0843CDF8DC061F981C30DDF8FC161E
:10A9B000085C4FF07F4101EA00611F981D30DDF80F
:10A9C000FC26105C4FF47F0202EA004008431F9906
:10A9D0001E31DDF8FC26515C4FF47F4202EA012172
:10A9E00008431F991F31DDF8FC26515C0843CDF860
:10A9F000D8061F982830DDF8FC16085C4FF07F4120
:10AA000001EA00611F982930DDF8FC26105C4FF444
:10AA10007F0202EA004008431F992A31DDF8FC2634
:10AA2000515C4FF47F4202EA012108431F992B3108
:10AA3000DDF8FC26515C0843CDF8D4061F982C3075
:10AA4000DDF8FC16085C4FF07F4101EA00611F98B9
:10AA50002D30DDF8FC26105C4FF47F0202EA004046
:10AA600008431F992E31DDF8FC26515C4FF47F42DC
:10AA700002EA012108431F992F31DDF8FC26515CC1
:10AA80000843CDF8D0061F9840003030DDF8FC16A2
:10AA9000085C4FF07F4101EA00611F9840003130AF
:10AAA000DDF8FC26105C4FF47F0202EA0040084308
:10AAB0001F9949003231DDF8FC26515C4FF47F428A
:10AAC00002EA012108431F9949003331DDF8FC26D1
:10AAD000515C0843CDF8CC062E49DDF8F4068842D7
:10AAE00009D0491CDDF8F406884204D001201C90EE
:10AAF0000220CDF8F806DDF8F80600287ED1DDF852
:10AB0000CC0600287AD0DDF8CC0680000A90FFF74A
:10AB100013FEB190B19810B90120CDF8F806DDF818
:10AB2000F80658B9DDF8CC0680000A90FFF704FE5D
:10AB3000B090B09810B90120CDF8F806DDF8F8060D
:10AB400048B9DDF8CC06FFF7F7FDAF90AF9810B924
:10AB50000120CDF8F806DDF8F80660B92098002845
:10AB600009DDDDF8D006FFF7E7FDAE90AE9810B92D
:10AB70000120CDF8F806DDF8F8060028BED12098AF
:10AB800040001F90002014905BE10000B40008100A
:10AB9000B8000810004D414A1F980B30DDF8E4263C
:10ABA000149900FB012011901198C01C1F990144B9
:10ABB000DDF8FC06405C4FF07F4101EA006111982E
:10ABC000C01C1F9A1044401CDDF8FC26105C4FF49A
:10ABD0007F0202EA004001431198C01C1F9A1044F2
:10ABE000801CDDF8FC26105C4FF47F4202EA002056
:10ABF00001431198C01C1F9A104400E027E1C01CBB
:10AC0000DDF8FC26105C01431091DDF8FC1611986C
:10AC10000A5C1499AF9842541499AF98405C00F0C4
:10AC20007F02AF9842541198C01D1F990144DDF86E
:10AC3000FC06405C4FF07F4101EA00611198C01DA5
:10AC40001F9A1044401CDDF8FC26105C4FF47F0274
:10AC500002EA004001431198C01D1F9A1044801C55
:10AC6000DDF8FC26105C4FF47F4202EA002001432D
:10AC70001198C01D1F9A1044C01CDDF8FC26105C02
:10AC80000143149AB09840F822101499AF98405C90
:10AC900000F00C00042805D1149AB199109841F8DD
:10ACA0002200CBE01499AF98405C00F01E000E2803
:10ACB00047D11099DDF8E0060144DDF8FC060844B0
:10ACC0000A9002F0F7FE12901298FFF735FD149AE1
:10ACD000B19941F822001499B19850F8210018B99F
:10ACE0000120CDF8F806A9E01499AF98405C40F037
:10ACF0008002AF984254209800901499B19850F86F
:10AD000021000A90B09850F8210009901099DDF8C0
:10AD1000E0060144DDF8FC0608440890129BDDE9DA
:10AD20000912F9F704F81299884203D00220CDF8ED
:10AD3000F80683E01298C2001499B09840F82120D8
:10AD40007CE01499AF98405C00F01E000C280BD1F9
:10AD5000DDF8E01610980144DDF8FC060A18149995
:10AD6000B19840F8212069E01499AF98405C00F058
:10AD70001C001C2808D1DDF8E01610984218149920
:10AD8000B19840F8212059E01499AF98405C00F048
:10AD90000C0008284DD11499AF98405C40F0800217
:10ADA000AF9914980A541499B09850F821000028CB
:10ADB00039DD1499AF98405C00F0100030B114995F
:10ADC000B09850F8210080000A900AE01499B098D9
:10ADD00050F82100C01DC117099000EB5170C01040
:10ADE0000A900A98FFF7A8FC149AB19941F822003A
:10ADF0001499B19850F8210018B90120CDF8F8063F
:10AE000010E00020139009E000221499B19850F846
:10AE1000211013980A541398401C13900A99139800
:10AE20008842F1D30AE000221499B19840F8212019
:10AE300004E000221499B19840F821201498401C95
:10AE40001490DDF8CC1614988842FFF4A5AEDDF816
:10AE5000F80600287ED1DDF8140700287AD0209863
:10AE6000002877D1209840001F9000201A9090E091
:10AE70001A99DDF8140750F821000E9000200D906B
:10AE800005E00E98401C0E900D98401C0D900E98F9
:10AE900000783D2803D00E9800780028F1D10E9854
:10AEA00000783D2872D10E98401C0E900E98F8F74D
:10AEB00043FF10901A99DDF8140750F821000A900A
:10AEC0000146B2A80D9AF8F73CFF0021B2AA0D98EE
:10AED00011540020149054E01F980B30DDF8E42644
:10AEE000149900FB01201190209878B91198401C0A
:10AEF000DDF8FC16085C4FF47F4101EA002111984F
:10AF0000801CDDF8FC26105C084322E01198401CF0
:10AF1000DDF8FC16085C4FF07F4101EA00611198F2
:10AF2000801CDDF8FC26105C4FF47F0202EA004032
:10AF300008431199C91CDDF8FC26515C4FF47F428F
:10AF400002EA012108431199091DDDF8FC26515C34
:10AF5000084300E025E0A790DDF8E816A798014433
:10AF6000DDF8FC0608440B90B2A80B99F8F7EEFE4A
:10AF700020B9149AB199109841F822001498401CF5
:10AF80001490DDF8CC1614988842A5D31A98401C6A
:10AF90001A901A99DDF8140750F8210000287FF460
:10AFA00067AFDDF8F80608B101201C90F8F7D3FE72
:10AFB000DDF8DC06AD9000208DF8C802209800284E
:10AFC0007EDDDDF8100728B91820CDF8F80601203D
:10AFD0001C9095E000200A90149080E00C221499B7
:10AFE000DDF8F00602FB0101DDF8FC06405C4FF0E5
:10AFF0007F4101EA00600C23149ADDF8F01603FB90
:10B000000211491CDDF8FC26515C4FF47F0202EA74
:10B0100001410843149ADDF8F01603FB0211891C64
:10B02000DDF8FC26515C4FF47F4202EA012108431F
:10B03000149ADDF8F01603FB0211C91CDDF8FC269A
:10B04000515C0843A790A799DDF8E8060144DDF8B4
:10B05000FC0608440B900B99DDF81007F8F776FE14
:10B0600078BB01200A900C221499DDF8F00602FB4F
:10B0700001000830DDF8FC16085C4FF07F4101EA62
:10B0800000610C23149ADDF8F00603FB020009307E
:10B09000DDF8FC26105C4FF47F0202EA0040084312
:10B0A000DDF8F026149903FB01210A31DDF8FC26B6
:10B0B000515C4FF47F4202EA01210843149A01E0F7
:10B0C000A0E009E0DDF8F01603FB02110B31DDF81A
:10B0D000FC26515C08430F901498401C1490DDF836
:10B0E000D4161498884203D20A9800283FF476AF09
:10B0F0000A9820B91820CDF8F80601201C9000BF4E
:10B10000DDF8F80600287DD101200A900F981490F0
:10B11000E3E000200A900D221499DDF8EC0602FB12
:10B1200001000830DDF8FC16085C00F003021499F9
:10B13000AE9842541499AE98405C00287ED0DDF859
:10B14000140700287AD00D221499DDF8EC0602FBD2
:10B150000101DDF8FC06405C4FF07F4101EA006030
:10B160000D23149ADDF8EC1603FB0211491CDDF8DF
:10B17000FC26515C4FF47F0202EA01410843149A15
:10B18000DDF8EC1603FB0211891CDDF8FC26515C8E
:10B190004FF47F4202EA01210843149ADDF8EC16CD
:10B1A00003FB0211C91CDDF8FC26515C0843A79083
:10B1B000A799DDF8E8060144DDF8FC0608440B9089
:10B1C00000201A904CE01A99DDF8140750F821007D
:10B1D0000E9000200D9005E00E98401C0E900D98EA
:10B1E000401C0D900E9800783D2803D00E980078F2
:10B1F0000028F1D10E9800783D282ED10E98401CE1
:10B200000E9000E015E11A99DDF8140750F82100BE
:10B2100009900146B2A80D9AF8F793FD0021B2AA51
:10B220000D981154B2A80B99F8F790FDA8B90E9893
:10B23000F8F782FD50B91499AE9800E017E0405C31
:10B2400040F04002AE9914980A5406E01499AE9862
:10B25000405C40F08002AE9842541A98401C1A900C
:10B260001A99DDF8140750F821000028ABD10D22FF
:10B27000DDF8EC16149802FB0010001DDDF8FC163A
:10B28000085C4FF07F4101EA00610D23149ADDF85C
:10B29000EC0603FB0200401DDDF8FC26105C4FF4B9
:10B2A0007F0202EA00400843149ADDF8EC1603FB23
:10B2B0000211891DDDF8FC26515C4FF47F4202EA41
:10B2C00001210843149ADDF8EC1603FB0211C91D95
:10B2D000DDF8FC26515C08431490149800287FF494
:10B2E00018AF0A980028FAD10F98149035E00D2273
:10B2F0001499DDF8EC0602FB0100001DDDF8FC16D8
:10B30000085C4FF07F4101EA00610D23149ADDF8DB
:10B31000EC0603FB0200401DDDF8FC26105C4FF438
:10B320007F0202EA00400843149ADDF8EC1603FBA2
:10B330000211891DDDF8FC26515C4FF47F4202EAC0
:10B3400001210843149ADDF8EC1603FB0211C91D14
:10B35000DDF8FC26515C08431490149858B11499F8
:10B36000AE98405C0128C2D01499AE98405C00F0C1
:10B37000C0004028BBD0149868B91498F0BB0F984F
:10B38000E0BBAE980078012850D0AE98007800F06D
:10B39000C00040284AD014980F900D22DDF8EC161A
:10B3A000149802FB00100930DDF8FC16085C4FF021
:10B3B0007F4101EA00610D23DDF8EC26149803FBC0
:10B3C00000200A30DDF8FC26105C4FF47F0202EA10
:10B3D00000400843DDF8EC26149903FB01210B31F2
:10B3E000DDF8FC26515C4FF47F4202EA012108435C
:10B3F000DDF8EC26149903FB012100E016E00C3186
:10B40000DDF8FC26515C0843DDF8DC160844AD90FD
:10B41000DDF8DC16AD98884204D3DDF8D816AD9877
:10B42000884205D30B20CDF8F80601E001201C90DE
:10B4300000BF00208DF8C80202F051B8AD99DDF8C8
:10B44000FC06405CA890AD98AC90AD98401CAD90C7
:10B45000A89880091D90002014902BE0AD99DDF88C
:10B46000FC06405C4FF07F4101EA0062AD98401C51
:10B47000DDF8FC16085C4FF47F0101EA0040104340
:10B48000AD99891CDDF8FC26515C4FF47F4202EA3D
:10B4900001210843AD99C91CDDF8FC26515C084325
:10B4A000A9AA149942F82100AD98001DAD901498F6
:10B4B000401C14901D9914988842CFD3A8982A282C
:10B4C0006FD019DC2A2881F0EC87DFE800F0787A69
:10B4D0008EAAC3EEEDECEBEAE9E8E7E6E5E4E3E2A9
:10B4E000E1E0DFDEDDDCDBDAD9D8D7D6D5D4D3D2C4
:10B4F000D1D0CFCECDCCCBCA502801F036812ADCBA
:10B50000A0F12B002528DED2DFE810F05B055E05F8
:10B51000770571067406CB0FCB0FCB0FCB0FCB0F7C
:10B52000CB0FCB0FCB0FCB0FCB0FCB0FCB0FCB0F4B
:10B53000CB0FCB0FCB0F7C0684068F06A206BC0672
:10B540000B0727072A0732073A0742074A076D0702
:10B550008607980733085B2801F0B7830FDCA0F15A
:10B5600051000A28AFD2DFE810F021092209BA09F8
:10B57000E3090C0A350A5E0A790ADA0A390B8328CC
:10B5800001F099850EDC5C2801F0A283802801F08F
:10B590004484812801F08B85822841F0828701F064
:10B5A00089BDF9E3842801F07686852801F0B98603
:10B5B000C02801F0B986C128EFD101F06FBF01F0BA
:10B5C00073BF1E98012803DA1420CDF8F8060BE0AB
:10B5D0001E98401E27A951F8201027AA1E9842F84D
:10B5E00020101E98401C1E90E9E71E98022803DADE
:10B5F0001420CDF8F80613E01E98801E27A951F8F4
:10B60000200025901E98401E51F820101E98801E84
:10B6100027AA42F820101E98401E259942F82010B3
:10B62000CDE71E98022803DA1420CDF8F80610E0C2
:10B630001E98401E1E901E98401E27A951F82010EB
:10B6400027AA1E9852F8200001441E98401E42F876
:10B650002010B4E71E98022828DA1420CDF8F80646
:10B6600035E0FDE3FDE3FDE3FDE3FDE3FDE3FDE3A5
:10B67000FDE3DEE3C7E3A6E38FE36DE356E352E3C6
:10B680004EE34AE31EE3FDE2D1E2B0E2A8E28EE23D
:10B690004AE24FE130E111E1FAE0E0E0C6E0ACE07F
:10B6A00098E07EE064E046E02BE011E01E98401E4A
:10B6B0001E901E98401E27A951F8201027AA1E98F8
:10B6C00052F82000091A1E98401E42F8201076E712
:10B6D0001E98022803DA1420CDF8F80610E01E9810
:10B6E000401E1E901E98401E27A951F8201027AA20
:10B6F0001E9852F8200041431E98401E42F8201028
:10B700005DE71E98022803DA1420CDF8F80611E050
:10B710001E98401E1E901E98401E27A951F820100A
:10B7200027AA1E9852F8200091FBF0F11E98401EA7
:10B7300042F8201043E71E98022803DA1420CDF8BF
:10B74000F80614E01E98401E1E901E98401E27A961
:10B7500051F8201027AA1E9852F8200091FBF0F211
:10B7600000FB12111E98401E27AA42F8201026E75F
:10B770001E98022803DA1420CDF8F80610E01E986F
:10B78000401E1E901E98401E27A951F8201027AA7F
:10B790001E9812F8200081401E98401E42F820108A
:10B7A0000DE71E98022803DA1420CDF8F80610E001
:10B7B0001E98401E1E901E98401E27A951F820106A
:10B7C00027AA1E9812F8200001411E98401E42F838
:10B7D0002010F4E61E98012803DA1420CDF8F806AC
:10B7E0000AE01E98401E27A951F82000C1431E9868
:10B7F000401E27AA42F82010E1E61E98022803DA2C
:10B800001420CDF8F80610E01E98401E1E901E98D9
:10B81000401E27A951F8201027AA1E9852F8200090
:10B8200001401E98401E42F82010C8E61E980228CB
:10B8300003DA1420CDF8F80610E01E98401E1E9082
:10B840001E98401E27A951F8201027AA1E9852F8CA
:10B85000200001431E98401E42F82010AFE61E98BB
:10B86000022803DA1420CDF8F80610E01E98401ED6
:10B870001E901E98401E27A951F8201027AA1E9836
:10B8800052F8200041401E98401E42F8201096E6D3
:10B890001E98012803DA1420CDF8F8060DE01E9852
:10B8A000401E27A951F8200008B9012100E000211D
:10B8B0001E98401E27AA42F8201080E61E980228F3
:10B8C00003DA1420CDF8F80615E01E98401E1E90ED
:10B8D0001E98401E27A951F8201027AA1E9852F83A
:10B8E0002000814201DD012100E000211E98401E60
:10B8F00027AA42F8201062E61E98022803DA1420D4
:10B90000CDF8F80615E01E98401E1E901E98401EA9
:10B9100027A951F8201027AA1E9852F8200081422A
:10B9200001DA012100E000211E98401E27AA42F8FA
:10B93000201044E62098002838DD1E98B0BB0D2268
:10B94000DDF8EC160F9802FB0010001DDDF8FC1668
:10B95000085C4FF07F4101EA00610D230F9ADDF88A
:10B96000EC0603FB0200401DDDF8FC26105C4FF4E2
:10B970007F0202EA004008430F9ADDF8EC1603FB51
:10B980000211891DDDF8FC26515C4FF47F4202EA6A
:10B99000012108430F9ADDF8EC1603FB0211C91DC3
:10B9A000DDF8FC26515C0843149036E095E00D224A
:10B9B0001499DDF8EC0602FB0100001DDDF8FC1611
:10B9C000085C4FF07F4101EA00610D23149ADDF815
:10B9D000EC0603FB0200401DDDF8FC26105C4FF472
:10B9E0007F0202EA00400843149ADDF8EC1603FBDC
:10B9F0000211891DDDF8FC26515C4FF47F4202EAFA
:10BA000001210843149ADDF8EC1603FB0211C91D4D
:10BA1000DDF8FC26515C08431490149858B1149931
:10BA2000AE98405C0128C2D01499AE98405C00F0FA
:10BA3000C0004028BBD0149830B901201C900021D0
:10BA4000DDF8200701606EE014980F900D22DDF8FC
:10BA5000EC16149802FB00100930DDF8FC16085CA7
:10BA60004FF07F4101EA00610D23DDF8EC261498C8
:10BA700003FB00200A30DDF8FC26105C4FF47F0247
:10BA800002EA00400843DDF8EC26149903FB01218B
:10BA90000B31DDF8FC26515C4FF47F4202EA0121B4
:10BAA0000843DDF8EC26149903FB01210C31DDF885
:10BAB000FC26515C0843DDF8DC160844AD90DDF847
:10BAC000DC16AD98884204D3DDF8D816AD988842CC
:10BAD00029D30B20CDF8F80625E01E98012803DABB
:10BAE0001420CDF8F8061EE01E98401E27A91E90CF
:10BAF00051F82010DDF8DC060844AD90DDF8DC16C6
:10BB0000AD98884204D3DDF8D816AD98884202D3A8
:10BB10000B20CDF8F806DDF8DC16AD98884202D18E
:10BB20000B20CDF8F8064AE51E98042803DA142005
:10BB3000CDF8F8063AE01E98401E27A91E9051F84D
:10BB400020000A901E98401E1E9051F82000099077
:10BB50001E98401E1E9051F8200025901E98401EF1
:10BB600051F820001A901A9810B11A98202803D979
:10BB70000B20CDF8F80618E01A98C0F120014FF01C
:10BB8000FF30084125990840259025990A980140E1
:10BB9000259A09981040814201D1012100E000213D
:10BBA0001E98401E27AA42F8201000BF07E51E98E5
:10BBB000012803DA1420CDF8F80610E0B2A8F8F74F
:10BBC000CFF8B2A908440A901E98401E27A91E90DB
:10BBD00051F82000014609900A98F8F7C6F8EEE4FB
:10BBE000B2A8F8F7C7F800208DF8C802E7E41E985D
:10BBF000022803DA1420CDF8F80617E01E98401E3C
:10BC000027A91E9051F8200025901E98401E1E90D6
:10BC100051F820001A9026A8259902F0E9F900228F
:10BC200026A91A98F8F7ABF8CDF8F806C7E41E98DD
:10BC3000022803DA1420CDF8F80622E01E98401EF0
:10BC400027A91E9051F8200025901E98401E51F8FB
:10BC500020001A9026A8259902F0CAF9002026ABE8
:10BC6000024626A900901A9801F07CFCCDF8F8064F
:10BC700026A801F01FFF01461E98401E27AA42F881
:10BC800020109CE41E98022803DA1420CDF8F80650
:10BC900017E01E98401E27A91E9051F820002590FD
:10BCA0001E98401E1E9051F820001A9026A8259933
:10BCB00002F09EF9002226A91A9801F04FFECDF855
:10BCC000F8067CE41E98022803DA1420CDF8F80662
:10BCD00022E01E98401E27A91E9051F820002590B2
:10BCE0001E98401E51F820001A9026A8259902F0AF
:10BCF0007FF9002026AB024626A900901A98F8F793
:10BD000043F8CDF8F80626A801F0D4FE01461E98A7
:10BD1000401E27AA42F8201051E401201B904EE457
:10BD200001201B904BE401201B9048E41E98012841
:10BD300003DA1420CDF8F8060DE01E98401E27A95E
:10BD40001E9051F820001A90002211461A9802F015
:10BD5000E9FFCDF8F80632E41E98022803DA142031
:10BD6000CDF8F80617E01E98401E27A91E9051F83E
:10BD700020001A901E98401E1E9051F82000259019
:10BD800026A8259902F034F926AA00211A9802F073
:10BD9000C9FFCDF8F80612E410E11E98012803DA75
:10BDA0001420CDF8F8060DE01E98401E27A91E901D
:10BDB00051F820001A90002211461A9803F02AF830
:10BDC000CDF8F80610E41E98022803DA1420CDF806
:10BDD000F80617E01E98401E27A91E9051F8200073
:10BDE0001A901E98401E1E9051F82000259026A8FB
:10BDF000259902F0FDF826AA00211A9803F00AF806
:10BE0000CDF8F8060CE41E98012803DA1420CDF8CA
:10BE1000F8060DE01E98401E27A91E9051F820003C
:10BE20001A90002211461A98F7F7B3FFCDF8F806DA
:10BE30000FE41E98022803DA1420CDF8F80620E05B
:10BE40001E98401E27A91E9051F820001A901E9897
:10BE5000401E1E9051F82000259026A8259907E045
:10BE6000A9E0A5E099E07AE066E041E020E009E0A1
:10BE700002F0BEF826AA00211A98F7F78AFFCDF83B
:10BE8000F80624E41E98012803DA1420CDF8F806F9
:10BE90000DE01E98401E27A91E9051F820001A9010
:10BEA000002211461A98F7F779FFCDF8F8060EE44C
:10BEB0001E98022803DA1420CDF8F80617E01E9821
:10BEC000401E27A91E9051F820001A901E98401E6F
:10BED0001E9051F82000259026A8259902F088F898
:10BEE00026AA00211A98F7F759FFCDF8F80607E4BB
:10BEF0001E98012803DA1420CDF8F8061BE0B2A83A
:10BF0000F7F72EFF1A901E98401E27A91E9011F8D1
:10BF100020000A900A98012802DB0A987F2801DD98
:10BF20007F200A90B2AA1A990A98505400211A98B0
:10BF3000401C115400BF1AE41E98012803DA142093
:10BF4000CDF8F80608E01E98401E27A91E9051F86B
:10BF50002010DDF82007016001201C9007E41E98E6
:10BF6000022803DA1420CDF8F80615E01E98401ECA
:10BF70001E901E98401E27A951F8201027AA1E982F
:10BF800052F82000814201D1012100E000211E98D9
:10BF9000401E27AA42F820101BE41E98012803DA4D
:10BFA0001420CDF8F80602E01E98401E1E9010E402
:10BFB00001201B900DE401201B900AE401201B903E
:10BFC00007E401201B9004E41E98012803DA1420E2
:10BFD000CDF8F80610E01E98401E27A951F8200061
:10BFE000002809DA1E98401E51F8200041421E9890
:10BFF000401E27AA42F8201017E41E98022803DAF0
:10C000001420CDF8F80613E01E98801E27A951F8D9
:10C01000200025901E98401E51F820101E98801E6A
:10C0200027AA42F820101E98401E259942F8201099
:10C030000820199019991E98884203DA1420CDF827
:10C04000F80616E019991E98401A27A951F8200001
:10C0500025901E98401E51F8202019991E98401ACC
:10C0600027A941F820201E98401E27AA259942F8AA
:10C0700020101E98022803DA1420CDF8F80613E0E9
:10C080001E98801E27A951F8200025901E98401E5A
:10C0900051F820101E98801E27AA42F820101E98E2
:10C0A000401E259942F82010072019901E991998D2
:10C0B000814203DA1420CDF8F80616E019991E988B
:10C0C000401A27A951F8200025901E98401E51F8CB
:10C0D000202019991E98401A27A941F820201E985F
:10C0E000401E27AA259942F8201009201990199975
:10C0F0001E98884203DA1420CDF8F8060CE019994E
:10C100001E98401A27A951F8201027AA1E9842F815
:10C1100020101E98401C1E900320199019991E98FB
:10C12000884203DA1420CDF8F80616E019991E9813
:10C13000401A27A951F8200025901E98401E51F85A
:10C14000202019991E98401A27A941F820201E98EE
:10C15000401E27AA259942F820101E98022803DACB
:10C160001420CDF8F80613E01E98801E27A951F878
:10C17000200025901E98401E51F820101E98801E09
:10C1800027AA42F820101E98401E259942F8201038
:10C190000720199019991E98884203DA1420CDF8C7
:10C1A000F8060CE019991E98401A27A951F820109A
:10C1B00027AA1E9842F820101E98401C1E900720A7
:10C1C000199019991E98884203DA1420CDF8F806C0
:10C1D0000CE019991E98401A27A951F8201027AA97
:10C1E0001E9842F820101E98401C1E909BE40120CF
:10C1F0001B9098E400221E99481C1E9027A840F826
:10C20000212090E41E98411CA99A1E9127A941F86B
:10C21000202088E4A999B19850F821201E98411C4B
:10C220001E9127A941F820207DE4A999DDF8DC06BC
:10C230000844AD90DDF8DC16AD98884204D3DDF8F3
:10C24000D816AD98884202D30B20CDF8F8066AE4E0
:10C250001E98421CAD991E9227AA42F82010A99957
:10C26000DDF8DC060844AD90DDF8DC16AD988842B8
:10C2700004D3DDF8D816AD98884202D30B20CDF850
:10C28000F80650E41E98032803DA1420CDF8F806C7
:10C2900046E01E98401E27A951F820000A901E98DB
:10C2A000801E51F8200009901E98C01E51F82000F1
:10C2B0000890A999B19850F82100079000200690A5
:10C2C0000A98002806DA09990798884208DC0120B4
:10C2D000069005E009990798884201DB0120069045
:10C2E000069818B11E98C01E1E9018E00A9907986B
:10C2F0000144A99AB19840F82210DDF8DC1608989C
:10C300000844AD90DDF8DC16AD98884204D3DDF822
:10C31000D816AD98884202D30B20CDF8F80600BF9E
:10C3200044E4B2A8F7F71CFD1A901A98C0F5806093
:10C330000A90A999DDF8E8060144DDF8FC060844F6
:10C34000B2A909901A9808440890DDE90912F7F794
:10C35000F8FC00208DF8C80628E401201B9025E495
:10C36000A99840B20A9002F061FCCDF8F8061DE4ED
:10C37000A99840B20A9002F059FCCDF8F80615E4ED
:10C38000A99840B20A9002F0BDFDCDF8F8060DE480
:10C39000A99840B20A90F7F706FDCDF8F80605E433
:10C3A000A998401C199019991E98884203DA142004
:10C3B000CDF8F80616E019991E98401A27A951F8E9
:10C3C000200025901E98401E51F8202019991E9893
:10C3D000401A27A941F820201E98401E27AA259917
:10C3E00042F8201022E4A998401C199019991E982F
:10C3F000884203DA1420CDF8F8060CE019991E984B
:10C40000401A27A951F8201027AA1E9842F8201098
:10C410001E98401C1E9009E41E98012803DA14207F
:10C42000CDF8F80609E01E98401E27A91E9051F885
:10C430002010A99AB19840F8221022E41E980228F0
:10C4400003DA1420CDF8F80692E0A99924912098F7
:10C4500000286DDD2499AF98405C00F09C001C28FA
:10C4600066D12499B09850F821001A902499B19877
:10C4700050F8210025901A9880000A90FEF75CF988
:10C480002190249AB199219841F822002499B198D9
:10C4900050F8210018B90120CDF8F80611E4002069
:10C4A00014902BE02599DDF8FC06405C4FF07F41AD
:10C4B00001EA00622598401CDDF8FC16085C4FF488
:10C4C0007F0101EA004010432599891CDDF8FC2614
:10C4D000515C4FF47F4202EA012108432599C91CAF
:10C4E000DDF8FC26515C0843149A219941F822009A
:10C4F0002598001D25901498401C14901A991498A2
:10C500008842CFD32499AF98405C40F08002AF9925
:10C5100024980A542499AF98405C20F00402AF9804
:10C5200042542499AF98405C40F00102AF984254C5
:10C530002499AF98405C00F01C00182803D00B2011
:10C54000CDF8F80614E02499B19850F82100219014
:10C550001E98401E27A91E9051F8200019901E9881
:10C56000401E1E9051F820201999219840F8212052
:10C5700011E41E98032803DA1420CDF8F806F3E03E
:10C58000A99924912098002872DD2499AF98405CE5
:10C5900000F09C000C286BD12499B09850F8210031
:10C5A000C01DC01025902499B19850F82100229008
:10C5B0002598FEF7C1F82390DDE92302B19941F8EF
:10C5C00022002499B19850F8210018B90120CDF823
:10C5D000F8064DE00020169006E0002216992398F8
:10C5E00042541698401C1690259916988842F4DB00
:10C5F0000020169020E0169815902299159801EBCE
:10C60000E0000178159800F00702012090400140F9
:10C6100079B11699239800EBE100007801F0070248
:10C62000012191400843C2B21699239800EBE10022
:10C6300002701698401C16902499B09850F821105A
:10C6400016988142D7DC2499AF98405C40F0800274
:10C65000AF9842542499AF98405C20F00402AF9800
:10C6600042542499AF98405C40F00102AF98425484
:10C670002499AF98405C00F01C00082803D00B20E0
:10C68000CDF8F80670E02499B19850F82100239075
:10C690001E98401E27A91E9051F8200017901E9842
:10C6A000401E1E9051F82000169000200C902098FB
:10C6B000002817DDDDE9160188420EDD01200C900F
:10C6C000179925911698411C1798081A17902598C4
:10C6D00016900B20CDF8F80609E41798401C16991F
:10C6E000401A17901E98401E27A91E9051F820004E
:10C6F00025901798012803DA0B20CDF8F80633E0CF
:10C70000002014902CE00121149801FA00F02599E2
:10C71000084080B11699239800EBE100007801F001
:10C720000702012191400843C2B21699239800EBF9
:10C73000E10002700EE01699239800EBE10000780A
:10C7400001F00702012191408843169A239901EBD9
:10C75000E20108701698401C16901498401C149022
:10C76000179914988842CED316E41E98012803DA4C
:10C770001420CDF8F80618E01E98401E27A91E9038
:10C7800051F8200088B9A999DDF8DC060844AD907D
:10C79000DDF8DC16AD98884204D3DDF8D816AD98E4
:10C7A000884202D30B20CDF8F80606E400BF1E989D
:10C7B000022803DA1420CDF8F8068FE01E98401EF8
:10C7C00027A91E9051F8200016901E98401E1E901A
:10C7D00051F82000179000200C90209800280FDDC1
:10C7E000179825901E98401E1E9051F82000179013
:10C7F00025991698884203DD01200C902598169003
:10C80000A999B19850F8210023900C9898B32399D6
:10C8100022910121179801EBE0000A90FDF78CFFAF
:10C820002390239818B90120CDF8F806DEE4DDE95D
:10C8300016010844401E25900020159031E02599EE
:10C84000229800EBE100007801F0070201219140FD
:10C85000084088B11599239800EBE100007801F0B9
:10C860000702012191400843C2B21599239800EBB9
:10C87000E10002700FE018E01599239800EBE10049
:10C88000007801F00702012191408843159A23990D
:10C8900001EBE20108702598401E25901598401C78
:10C8A0001590179915988842C9DBA898512807D187
:10C8B000DDE916202399F7F762FACDF8F80606E0CD
:10C8C000DDE91620239901F049F8CDF8F8060C9817
:10C8D00020B1239810B1239803F026FD86E41E981A
:10C8E000022803DA1420CDF8F80620E01E98401E36
:10C8F00027A91E9051F8200019901E98401E1E90E6
:10C9000051F820001A902098002804DD1A98401C45
:10C910001999401A1A90A999B19850F821002390BA
:10C92000239ADDE9191002F0FDF9CDF8F8065DE46F
:10C930001E98022803DA1420CDF8F80620E01E988D
:10C94000401E27A91E9051F8200019901E98401EE5
:10C950001E9051F820001A902098002804DD1A98A3
:10C96000401C1999401A1A90A999B19850F82100C1
:10C970002390239ADDE9191002F04CFACDF8F8065D
:10C9800034E41E98022803DA1420CDF8F80620E0DB
:10C990001E98401E27A91E9051F8200019901E983D
:10C9A000401E1E9051F820001A902098002804DDA7
:10C9B0001A98401C1999401A1A90A999B19850F8E0
:10C9C00021002390239ADDE91910F7F7E2F9CDF859
:10C9D000F8060BE41E98022803DA1420CDF8F806B6
:10C9E00020E01E98401E27A91E9051F820001990A3
:10C9F0001E98401E1E9051F820001A902098002882
:10CA000004DD1A98401C1999401A1A90A999B198F6
:10CA100050F821002390239ADDE91910F7F7BEF9A9
:10CA2000CDF8F80613E41E98012803DA1420CDF897
:10CA3000F80612E0A999DDF8E8060144DDF8FC06E5
:10CA400008440B901E98401E27A91E9051F8200004
:10CA5000259025990B9802F04BF812E41E980128B6
:10CA600003DA1420CDF8F80658E0A99924911E980D
:10CA7000401E27A951F8200019902499AF98405CD6
:10CA800000F01F0019280ED12499B19850F8210008
:10CA900021901999219850F821101E98401E27AA1C
:10CAA00042F820103AE02499AF98405C00F01F0053
:10CAB0001C2830D12499B19850F8211004221998DB
:10CAC00002FB001025902599DDF8FC06405C4FF034
:10CAD0007F4101EA00622598401CDDF8FC16085CE5
:10CAE0004FF47F0101EA004010432599891CDDF8CD
:10CAF000FC26515C4FF47F4202EA0121084325994C
:10CB0000C91CDDF8FC26515C01431E98401E27AA73
:10CB100042F8201002E00B20CDF8F8061CE41E9825
:10CB2000022803DA1420CDF8F80656E0A9992491DA
:10CB30002499AF98405C00F01800082803D00B201F
:10CB4000CDF8F80649E02499B19850F821002390D7
:10CB50001E98401E27A91E9051F820001A901E987A
:10CB6000401E51F8200019902098002804DD1A98E2
:10CB7000401C1999401A1A901A9810B11A98202836
:10CB800003D90B20CDF8F80627E00020259014905B
:10CB900019E0199914980144239800EBD10000780A
:10CBA000199A1499114401F007020121914008409B
:10CBB00030B10121149801FA00F02599084325901D
:10CBC0001498401C14901A9914988842E1D31E9826
:10CBD000401E27AA259942F8201017E21E98012826
:10CBE00003DA1420CDF8F8066EE0A99924911E9876
:10CBF000401E27A91E9051F8200025902499B09836
:10CC000050F82110259881425EDADDE92420B099A0
:10CC100041F822002499AF98405C00F0100018B150
:10CC200025988000259003E02598C01DC010259010
:10CC30002499AF98405C00F0800080B12499B198AD
:10CC400050F8210058B12499B19850F821000A9069
:10CC500003F06AFB00222499B19840F8212025981E
:10CC6000FDF76AFD249AB19941F822002499B19800
:10CC700050F8210018B90120CDF8F80624E02499D5
:10CC8000AF98405C40F08002AF9842542499B0982D
:10CC900050F82100C01DC1170A9000EB5170C01060
:10CCA0001A902499B19850F82100239000201990EF
:10CCB00006E000221999239842541998401C1990B3
:10CCC000DDE919018842F4D3EEE301201B90EBE388
:10CCD0001E98032803DA1420CDF8F8069CE020986B
:10CCE00010B901201B90DFE3A999DDF8E8060144A3
:10CCF000DDF8FC0608440B901E98401E27A91E90E4
:10CD000051F8200024901E98401E1E9051F82000DB
:10CD100016901E98401E1E9051F820001590DDE9D7
:10CD20001510884203DD0B20CDF8F806BCE31598FA
:10CD3000401C1699401A17902499B19850F8210078
:10CD4000239000202290169800F0070088B31798CF
:10CD5000C01DC1170A9000EB5170C0100990FDF77B
:10CD6000EBFC2290229818B90120CDF8F8069BE33D
:10CD700016980A900020149032E00A99239800EB4C
:10CD8000E100007801F0070201219140084088B1DC
:10CD90001499229800EBD100007801F007020121DC
:10CDA00091400843C2B22299149801EBD00002705E
:10CDB00010E01CE01499229800EBD100017814983F
:10CDC00000F00702012090408143149A229800EB62
:10CDD000D20001700A98401C0A901498401C1490CC
:10CDE000179914988842C8D32298239006E0169881
:10CDF00020B11699239800EBE1002390179A23990C
:10CE00000B98F6F7D5FF169800F0070020B122988E
:10CE100010B1229803F088FA46E31E98032803DA3B
:10CE20001420CDF8F80641E11E98401E27A91E9057
:10CE300051F820000A901E98401E1E9051F82000C4
:10CE400009901E98401E1E9051F820000890002066
:10CE5000049003900C902098002845DD1E98401EF9
:10CE60001E9051F820000790DDE90910884208DD86
:10CE7000012004900C900A98401C0999401A0690D1
:10CE800006E00998401C0A99401A06900A980990F1
:10CE9000DDE9071088420FDD012003900C9808B9E6
:10CEA000012000E000200C900898401C0799401ACF
:10CEB00005900798089004E00798401C0899401ACC
:10CEC0000590DDE90510884201DA069800E0059832
:10CED0000A90049808B9039830B1DDE9051088423A
:10CEE00002D00B20CDF8F8060A991A9109991991E8
:10CEF00008991891AA9924912098002872DD249904
:10CF0000AF98405C00F09C000C286BD12499B0983D
:10CF100050F82100C01DC01025902499B19850F8F8
:10CF2000210022902598FDF707FC2390DDE92302DC
:10CF3000B19941F822002499B19850F8210018B90C
:10CF40000120CDF8F806AFE20020169006E000229E
:10CF50001699239842541698401C169025991698B5
:10CF60008842F4DB0020169020E016981590229954
:10CF7000159801EBE0000178159800F007020120F8
:10CF80009040014079B11699239800EBE1000078B8
:10CF900001F00702012191400843C2B2169923987B
:10CFA00000EBE10002701698401C16902499B0988E
:10CFB00050F8211016988142D7DC2499AF98405C34
:10CFC00040F08002AF9842542499AF98405C20F022
:10CFD0000402AF9842542499AF98405C40F001029B
:10CFE000AF984254AA99B19850F821002390A9997A
:10CFF000B19850F821002290AA99AF98405C00F0B7
:10D000001C00082803D00B20CDF8F8064CE21A9833
:10D0100018B90B20CDF8F80647E00C9820B11A9803
:10D02000401E1899084418900020149039E019996E
:10D03000229800EBD100007801F007020121914015
:10D04000084080B11899239800EBD100007801F0D6
:10D050000702012191400843C2B21899239800EBBE
:10D06000D10002700EE01899239800EBD1000078EF
:10D0700001F00702012191408843189A239901EB9E
:10D08000D20108701998401C19900C9818B1189882
:10D09000401E189002E01898401C18901498401CEC
:10D0A00014901A9914988842C1D300BFFCE1012062
:10D0B0001B90F9E100BF1E98032803DA1420CDF875
:10D0C000F806E7E00020089007901E98401E27A968
:10D0D0001E9051F8200006901E98401E1E9051F898
:10D0E000200005902098002817DD1E98401E1E90F5
:10D0F00051F820000A901E98401E1E9051F8200002
:10D1000009900598401C0699401A08900998411CFE
:10D110000A98081A07900A9805901E98401E27A999
:10D120001E9051F820001790AA9924912098002869
:10D1300072DD2499AF98405C00F09C000C286BD104
:10D140002499B09850F82100C01DC0102590249952
:10D15000B19850F8210022902598FDF7EDFA239020
:10D16000DDE92302B19941F822002499B19850F8E1
:10D17000210018B90120CDF8F80695E1002016909D
:10D1800006E000221699239842541698401C1690E7
:10D19000259916988842F4DB0020169020E0169816
:10D1A00015902299159801EBE0000178159800F090
:10D1B000070201209040014079B11699239800EBB5
:10D1C000E100007801F00702012191400843C2B25A
:10D1D0002399169801EBE00002701698401C1690F7
:10D1E0002499B09850F8211016988142D7DC2499E0
:10D1F000AF98405C40F08002AF9842542499AF98B9
:10D20000405C20F00402AF9842542499AF98405CEF
:10D2100040F00102AF984254A999B19850F821000A
:10D220002390AA99B19850F82100229020980028C4
:10D230000ADD08991798884203DC079917988842F5
:10D2400002DD0B20CDF8F806AA99AF98405C00F0FB
:10D250001C00082802D00B20CDF8F806DDF8F806EF
:10D26000B8B9A89882280AD106980090DDE9223141
:10D27000059A179800F076F9CDF8F80609E00698B7
:10D280000090DDE92231059A1798F6F77DFDCDF87B
:10D29000F80600BF08E11E98022803DA1420CDF832
:10D2A000F8063DE01E98401E27A91E9051F8200068
:10D2B0002590259840B1A99840B201460A9025983A
:10D2C000F6F77BFDCDF8F8061E98401E27A91E90A4
:10D2D00051F820002590DDF8F80650B9259840B1A6
:10D2E000A99840B201460A90259801F013FECDF8A6
:10D2F000F806DDF8F80650B9A999AA98884206D030
:10D30000AA9840B20A9001F091FCCDF8F806209856
:10D31000002805DD1E98401E1E901E98401E1E907F
:10D32000C2E001201B90BFE01E98042803DA1420FD
:10D33000CDF8F806B1E0A999B19850F8210008900D
:10D34000AA99B19850F821000790AB99B19850F87C
:10D35000210006901E98401E27A91E9051F820001B
:10D3600005901E98401E1E9051F8200004901E98B3
:10D37000401E1E9051F8200003901E98401E1E90E3
:10D3800051F8200017902098002831DD1E98401E8B
:10D390001E9051F8200002901E98401E1E9051F8D9
:10D3A000200001900498401C0599401A0A90179893
:10D3B000401C0399411A0991DDE90910884201DAFC
:10D3C0000A9800E009980A900198401C0299401AB6
:10D3D0000990DDE90910884201DA0A9900E009990B
:10D3E0000A9103990491029903910A98179000BF3A
:10D3F000012025901798012803DA0B20CDF8F806B4
:10D4000043E017981A90002014903AE00399069888
:10D4100000EBD100007801F00702012191400840A3
:10D4200018B30599089800EBD100007801F00702C5
:10D4300001219140084008B1012000E000200A903D
:10D440000499079800EBD100007801F00702012150
:10D450009140084008B1012000E000200990DDE97A
:10D460000910884201D0002025900598401C0590A5
:10D470000498401C04900398401C03901498401C8E
:10D4800014901A9914988842C0D31E98421C25996A
:10D490001E9227AA42F8201000BF05E001201B9031
:10D4A00002E001201B9000BF00BF1B9810B11520A7
:10D4B000CDF8F8061E98002802DB1E98802802DBB3
:10D4C0001420CDF8F806DDF8F80640B101201C90D4
:10D4D000DDF8DC16AC98411ADDF81C0701601C98D9
:10D4E00000283DF4ABAFDDF8180701F01DFEAF9842
:10D4F000F0B1B198E0B10020149014E01499AF9805
:10D50000405C00F0800058B11499B19850F82100A7
:10D5100030B11499B19850F821000A9002F004FF3C
:10D520001498401C1490DDF8CC1614988842E5D36A
:10D53000B19810B1B19802F0F7FEB09810B1B09860
:10D5400002F0F2FEAF9810B1AF9802F0EDFEAE9887
:10D5500010B1AE9802F0E8FEDDF8F8060DF20C7D91
:10D5600000BD00002DE9F04F85B005460F469046FE
:10D5700099460020049082464D48006828444D4951
:10D580000968461800244FF0FF3B4B4890F9000013
:10D59000401C112827D2DFE800F0090A0B101112F5
:10D5A000131415161B1C1D1E1F20210000BF00BFD9
:10D5B000002004904FF0010B17E000BF00BF00BF38
:10D5C00000BF00BF00BF012004904FF0060B0CE02D
:10D5D00000BF00BF00BF00BF00BF00BF022004901B
:10D5E0004FF00D0B01E00A2400BF00BF44B93248E0
:10D5F00090F90000584503D0584601F017FB044647
:10D6000004BB2E48006820B1B6F5006F1AD901247A
:10D6100018E02B480068864214D9F01D4FEAD00A62
:10D620002848006802F080FE5046FDF785F825493D
:10D6300008600846006808B9012403E04FEACA0000
:10D640001F490860D4B91B4800681F4909683B4658
:10D65000CDE90085CDE90210154802681B48016834
:10D660001848006801F070FC1648036831460268EB
:10D670000498F6F7A7FB06200F4908704CB9144828
:10D680000078062805D0124890F9000001F0CEFA83
:10D69000044644B9064800950368494609480E9A6D
:10D6A000006801F002FD204605B0BDE8F08F0000E3
:10D6B000C0000810C4000810BC000810B400081016
:10D6C000D0000810E8000810DC000810D80008108E
:10D6D000BD0008100146612904DB7A2902DCA1F1B2
:10D6E000200000E00846C0B270470A46106070474C
:10D6F00010B504462146024804F0A0FC10BD00000D
:10D70000C0020020F0B587B007460D463C463AE01F
:10D7100014B1012C34D10BE002A809F0CEFD02A90E
:10D720000A20F6F754FB10B91CA0F5F78FF828E093
:10D730000020069006A91120F6F749FB10B922A097
:10D74000F5F784F800BF2B4890ED000AD0ED010AF0
:10D750008DED040ACDED050A274A07CA01AB07C3C0
:10D7600000260AE001A951F8260004A9F6F72FFBCC
:10D7700010B922A0F5F76AF8761C032EF2D300BF89
:10D7800000BF00BF641CAC42C2D303E000BF00BFB7
:10D7900000BF641EAC42F9D807B0F0BD4572726F8D
:10D7A000722077726974696E67206C61736572208C
:10D7B00064656C61797320696E207570646174654D
:10D7C000454550524F4D00004572726F722077727E
:10D7D0006974696E67206175746F44656C65746502
:10D7E00020696E20757064617465454550524F4DD7
:10D7F000000000007C0000208826031A4572726F2A
:10D80000722077726974696E6720757365725363ED
:10D81000616C6520696E2075706461746545455260
:10D82000504F4D002DE9F04F85B004460E46174687
:10D830009C46002004904FF6FF7100238246009022
:10D840000025342E3DDD20784FF07F4B0BEA006041
:10D8500094F801B04FF47F0E0EEA0B4B40EA0B0038
:10D8600094F802B04FF47F4E0EEA0B2B40EA0B0007
:10D8700094F803B040EA0B0A0AF001000090009807
:10D88000C50005F12000205C4FF07F4B0BEA006BD8
:10D8900005F12100205C4FF47F0E0EEA00404BEAB8
:10D8A000000005F1220B14F80BB04FF47F4E0EEA86
:10D8B0000B2B40EA0B0005F1230B14F80BB040EAE8
:10D8C0000B032548824504D0401C824501D002202C
:10D8D0000490B34201D3022004900498002837D169
:10D8E000E05C4FF47F4B0BEA002003F1010B14F8CE
:10D8F0000BB040EA0B080FB1A7F80080002219E036
:10D90000A05C01900020039010E00198484000F0D6
:10D91000010002904910029810B148F208404140BD
:10D920000198401001900398401C03900398082828
:10D93000EBDB521C9A42E3D3C8431FFA80F9BCF1D7
:10D94000000F01D0ACF80090C84501D00920049028
:10D95000049805B0BDE8F08F004D414A2DE9FF5F06
:10D9600006460F4690464FF0000BD94648480068DF
:10D97000304448490968451800244FF0FF3A4648AA
:10D9800090F90000401C112827D2DFE800F0090AB6
:10D990000B101112131415161B1C1D1E1F20210025
:10D9A00000BF00BF4FF0000B4FF0010A17E000BFAF
:10D9B00000BF00BF00BF00BF00BF4FF0010B4FF022
:10D9C000060A0CE000BF00BF00BF00BF00BF00BFE1
:10D9D0004FF0020B4FF00D0A01E00A2400BF00BF18
:10D9E00044B92D4890F90000504503D0504601F04D
:10D9F0001DF9044604BB2948006820B1B5F5007F35
:10DA00001AD9012418E026480068854214D9E81D77
:10DA10004FEAD0092348006802F086FC4846FCF72C
:10DA20008BFE204908600846006808B9012403E01D
:10DA30004FEAC9001A490860D4B9164800681A4963
:10DA400009683B46CDE90086CDE90210104802681E
:10DA5000164801681348006801F076FA002311485F
:10DA6000294602685846F6F7B7F90D200A490870AA
:10DA70004CB90F4800780D2805D00D4890F90000EA
:10DA800001F0D4F80446204604B0BDE8F09F000041
:10DA9000C8000810CC000810BC000810B400081022
:10DAA000D4000810EC000810E4000810E000081092
:10DAB000BE000810014608784A7840EA02208A78B9
:10DAC00040EA0240CA7840EA026070472DE9F04F10
:10DAD00095B00020149080460024139012900027E7
:10DAE0001190109000266BA5814682464FF0010BE5
:10DAF0006A4908600690F6F774F969486949086050
:10DB000069486A490860002F6FD112AB13AA6548B3
:10DB1000016866480068FFF785FE8046B8F1000F8F
:10DB200003D0012015B0BDE8F08F10A811A914AAE8
:10DB3000CDE902B2CDE9041006A84B463246CDE944
:10DB400000505848016859480068FCF703FE044635
:10DB5000002C77D11098022848D11198122840D271
:10DB6000DFE800F0090C0F1215181B1E2124272ACC
:10DB70002D303336393C0FF2381A35E00FF2381AAF
:10DB800032E00FF24C1A2FE00FF25C1A2CE00FF289
:10DB9000741A29E00FF2841A26E00FF2981A23E093
:10DBA0000FF2A41A20E00FF2C41A1DE00FF2CC1AF3
:10DBB0001AE00FF2DC1A17E00FF2F01A14E00FF27D
:10DBC000042A11E00FF20C2A0EE00FF2282A0BE0D3
:10DBD0000FF2402A08E00FF25C2A05E00FF2682AF3
:10DBE00002E00FF2842A00BF25E04AE011980828DD
:10DBF0001DD2DFE800F004070A0D101316190FF20A
:10DC0000B00A17E00FF2742A14E00FF2281A11E09C
:10DC10000FF2341A0EE00FF2781A0BE00FF25C1AD2
:10DC200008E00FF2881A05E00FF2702A02E00FF206
:10DC3000382A00BF00BF52469FA01199F6F7D6F8C8
:10DC40001FE0FFE7109802280DD1182C0BD10DB161
:10DC5000287818B99E48F6F7C9F812E029469D4879
:10DC6000F6F7C4F80DE01A2C07DA9B4850F8242088
:10DC70009AA01499F6F7BAF803E02146A3A0F6F7A4
:10DC8000B5F800F091FF16B1304602F04DFB384672
:10DC900048E7000050524F4752414D009401001098
:10DCA000F33903007001001084AF011B68010010FC
:10DCB0005375636365737300436865636B696E676F
:10DCC00020636861696E206661696C757265000029
:10DCD00052656164696E67204944434F444520663C
:10DCE00061696C757265000052656164696E6720D8
:10DCF00055534552434F4445206661696C757265C2
:10DD00000000000052656164696E67205545534309
:10DD10004F4445206661696C75726500456E746597
:10DD200072696E6720495350206661696C7572652F
:10DD300000000000556E7265636F676E697A6564F6
:10DD40002064657669636500446576696365207261
:10DD500065766973696F6E206973206E6F742073C6
:10DD60007570706F727465640000000045726173B5
:10DD700065206661696C75726500000044657669AE
:10DD80006365206973206E6F7420626C616E6B0036
:10DD90004465766963652070726F6772616D6D6945
:10DDA0006E67206661696C7572650000446576690E
:10DDB000636520766572696679206661696C757243
:10DDC0006500000052656164206661696C7572656A
:10DDD0000000000043616C63756C6174696E6720BC
:10DDE000636865636B73756D206661696C757265D8
:10DDF0000000000053657474696E67207365637575
:10DE00007269747920626974206661696C757265E3
:10DE1000000000005175657279696E672073656353
:10DE2000757269747920626974206661696C7572B3
:10DE30006500000045786974696E67204953502079
:10DE40006661696C75726500506572666F726D69A6
:10DE50006E672073797374656D20746573742066C2
:10DE600061696C7572650000556E6B6E6F776E2020
:10DE70006578697420636F6465000000496C6C65A7
:10DE800067616C20696E697469616C697A61746933
:10DE90006F6E2076616C7565730000005352414DC2
:10DEA00020636F6E66696775726174696F6E206654
:10DEB00061696C75726500004578697420636F64F0
:10DEC00065203D2025642E2E2E2025730A0000009B
:10DED000C0FF041B0400051B980100104572726FFF
:10DEE00072206174206164647265737320256C64B0
:10DEF0003A2025732E0A50726F6772616D20746527
:10DF0000726D696E617465642E0A0000556E6B6EE9
:10DF10006F776E206572726F7220636F6465202563
:10DF20006C640A0070B504460D4624B1012C09D07A
:10DF3000022C15D10DE00B4A517810782A46F8F7DB
:10DF40001FFB0DE0084A517810782A46F8F718FBB5
:10DF500006E0064A517810782A46F8F711FB00BF10
:10DF600000BF70BDEC86041AFC86041A0C87041AE4
:10DF700010B500BF00F044F80446601C08B120460C
:10DF800010BD0020F5F737FF18B10020FAF70EFD9D
:10DF90000446601C0028EDD02046F1E770B5054628
:10DFA00000201049087000264FF0004415E03EB9EB
:10DFB00005EA0400A04201D1012000E0002006464D
:10DFC00056B105EA0400A04201D107A000E007A075
:10DFD00001460448F3F749F96408002CE7D10148E9
:10DFE00070BD0000F0BA00203100000030000000D9
:10DFF00001700A0A42700A0C82700A0EC2707047E1
:10E000004FF0FF3005490968054A914204D00349A1
:10E0100008681146014A1160704700005C00081052
:10E02000A55AA55AF0B5034600200022002431E08D
:10E030001A4D2D685C5D1A4D2D68C5F1080524FA4E
:10E0400005F5174E3668C6F10807FF263E413540F4
:10E0500095402843124D2D68A9420DD88D18C5F161
:10E0600010064FF6FF75354128400D4D2D686D1A8D
:10E070000B4E356000210DE0084D2D686D1C074EDC
:10E080003560074D2D682A44054D2D68491B08252C
:10E09000034E35600029CBD1F0BD0000AC00081064
:10E0A000B000081070B504460D462E4604B970BD88
:10E0B0000020206161680870616848706068A06035
:10E0C0000120E0610020E062706920B1F1687069B0
:10E0D00050F8210000E00020A04202D12846F5F7C8
:10E0E0008FFE00BFE3E7000010B5034A51781078B7
:10E0F0000022F8F745FA10BDDC86041A10B501209D
:10E10000F8F750FA00243CE0784B03EB04139A68CC
:10E11000764B03EB04135979744B03EB0413187912
:10E12000F5F7A7FC714800EB04100078FF2813D026
:10E130006E4800EB04104078FF280DD06B4B03EBCA
:10E1400004131A7B694B03EB04135978674B03EBF9
:10E1500004131878F8F748FA644800EB0410007BC1
:10E1600001280DD1614B03EB04135A7B5F4B03EB8A
:10E17000041359785D4B03EB04131878F8F700FA91
:10E18000641C432CC0D3F220594908605849803997
:10E19000C1F88400564908310860F320091D086061
:10E1A000091D0860091D0860091D0860091D086037
:10E1B000091D0860091D0860091D0860091D086027
:10E1C000091D0860091D0860091D0860F220484902
:10E1D00080310860091D0860091D086044499831B4
:10E1E0000860F320091D0860091D0860091D08600A
:10E1F000091D0860091D0860091D0860091D0860E7
:10E20000F2203C490860091D0860091D0860091DCD
:10E210000860091D0860091D0860091D0860091DC6
:10E220000860F120334984310860091D0860F3203B
:10E23000091D0860091D0860091D0860F120091DFD
:10E240000860091D0860091D0860F320091D0860A9
:10E25000091D0860091D0860091D0860264908603D
:10E26000F22026490860091D0860091D0860091D83
:10E270000860091D0860091D0860091D0860091D66
:10E280000860091D0860091D0860091D0860091D56
:10E290000860091D0860091D0860091D0860091D46
:10E2A0000860091D0860F320144980310860091DC9
:10E2B0000860091D0860091D0860091D0860091D26
:10E2C0000860091D0860091D0860091D0860091D16
:10E2D0000860091D0860091D0860091D0860091D06
:10E2E0000860091D0860091D086010BD8408001041
:10E2F00080600840806208401065084080660840E1
:10E3000070B5B0B0054602202E90F5F77EFD2E992F
:10E3100088420DD0F5F779FD04462E99FFF7F2F902
:10E320002EA91020F5F753FD10B9E6A0F4F78EFAE8
:10E3300000202D902DA90CF0E5FA10B9ECA0F4F70F
:10E3400085FA2DA9F448F5F765FD00202C902CA93D
:10E3500005200CF0D7FA10B9F0A0F4F777FA2C9951
:10E3600088B2F9490968488700BFF84A07CA29AB4B
:10E3700007C30020099036E0099905A803F0F8FDCD
:10E3800029A9099A51F8220005A90CF0BBFA58B93D
:10E39000EFA00999F5F72AFD01A8099903F0E8FD16
:10E3A00001A80FC805AC0FC49DF8140098B901A8C6
:10E3B000099903F0DDFD01A80FC805AC0FC429A918
:10E3C000099A51F8220005A9F5F701FD18B9EBA04B
:10E3D0000999F5F70BFD09AA05A9CF48F5F71FFD27
:10E3E0000998401C099009980328C5D3002028905B
:10E3F00028A901200CF086FA10B9EBA0F4F726FA50
:10E4000000202FAA28A92F90C34803F0A2FDCF4ACD
:10E410000C3207CA25AB07C300242CE008A8F5F787
:10E4200003FD25A951F8240008A90CF06BFA58B98E
:10E430002146E9A0F5F7DAFC06A8F5F7F5FCDDE9D9
:10E440000601CDE9080110E0BDF82000002803DD39
:10E45000BDF82200002808DC06A8F5F7E5FCDDE998
:10E460000601CDE9080100202870224608A9E548E8
:10E47000F5F7DFFC641C032CD0D3B44A183207CA6A
:10E4800022AB07C3002463E000BFDF4890ED000A21
:10E49000D0ED010A8DED080ACDED090A22A951F847
:10E4A000240008A90CF02EFA18B9D8A0F4F7CEF978
:10E4B00048E0002108A8F5F7C1FC90ED000ADFED67
:10E4C000DD0AB4EEE00AF1EE10FA26DC002108A81D
:10E4D000F5F7B4FC90ED000ADFEDD70AB4EEE00AE0
:10E4E000F1EE10FA19D3012108A8F5F7A7FC90ED79
:10E4F000000ADFEDD00AB4EEE00AF1EE10FA0CDC0F
:10E50000012108A8F5F79AFC90ED000ADFEDCA0A90
:10E51000B4EEE00AF1EE10FA14D200BFBA4890ED62
:10E52000000AD0ED010A8DED080ACDED090A22A9F5
:10E5300051F8240008A9F5F74AFC18B92146BFA0F4
:10E54000F5F754FC224608A9AE48F5F77CFC641C9C
:10E55000032C99D3DFEDC52A9FEDC52ADFEDC51A3F
:10E560009FEDC51ADFEDC50A9FEDC00A18A81EF081
:10E57000E7FA18A8F5F76CFC8DED140ACDED150A35
:10E580008DED161ACDED171A14A906200CF0BAF964
:10E5900010B9BBA0F4F75AF900BF9DED140AB5EE0F
:10E5A000C00AF1EE10FA01DD012100E00021084669
:10E5B0009DED150AB5EEC00AF1EE10FA01DD01215C
:10E5C00000E0002108409DED160AB5EEC00AF1EE0C
:10E5D00010FA01DD012100E0002108409DED170A3D
:10E5E000B5EEC00AF1EE10FA01D2012100E00021DF
:10E5F000084000BF90B918A8F5F72AFC8DED140A61
:10E60000CDED150A8DED161ACDED171A14A90620B9
:10E61000F5F7DDFB10B9A6A0F4F718F9794E06F16D
:10E6200078049DED140A84ED010A9DED150A84ED30
:10E63000020A9DED170A84ED040A9DED160A84ED89
:10E64000030A2046F5F709FC00BF00BF0020139025
:10E6500013A908200CF056F910B9A1A0F4F7F6F8A8
:10E6600013A92D4805F0FFF90EA90A200CF04AF96C
:10E6700028B9A4A0F4F7EAF80EA808F01EFE00BF1F
:10E680000120BDF93C10BDF93A20914201DD012184
:10E6900000E000210840BDF84010BDF93A201144C7
:10E6A000BDF93C20914201DD012100E0002108403C
:10E6B000BDF84210BDF93A205242914201DD0121DC
:10E6C00037E135E14572726F722077726974696E55
:10E6D000672076657273696F6E20696E207265734C
:10E6E000746F726546726F6D454552504F4D000014
:10E6F0004661696C656420746F2072656164207482
:10E7000061626C65207A65726F2066726F6D20455C
:10E710004550524F4D0A0000C00200204661696C0E
:10E72000656420746F207265616420737465707015
:10E7300065722073656E73652066726F6D20454546
:10E7400050524F4D00000000940000109426031A10
:10E750004661696C656420746F207265616420662F
:10E7600069656C642073697A652025642066726F20
:10E770006D20454550524F4D0A0000004572726FA2
:10E78000722077726974696E6720636F6E6669675D
:10E7900075726174696F6E20666F72206669656C50
:10E7A000642025640A0000004661696C6564207479
:10E7B0006F20726561642063757272656E74206685
:10E7C00069656C642073697A652066726F6D204597
:10E7D0004550524F4D0000004661696C65642074DD
:10E7E0006F207265616420616C69676E6D656E741F
:10E7F0002025642066726F6D20454550524F4D0AAA
:10E800000000000040B300207C0000204661696CDD
:10E81000656420746F207265616420757365722071
:10E820007363616C652066726F6D20454550524F71
:10E830004D0A00009A99993FCDCC4C3F4572726FBA
:10E84000722077726974696E6720696E76616C698F
:10E85000642075736572207363616C657220666FE6
:10E8600072206669656C642025640A00000000005F
:10E870004A2729C2789CF34252B8AF4200001442A2
:10E880004661696C656420746F207265616420471D
:10E89000616C766F20706172616D65746572732052
:10E8A00066726F6D20454550524F4D0A00000000C2
:10E8B0004572726F722077726974696E6720676142
:10E8C0006C766F20706172616D7320696E20726565
:10E8D00073746F726546726F6D454550524F4D00AF
:10E8E0004661696C656420746F20726561642055AF
:10E8F0004E4954532066726F6D20454550524F4D1E
:10E900000A0000004661696C656420746F207265BE
:10E910006164206C617365722064656C6179732039
:10E9200066726F6D20454550524F4D0A0000000041
:10E930000021084000BF50B90EA808F0BEFC0EA987
:10E940000A20F5F744FA10B926A0F3F77FFF0EA9C5
:10E95000304808F0CFFE0DA90D200BF0D3FF20B9F1
:10E960002DA0F3F773FF04200D900D9848B90420F3
:10E970000D900DA90D20F5F72AFA10B930A0F3F784
:10E9800065FF0D98C1B23A48F5F76CFA00200C907B
:10E990000CA90E200BF0B6FF20B936A0F3F756FFF6
:10E9A00000200C900CA9324803F036F800200B90A0
:10E9B0000BA90F200BF0A6FF10B939A0F3F746FF03
:10E9C00000200A900AA911200BF09CFF10B93EA06C
:10E9D000F3F73CFF9DF828102548F5F748FA30B0CA
:10E9E00070BD00004572726F722077726974696E33
:10E9F00067206C617365722064656C61797320694E
:10EA00006E20726573746F726546726F6D45455006
:10EA1000524F4D0004AF00204661696C656420745C
:10EA20006F2072656164204C415345525F4D4F44E5
:10EA3000454C2066726F6D20454550524F4D0A007F
:10EA40004572726F722077726974696E67206C61AB
:10EA5000736572206D6F64656C20696E20726573DA
:10EA6000746F726546726F6D454550524F4D000090
:10EA7000C00200204661696C656420746F20726575
:10EA800061642053455249414C5F4E554D424552B9
:10EA90002066726F6D20454550524F4D0A000000B0
:10EAA0004661696C656420746F20726561642050F2
:10EAB000617373636F64652066726F6D20454550A6
:10EAC000524F4D0A000000004661696C6564207475
:10EAD0006F2072656164204175746F44656C657464
:10EAE000652066726F6D20454550524F4D0A0000FB
:10EAF00070B504460D460648006838B12A462146DE
:10EB000004A0F5F773F90C48F5F7B6F970BD0000ED
:10EB1000940100104578706F72743A206B6579200B
:10EB20003D20222573222C2076616C7565203D20C6
:10EB3000256C640A0000000038EF002070B505461F
:10EB40002C46606920B1E168606950F8210000E05E
:10EB5000002000B970BD616921B1E268616951F8B6
:10EB6000221000E0002108462946F5F78AF9002026
:10EB7000E268616941F82200E06810B1E068401E77
:10EB8000E060606920B1E168606950F8210000E050
:10EB9000002020B12846F5F733F90120206300BF9B
:10EBA000D8E700BF00BF704710B501220021042044
:10EBB000F7F7E6FC00221A210520F7F7E1FC10BD6B
:10EBC00008B504469FED130A1348F5F75FF913489B
:10EBD00090ED000A104808F09BFD114890ED000AE6
:10EBE0000D4808F098FD9FED0F0A0B48F5F753F913
:10EBF0000D4890ED000A0848F5F752F928206946BB
:10EC000000900548F5F751F900BF21460248F5F795
:10EC100051F9FAE7BD37863504AF00200C00081023
:10EC2000100008106F12833A140008102DE9F0410B
:10EC30000446002600272D4890F90000401C08B922
:10EC400000F05AF8294890F90000A04216D1012C92
:10EC500007D0042C05D0062C03D00B2C01D00D2C92
:10EC600005D1002211461046F5F729F935E0A4BB7D
:10EC7000002211460120F5F722F92EE026E01C487B
:10EC80001A4991F9001030F811000121A140084003
:10EC900008B1012000E00020054600221146284668
:10ECA000F5F70DF945B11348104991F9001010F826
:10ECB00011000E49087008E00E480C4991F9001047
:10ECC00000EB4100407809490870761C074890F92C
:10ECD0000000A04201D0092ED1DB044890F90000C9
:10ECE000A04200D00A273846BDE8F081BC000810D9
:10ECF00010010810F000081010B5002405E00022F3
:10ED000011460120F5F7DBF8641C052CF7DB002227
:10ED100011461046F5F7D3F801200149087010BDDF
:10ED2000BC0008102DE9F0470546884616464FF00E
:10ED300000093548006840B1B5F5806F02D94FF041
:10ED400001091BE03148056018E030480068854241
:10ED500012D92F48006801F0E7FAE91DC808FBF74F
:10ED6000EBFC2B4908600846006810B94FF0010918
:10ED700004E02648056001E024480560B9F1000F71
:10ED80003FD100243BE004EB08077EB9204800682F
:10ED900000EBD400007804F0070201219140084301
:10EDA0001B49096801EBD401087027E006EBD70086
:10EDB000007807F0070201219140084078B114481B
:10EDC000006800EBD400007804F0070201219140B4
:10EDD00008430F49096801EBD40108700EE00C48A4
:10EDE000006800EBD400007804F007020121914094
:10EDF00088430749096801EBD4010870641CAC42E0
:10EE0000C1D34846BDE8F087B4000810C000081020
:10EE1000D80008102DE9F0470546884616464FF001
:10EE200000093548006840B1B5F5806F02D94FF050
:10EE300001091BE03148056018E030480068854250
:10EE400012D92F48006801F06FFAE91DC808FBF7D6
:10EE500073FC2B4908600846006810B94FF001099F
:10EE600004E02648056001E024480560B9F1000F80
:10EE70003FD100243BE004EB08077EB9204800683E
:10EE800000EBD400007804F0070201219140084310
:10EE90001B49096801EBD401087027E006EBD70095
:10EEA000007807F0070201219140084078B114482A
:10EEB000006800EBD400007804F0070201219140C3
:10EEC00008430F49096801EBD40108700EE00C48B3
:10EED000006800EBD400007804F0070201219140A3
:10EEE00088430749096801EBD4010870641CAC42EF
:10EEF000C1D34846BDE8F087B4000810C40008102C
:10EF0000DC00081001460248017000207047000034
:10EF1000BE00081070B506460C460025094890F959
:10EF20000000401C40B1074890F90000A04203D007
:10EF30002046FFF77BFE054615B93046F4F7C4FFBF
:10EF4000284670BDBC0008102DE9F04F04460E465F
:10EF50009946DDE90BC8DDE90975002030E006EBD4
:10EF6000D00A9AF800A000F0070E4FF0010B0BFA40
:10EF70000EFB0AEA0B0ABAF1000F10D004EBD00A1C
:10EF80009AF800A000F0070E4FF0010B0BFA0EFBF1
:10EF90004AEA0B0A04EBD00B8BF800A00FE004EB5D
:10EFA000D00A9AF800A000F0070E4FF0010B0BFA00
:10EFB0000EFB2AEA0B0A04EBD00B8BF800A0401CD6
:10EFC0009042CCD33946531931E009EBD10A9AF873
:10EFD00000A001F0070E4FF0010B0BFA0EFB0AEA3E
:10EFE0000B0ABAF1000F10D004EBD00A9AF800A077
:10EFF00000F0070E4FF0010B0BFA0EFB4AEA0B0A6A
:10F0000004EBD00B8BF800A00FE004EBD00A9AF8C9
:10F0100000A000F0070E4FF0010B0BFA0EFB2AEADE
:10F020000B0A04EBD00B8BF800A0401C491C984243
:10F03000CBD3002102EB050A0AEB080331E00CEB0D
:10F04000D10A9AF800A001F0070E4FF0010B0BFA5D
:10F050000EFB0AEA0B0ABAF1000F10D004EBD00A3B
:10F060009AF800A000F0070E4FF0010B0BFA0EFB10
:10F070004AEA0B0A04EBD00B8BF800A00FE004EB7C
:10F08000D00A9AF800A000F0070E4FF0010B0BFA1F
:10F090000EFB2AEA0B0A04EBD00B8BF800A0401CF5
:10F0A000491C9842CBD3BDE8F08F2DE9F0430446CC
:10F0B0001D46079E2B469719104631E004EBD30CF2
:10F0C0009CF800C003F007094FF0010808FA09F89E
:10F0D0000CEA080CBCF1000F10D001EBD00C9CF82E
:10F0E00000C000F007094FF0010808FA09F84CEADF
:10F0F000080C01EBD00888F800C00FE001EBD00C41
:10F100009CF800C000F007094FF0010808FA09F860
:10F110002CEA080C01EBD00888F800C0401C5B1CEE
:10F12000B842CBD3BDE8F08310B5044634B12448CF
:10F1300090F90000401C08B1FFF7DEFD214800688F
:10F1400000283BD12048006830B11F48006801F01A
:10F15000EBF800201C4908601C48006830B11B48CF
:10F16000006801F0E1F800201849086018480068BC
:10F1700030B11748006801F0D7F800201449086042
:10F180001448006830B11348006801F0CDF8002041
:10F19000104908601048006830B10F48006801F05D
:10F1A000C3F800200C4908600C48006830B10B48D7
:10F1B000006801F0B9F800200849086010BD00009F
:10F1C000BC000810B4000810D8000810DC000810BB
:10F1D000E8000810E0000810E4000810EC00081037
:10F1E00001B58CB00C9807900798806A002831D13F
:10F1F0000121079881620798C06A08B90798C1621F
:10F200000798406810B9FC490798416007988068E2
:10F2100010B9FA49079881600798406928B10798A2
:10F220004169C06851F8200000E0002078B90C98CE
:10F230000BF0DEF90798406806904FF400710C9AC5
:10F24000F4F747FE07994A69C96842F821000C980B
:10F25000F4F7D6FD01F036B80798406A0A9007988F
:10F26000017E0A9801700A9809900798C06AE449DB
:10F2700051F820000B9000BF0A980078059015E027
:10F280000699B1F902100B9800EB81000B900B98D6
:10F2900030F8020C28B107990B98086407990A986E
:10F2A00048640A98401C0A900078059005990B98CC
:10F2B00000EB81000690B0F9001005988142DFD084
:10F2C00000BF0B9830F9020C08900799099808655F
:10F2D000DDE90910411A079801620A980178079838
:10F2E000017600210A98017007990A98486200BFC8
:10F2F0000898572880F0E187DFE810F05700630096
:10F300007A009000C100F200FA00100126013C01D1
:10F310005201680184019A01B001C601DC01F201C9
:10F3200008021E0234024A02600276028C02A20225
:10F33000B802CE02E402FA02100326033C03520391
:10F3400068037E039403AA03C003D603EC030204FC
:10F3500018042E0444049104A704BD04D304E90452
:10F36000FF0415052B05410557056D058305990516
:10F37000AC05BF05D205E505F8050B061E063106EE
:10F38000440657066A067D069006A306B606C90619
:10F39000DC06EF06020715072B072C0745073D077C
:10F3A0003E073F074007410742070798017E0A983A
:10F3B00001700798406C401C0A900798006C0B90F5
:10F3C0007FE70798006D06900798006840680590F1
:10F3D0000798006840680068006804900021DDE933
:10F3E0000430069A984701210798C16200F069BF6E
:10F3F0000798006D06900798006840680590079888
:10F40000006840680068006804900221DDE904306B
:10F41000069A984701210798C162E7E70798017E9D
:10F420000A9801700998401C0A9007994862079948
:10F4300009980865DDE90910411A079801620A98E0
:10F4400001780798017600210A98017007990A98B7
:10F4500048620798006D069007980068406805901C
:10F460000798006840680068006804900121DDE9A1
:10F470000430069A984703210798C162B6E70798B7
:10F48000017E0A9801700998401C0A900799486209
:10F49000079909980865DDE90910411A0798016282
:10F4A0000A9801780798017600210A980170079957
:10F4B0000A9848620798006D0690079800684068AF
:10F4C0000590079800684068006800680490012172
:10F4D000DDE90430069A984701210798C16285E763
:10F4E000079800688068401C0799096888607DE774
:10F4F0000798006D06900798006840680590079887
:10F50000006840680068006804900121DDE904306B
:10F51000069A984707210798C16267E70798006D28
:10F520000690079800684068059007980068406852
:10F530000068006804904A21DDE90430069A984783
:10F540000B210798C16251E70798006D0690079854
:10F550000068406805900798006840680068006887
:10F5600004904C21DDE90430069A98470121079860
:10F57000C1623BE70798006D0690079800684068F5
:10F5800005900798006840680068006804904B2167
:10F59000DDE90430069A98470B210798C16225E7F8
:10F5A0000798006D069007980068406805900798D6
:10F5B000006840680068006804900321DDE90430B9
:10F5C000069A984701210798C1620FE70798006DD6
:10F5D00006900798006840680590079800684068A2
:10F5E0000068006804900421DDE90430069A984719
:10F5F00001210798C162F9E6A065001038EF0020EC
:10F60000080000100798006D069007980068406891
:10F61000059007980068406800680068049005211C
:10F62000DDE90430069A984701210798C162DDE6BA
:10F630000798006D06900798006840680590079845
:10F64000006840680068006804900621DDE9043025
:10F65000069A984709210798C162C7E60798006D86
:10F660000690079800684068059007980068406811
:10F670000068006804900721DDE90430069A984785
:10F6800001210798C162B1E60798006D06900798BE
:10F690000068406805900798006840680068006846
:10F6A00004900821DDE90430069A98470121079863
:10F6B000C1629BE60798006D069007980068406855
:10F6C0000590079800684068006800680490092168
:10F6D000DDE90430069A984701210798C16285E662
:10F6E0000798006D06900798006840680590079895
:10F6F000006840680068006804900A21DDE9043071
:10F70000069A984701210798C1626FE60798006D35
:10F710000690079800684068059007980068406860
:10F720000068006804900B21DDE90430069A9847D0
:10F7300001210798C16259E60798006D0690079865
:10F740000068406805900798006840680068006895
:10F7500004900C21DDE90430069A984701210798AE
:10F76000C16243E60798006D0690079800684068FC
:10F7700005900798006840680068006804900D21B3
:10F78000DDE90430069A984701210798C1622DE609
:10F790000798006D069007980068406805900798E4
:10F7A000006840680068006804900E21DDE90430BC
:10F7B000069A984701210798C16217E60798006DDD
:10F7C00006900798006840680590079800684068B0
:10F7D0000068006804900F21DDE90430069A98471C
:10F7E00001210798C16201E60798006D069007980D
:10F7F00000684068059007980068406800680068E5
:10F8000004901021DDE90430069A984701210798F9
:10F81000C162EBE50798006D0690079800684068A4
:10F8200005900798006840680068006804901121FE
:10F83000DDE90430069A984701210798C162D5E5B1
:10F840000798006D06900798006840680590079833
:10F85000006840680068006804901221DDE9043007
:10F86000069A984701210798C162BFE50798006D85
:10F8700006900798006840680590079800684068FF
:10F880000068006804901321DDE90430069A984767
:10F8900001210798C162A9E50798006D06900798B5
:10F8A0000068406805900798006840680068006834
:10F8B00004901421DDE90430069A98470121079845
:10F8C000C16293E50798006D06900798006840684C
:10F8D000059007980068406800680068049015214A
:10F8E000DDE90430069A984701210798C1627DE559
:10F8F0000798006D06900798006840680590079883
:10F90000006840680068006804901621DDE9043052
:10F91000069A984701210798C16267E50798006D2C
:10F92000069007980068406805900798006840684E
:10F930000068006804901721DDE90430069A9847B2
:10F9400001210798C16251E50798006D069007985C
:10F950000068406805900798006840680068006883
:10F9600004901821DDE90430069A98470121079890
:10F97000C1623BE50798006D0690079800684068F3
:10F980000590079800684068006800680490192195
:10F99000DDE90430069A984701210798C16225E500
:10F9A0000798006D069007980068406805900798D2
:10F9B000006840680068006804901A21DDE904309E
:10F9C000069A984701210798C1620FE50798006DD4
:10F9D000069007980068406805900798006840689E
:10F9E0000068006804901C21DDE90430069A9847FD
:10F9F00001210798C162F9E40798006D0690079805
:10FA000000684068059007980068406800680068D2
:10FA100004901B21DDE90430069A984701210798DC
:10FA2000C162E3E40798006D06900798006840689B
:10FA300005900798006840680068006804901D21E0
:10FA4000DDE90430069A984701210798C162CDE4A8
:10FA50000798006D06900798006840680590079821
:10FA6000006840680068006804901E21DDE90430E9
:10FA7000069A984701210798C162B7E40798006D7C
:10FA800006900798006840680590079800684068ED
:10FA90000068006804901F21DDE90430069A984749
:10FAA00001210798C162A1E40798006D06900798AC
:10FAB0000068406805900798006840680068006822
:10FAC00004902021DDE90430069A98470121079827
:10FAD000C162F6E30798006D0690079800684068D9
:10FAE000059007980068406800680068049021212C
:10FAF000DDE90430069A984701210798C162E0E3E6
:10FB00000798006D06900798006840680590079870
:10FB1000006840680068006804902221DDE9043034
:10FB2000069A984701210798C162CAE30798006DB9
:10FB3000069007980068406805900798006840683C
:10FB40000068006804902321DDE90430069A984794
:10FB500001210798C162B4E30798006D06900798E9
:10FB60000068406805900798006840680068006871
:10FB700004902421DDE90430069A98470121079872
:10FB8000C1629EE30798006D039007980068406883
:10FB9000029007980068406800680068019025217D
:10FBA000DDE90130039A98470798006D801C0390A7
:10FBB000F1F726F904900020059016E00C98F4F770
:10FBC0008DF9C0B2069007980068406803900798C6
:10FBD000006840680068006806AA32210290DDE9EA
:10FBE000023098470598401C0590DDE904108842D2
:10FBF000E4DB0798006D0390079800684068029066
:10FC00000798006840680068006801902621DDE9D7
:10FC10000130039A984701210798C16251E3079880
:10FC2000006D069007980068406805900798006886
:10FC300040680068006804902721DDE90430069AD6
:10FC4000984701210798C1623BE30798006D069031
:10FC50000798006840680590079800684068006849
:10FC6000006804902821DDE90430069A98470121B4
:10FC70000798C16225E30798006D06900798006811
:10FC80004068059007980068406800680068049024
:10FC90002921DDE90430069A984701210798C162BD
:10FCA0000FE30798006D069007980068406805907C
:10FCB0000798006840680068006804902A21DDE920
:10FCC0000430069A984701210798C162F9E2079823
:10FCD000006D0690079800684068059007980068D6
:10FCE00040680068006804902B21DDE90430069A22
:10FCF000984701210798C162E3E20798006D0690DA
:10FD00000798006840680590079800684068006898
:10FD1000006804902C21DDE90430069A98470121FF
:10FD20000798C162CDE20798006D069007980068B9
:10FD30004068059007980068406800680068049073
:10FD40002D21DDE90430069A984701210798C16208
:10FD5000B7E20798006D0690079800684068059024
:10FD60000798006840680068006804902E21DDE96B
:10FD70000430069A984701210798C162A1E20798CA
:10FD8000006D069007980068406805900798006825
:10FD900040680068006804902F21DDE90430069A6D
:10FDA000984701210798C1628BE20798006D069081
:10FDB00007980068406805900798006840680068E8
:10FDC000006804903321DDE90430069A9847012148
:10FDD0000798C16275E20798006D06900798006861
:10FDE00040680590079800684068006800680490C3
:10FDF0003421DDE90430069A984701210798C16251
:10FE00005FE20798006D06900798006840680590CB
:10FE10000798006840680068006804903021DDE9B8
:10FE20000430069A984701210798C16249E2079871
:10FE3000006D069007980068406805900798006874
:10FE400040680068006804903521DDE90430069AB6
:10FE5000984736E20798006D06900798006840685A
:10FE60000590079800684068006800680490362193
:10FE7000DDE90430069A984723E20798006D069062
:10FE80000798006840680590079800684068006817
:10FE9000006804903721DDE90430069A984710E2A3
:10FEA0000798006D069007980068406805900798CD
:10FEB000006840680068006804903821DDE904307B
:10FEC000069A9847FDE10798006D0690079800682C
:10FED00040680590079800684068006800680490D2
:10FEE0003921DDE90430069A9847EAE10798006D68
:10FEF0000690079800684068059007980068406879
:10FF00000068006804903A21DDE90430069A9847B9
:10FF1000D7E10798006D0690079800684068059043
:10FF20000798006840680068006804903B21DDE99C
:10FF30000430069A9847C4E10798006D0690079828
:10FF4000006840680590079800684068006800688D
:10FF500004903C21DDE90430069A9847B1E1079806
:10FF6000006D069007980068406805900798006843
:10FF700040680068006804903D21DDE90430069A7D
:10FF800098479EE10798006D0690079800684068C2
:10FF900005900798006840680068006804903E215A
:10FFA000DDE90430069A98478BE10798006D0690CA
:10FFB00007980068406805900798006840680068E6
:10FFC000006804903F21DDE90430069A984778E103
:10FFD0000798006D0690079800684068059007989C
:10FFE000006840680068006804904021DDE9043042
:10FFF000069A984765E10798006D06900798006893
:020000041A01DF
:1000000040680590079800684068006800680490A0
:100010004121DDE90430069A984752E10798006DC6
:100020000690079800684068059007980068406847
:100030000068006804904221DDE90430069A984780
:100040003FE10798006D06900798006840680590AA
:100050000798006840680068006804904321DDE963
:100060000430069A98472CE10798006D069007988F
:10007000006840680590079800684068006800685C
:1000800004904521DDE90430069A984719E1079864
:10009000006D069007980068406805900798006812
:1000A00040680068006804904621DDE90430069A43
:1000B000984706E10798006D069007980068406829
:1000C0000590079800684068006800680490472120
:1000D000DDE90430069A9847F3E00798006D069032
:1000E00007980068406805900798006840680068B5
:1000F000006804904821DDE90430069A9847E0E062
:100100000798006D0690079800684068059007986A
:10011000006840680068006804904921DDE9043007
:10012000069A9847CDE00798006D069007980068FA
:10013000406805900798006840680068006804906F
:100140000121DDE90430069A984701210798C16230
:10015000B7E0B6E000BF0798806806900798006A8D
:1001600005900798006D04900122DDE90513F3F76F
:10017000BAFE00BFA5E000BF00BF00BF00BF00BFC8
:1001800000200DB000BD0798016D0A98401A401E6E
:1001900006900798017E0A98017007984169C06827
:1001A00051F82000C06AA8B907984169C06851F8A1
:1001B000200001690798C161079842694168C068D9
:1001C00052F820000160012107984269C06852F886
:1001D0002000C16207984169C06851F82000416859
:1001E0000798C06901440798406A814222D3079862
:1001F000016D06980144079841620C98F3F778FE68
:100200000B90DDE90B01F3F778FE05900798006D80
:100210000990059848B10798406A401C07994862C0
:100220000A9005980B90FFF727B80798406A0A9044
:10023000FFF747B80C98F3F765FEA8B1012802D084
:10024000022838D121E00021079801630798016D49
:1002500041620798C06A401E059000EBD0704010C4
:1002600051300890FFF744B80798016D0698014493
:10027000079841620C98F3F73BFE0B900798406A91
:100280000A900798006D0990CDE707984169C0680A
:1002900051F8200041680798C069014407984162FD
:1002A0000C98F3F725FE0B900798406A0A90079880
:1002B000006D0990BCE700BF03E003A00C99F3F7C1
:1002C00026FE00BFFEF7C8BF666174616C20666CD5
:1002D0006578207363616E6E657220696E746572F5
:1002E0006E616C206572726F722D2D6E6F2061636E
:1002F00074696F6E20666F756E64000070B5054698
:100300000C4626462846F3F7D3FA70BD10B50446CE
:100310000020F3F770FD18B121460020F8F753FBD9
:100320002046F3F7F9FD10BD70B504462CB1254603
:100330002C462046F3F7BCFA00BF70BD70B50646E8
:100340000D462C46606920B1E168606950F82100D3
:1003500000E0002060B928460AF04AF92A464FF426
:1003600000716068F3F7B5FDE268616941F8220049
:10037000616921B1E268616951F8221000E0002151
:1003800008462A4631460AF0FDF82846F3F738FDBC
:1003900070BD000010B50D480068816800208847D6
:1003A0000A4800680169022088470848006802215D
:1003B000826A08469047054800680021826A032047
:1003C0009047502002490870002010BD5C000020BA
:1003D000600000202DE9FC4104460E461546E0B2BF
:1003E0008DF804001848006801231A4601A94769DE
:1003F00016480078B84700BF13490968C86A8047A3
:10040000009000F001000028F6D10F48006800239A
:100410002A46314687690D480078B84700BF0A4927
:100420000968C86A8047009000F001000028F6D1F2
:1004300005490968486A8047A84203D04FF0FF3059
:10044000BDE8FC810020FBE75C000020600000208C
:1004500070B504460D464FF0FF3104F50B700AF0FD
:1004600085F8FF22294604F11400F3F75AFD04F53C
:100470000B70F3F75BFD70BD10B50446D4F828028D
:1004800030B9074904F58A70F0F7E4FDC4F8280292
:10049000D4F8280208B1012010BD0020FCE70000BC
:1004A000F0FB041A80F824127047016170478172D2
:1004B000704701B1C160704770B50446A07A08B9B1
:1004C000207A08B9012070BDD4F8280268B1D4F8A8
:1004D0002802F3F730FD08B9012000E000200546AE
:1004E0000020C4F828022846EDE70120EBE701468A
:1004F00091F85402704701210172704741607047C2
:1005000010B504464FF0FF3104F50B700AF02EF8D9
:100510000020C4F8480204F50B70F3F707FD10BD86
:1005200070B5044620461F49216000BF04461E489E
:10053000206004F50B751D481D4828601D4B0FCB2E
:1005400005F108060FC605F10800A86110301AF081
:1005500015FB686000BFA5F50B7400206060607239
:100560002072A072E0720120E0606FF00040206114
:100570000020C4F81402C4F818024FF47E70C4F8C6
:100580001C02C4F82002002084F82402C4F82802C7
:10059000C4F84802C4F84C02C4F8500284F854026B
:1005A000204670BD98F4041B18F5041A24F8041AA8
:1005B00084F8041B1C27031A70B50446204600F07B
:1005C00005F80546F3F7BCFC70BD000010B5044605
:1005D0000548206004F50B70F3F7B7FCA0F50B7429
:1005E000204600BF044610BD18F5041A00BF70472E
:1005F0000146486808B1486870470148FCE70000B8
:1006000058BA00204160704770B504462046F3F7A1
:10061000A1FC0546F3F794FC70BDC0F83412704796
:1006200038B50446D4F8E40240B9012000906A4687
:100630001021D4F85402F3F792FC00BFD4F8E4027E
:10064000401CC4F8E402012038BD000010B5044687
:10065000F3F75FFA0D490968421A0D48008842F223
:10066000107148430B49098842F21073594300EB5B
:100670002140824200D210BDF3F74BFA03490860D3
:100680000AF0EAF8C4F8180300BFF4E768000010A5
:100690000CE4041A0EE4041A00B5024602F55C707C
:1006A000F3F762FC00BDC0F83012704738B504465D
:1006B00094F8E102012803D1002084F8E00211E05F
:1006C00094F8E10270B900220121204600F044FABA
:1006D00040B1012000906A462021D4F85402F3F77B
:1006E0003EFC00BF38BD2DE9F04105460C461646DC
:1006F0002046F3F73EFC07463246394628460EF0C0
:1007000057FBBDE8F0817FB51368032B07D201F5D5
:100710004F73146803EB041678CE8DE878009DE8DB
:10072000780080E878007FBD0146D1F8E802704784
:100730002DE9F1432DED020B2DED048B84B0044621
:10074000DFF890814FF00A09B2EE040AF0EE409A09
:100750009FED610A8DED030A002008EE100A0025C6
:1007600094EDBE0AB5EEC00AF1EE10FA34D0B7EE41
:10077000000A8DED010A94EDBE0AB5EEC00AF1EE55
:1007800010FA01DD04250AE094EDBE0AB5EEC00AB8
:10079000F1EE10FA02D26FF0030500E0002594EDAF
:1007A000BE0AF0EEC00ACDED020A02A901A8F3F7D5
:1007B000E5FB90ED000ADDED080A9FED481A60EEBA
:1007C000810A20EE200ABDEEC00AB0EE408AD4F8BD
:1007D000F402C4F8FC023AE0D4F8FC12D4F80403A2
:1007E0000844D4F8F412451A281E01DB014600E043
:1007F000414200EE101AB8EEC00AF2EE040A80EE92
:10080000201A8DED021A94F8D40318B1B7EE000A3D
:100810008DED020A03AF02A908A8F3F7AFFB064665
:1008200097ED000AD6ED000AB4EEE00AF1EE10FAF8
:1008300001D2304600E0384690ED000ADFED270A8D
:1008400020EE200ABDEEC00AB0EE408A00BF15F1CE
:10085000040F0FDC0120F3F796FBD4F8540290F854
:100860007810E9B909F0D6FF0A2819D2002008EE5D
:10087000100A15E0042D10DB0020F3F784FBD4F8F8
:10088000540290F8781059B909F0C4FF1149884210
:1008900006D9002008EE100A02E0002008EE100A37
:1008A000F8EEC88A2020F0EE680A0D4991ED000AA2
:1008B000F3F76EFBB0EE409ABCEEC90A10EE100AD8
:1008C00008490968C1F80A0000BF04B0BDEC048BF8
:1008D000BDE8FE83002B0100CDCCCC3D0000DE4204
:1008E0003CAF011B9400001070B504460D4695ED19
:1008F000000AD4EDE90AB4EE600AF1EE10FA0AD06B
:1009000095ED000A84EDE90A00220521204600F059
:1009100023F900B170BD2046F3F73FFB00BFF9E7B4
:1009200010B50446F3F73EFB10BD000010B50446B9
:10093000D4F854020EF018FA012804D0D4F8540266
:100940000EF012FAD8BBF3F7E4F81F490968421A0F
:100950001E4800881E4948431E4909881C4B5943BC
:1009600000EB114082422AD9F3F7D3F81649086008
:100970002046F3F71CFB1848D0ED000AB4EE600ADD
:10098000F1EE10FA0AD12046F3F716FB1348D0ED2A
:10099000000AB4EE600AF1EE10FA10D02046F3F728
:1009A00006FB0D4880ED000A2046F3F705FB0B48D7
:1009B00080ED000AD4F85402026891688847204606
:1009C00001F088F810BD0000500000100CE4041A7B
:1009D000A08601000EE4041A480000104C0000102C
:1009E00070B5044620460EF037F900283FD094F841
:1009F000E10250B92046F3F7E4FA05460068816B3E
:100A000028468847C4F874032BE094F8E1020A28CA
:100A10001BD1D4F854020EF0A7F9B0B994F85C02D7
:100A2000012810D12046F3F7CCFA05460068816A08
:100A30002846884730B1022084F85C02D4F830029E
:100A4000F3F7C4FA00BF012070BD94F8B40340B1BD
:100A5000022084F8E00201220021204600F07CF808
:100A6000F2E700220221204600F076F8ECE70020B1
:100A7000EAE7000070B50446D4F8540201680A227F
:100A80008B6914A1984704F53A710020F3F79FF998
:100A900030B9D4F8540201680F228B6910A198472D
:100AA000F3F737F8054600BFF3F733F8421B104859
:100AB000008810494843104909880E4B594300EB00
:100AC00011408242F0D3D4F85402026891688847FA
:100AD000012070BD536176696E672E2E2E000000D6
:100AE00053617665204661696C65642E2E2E000088
:100AF0000CE4041A40420F000EE4041A70B50546D7
:100B00000C46207885F86D0322460121D5F8540261
:100B1000F3F725FA2078F3F75EFA70BD10B50122DD
:100B200080F8242300F54072D1E90034C2E90A3488
:100B300010BD012280F8242391ED000A80EDCC0A3B
:100B4000704710B5044600220721204600F004F843
:100B500010BDC0F84412704717B595B0179818B972
:100B6000159890F86C0320B9159890F8E1020B28BD
:100B700002D1002018B010BD159890F8E112169817
:100B8000814274D01698022872D1159890F8E1022B
:100B9000E8B1159890F8E102082818D0159890F857
:100BA000E102012813D0159890F8E10203280ED035
:100BB000159890F8E102042809D0159890F8E10200
:100BC000062804D0159890F8E10205287ED11598E2
:100BD0000EF042F8B0B31598D0F8D8020146139041
:100BE000159800F52B7020F077FC006814900068D1
:100BF000406D1390DDE91310884718B31598D0F8AD
:100C0000540213900EF0B0F8E8B90A2016900021B3
:100C10001598C0F87413159890F85C02002810D14C
:100C20000121159880F85C121598D0F854021390A1
:100C30001598D0F85402006880681290DDE912100F
:100C400088477EE101E0002094E7159890F8E102E2
:100C5000012824D1179860B1002012901598D0F87F
:100C6000540212AA20211190F3F779F917E0F2E368
:100C700093E1159890F8E00202280AD0159890F8B0
:100C80009C0330B11598D0F8480201211290F3F777
:100C9000A7F90221159880F8E01200206AE70621E2
:100CA0001598F3F7A2F94FF0FF311290F3F7A2F97C
:100CB000F3F7A5F903280FD10020F3F78CF90020F2
:100CC00012901598D0F8540212AA00E05EE10121BA
:100CD0001190F3F744F900BF159890F8E102E8B1DC
:100CE000159890F8E102012818D0159890F8E102C3
:100CF0000C2813D0159890F8E10203280ED015980F
:100D000090F8E102042809D0159890F8E10206282D
:100D100004D0159890F8E102052801D1012000E0E7
:100D2000002013901398002879D015980DF094FFA7
:100D30000028F9D0159890F8E10203281FD01598E3
:100D4000D0F8D80201461090159800F52B7020F0CD
:100D5000C3FB006812900068006C10901099129804
:100D6000884760B900211598C0F804131598D0F889
:100D7000FC021090F3F748F91599C1F8FC02159898
:100D8000D0F8D80201461090159800F52B7020F08D
:100D9000A3FB006811900068806B1090DDE91010D3
:100DA00088471599D1F87413884209D10021159804
:100DB000C0F8CC131598C0F8D013159880F89C1380
:100DC000159890F8E10203287DD0159890F8E1027B
:100DD000042878D0159890F8E102062873D0159869
:100DE00090F8E10205287BD01598D0F8A802109061
:100DF0001598D0F8D80201460A90159800F52B7086
:100E000020F06AFB0B9010980068C06800220A90DE
:100E1000DDE90A311098984710B90020AAE660E091
:100E20001598D0F87403401E1599C1F8740300207A
:100E3000F3F7EFF8012019F041FE0120F3F7E9F88C
:100E400018200EF01DFD0F9078B108200221CDE989
:100E500000101598D0F83C020B90FE480CC80B9976
:100E60000F981BF0B1FC0F9000E000200C9015983B
:100E7000D0F83C020B901FF07BFC0D900C980E906C
:100E80000D980068C0684FF0FF320EA90B900B9BC5
:100E90000D98984705211598F3F7A7F801210B90B5
:100EA000F3F7A8F81598D0F834020B9000210B98AE
:100EB00000F5805080F8A1100B9800F5805080F864
:100EC000A0100B9800E00BE000F5805080F8941023
:100ED00000BF1598D0F838020B90F3F79FF800BFC9
:100EE0002EE0159890F8E102082829D118200EF07C
:100EF000C7FC129070B10220009001901598D0F8B4
:100F000034020E90D4480CC80E9912981BF0DAFCEB
:100F1000129000E000200F901598D0F834020E9047
:100F20001FF026FC10900F98119010980068C06870
:100F30004FF0FF3211A90E900E9B1098984700BFFA
:100F400000BF159890F8E10220B1159890F8E102E1
:100F500001281AD100211598C0F858121598D0F818
:100F6000580212901598D0F85402119012991BF063
:100F700050FB002013901598D0F8540213AA4FF498
:100F800080611290F2F7EBFF00BF63E2159890F8D2
:100F9000E1020728F9D00020ECE5169801287CD161
:100FA000159890F8E10248B9159800F52B701FF0DC
:100FB00033FD1599D1F8D812884201D80020D9E51F
:100FC0001598D0F83C029FEDA50A0990F3F72BF88D
:100FD000DFEDA30A80EE201ABDEEC10A8DED0F0AE7
:100FE00002A81599F3F724F802A80FC806AC0FC49D
:100FF0001598D0F81003191A0F98081A019015982F
:10100000D0F83C0200900199F3F717F801211598E8
:1010100080F8B413159880F8E0121598F2F7D1FF14
:1010200014900BA8009014980068C06C0CAB0DAA2B
:101030000EA90990099C1498A0470021159800F565
:101040005F70F2F7FBFE9DED0E0AB8EEC00A80ED70
:10105000000A0121159800F55F70F2F7EFFE9DED93
:101060000D0AB8EEC00A80ED000A0021159800F5BF
:101070006170F2F7E3FE0C9A0E99114400EE101A1B
:10108000B8EEC00A80ED000A0121159800F56170E4
:10109000F2F7D4FE9DED0D0A00E07CE0B8EEC00A48
:1010A00080ED000A0021159800F56370F2F7C6FE86
:1010B0000C9A0E99114400EE101AB8EEC00A80ED99
:1010C000000A0121159800F56370F2F7B7FE0B9A3C
:1010D0000D99114400EE101AB8EEC00A80ED000A16
:1010E0000021159800F56570F2F7A8FE9DED0E0A37
:1010F000B8EEC00A80ED000A0121159800F5657070
:10110000F2F79CFE0B9A0D99114400EE101AB8EEFE
:10111000C00A80ED000A18200EF0B2FB139078B1DF
:1011200008200221CDE900101598D0F83C02099062
:1011300048480CC8099913981BF046FB139000E02F
:1011400000200A901598D0F83C0209901FF010FB7F
:1011500011900A98129011980068C0684FF0FF3201
:1011600012A90990099B1198984705211598F2F743
:101170003CFF01210990F2F73DFF0120F2F72BFF20
:10118000012010901598D0F8540210AA012109905E
:10119000F2F7E5FEF9E6169800285AD1159890F86E
:1011A000E1020B287ED0159890F8E1020D28F9D0C5
:1011B000159890F8E102012821D1179850B100202C
:1011C00010901598D0F8540210AA20210F90F2F731
:1011D000C6FE14E0159890F8E00250B1159890F80A
:1011E0009C0330B11598D0F8480201211090F2F715
:1011F000F7FE0021159880F8E0120020BAE4159857
:1012000090F8B403E0B109A81599F2F711FF09A805
:101210000FC80DAC0FC41598D0F81003181A089019
:101220001598D0F83C0207900899F2F706FF09F0EC
:1012300013FB1599C1F818030021159880F8B41311
:1012400000211598C0F804131598D0F8FC021090EE
:1012500008E003E1EC6C041AE46C041AE3A59B3D7E
:10126000A913503BF2F7D0FE1599C1F8FC020021FA
:10127000159880F85C1206211598F2F7B6FE002149
:101280001090F2F7B7FE05211598F2F7AEFE002197
:101290001090F2F7AFFE18200EF0F2FA149088B119
:1012A000082000E0D8E00121CDE900101598D0F821
:1012B0003C021090F7480CC8109914981BF084FA5F
:1012C000149000E0002011901598D0F83C02109086
:1012D0001FF04EFA12901198139012980068C0688F
:1012E0004FF0FF3213A91090109B12989847159851
:1012F00090F86D031090F2F76EFE1598D0F8540236
:101300001090159A02F26D320121F2F728FE15981D
:101310000DF0A2FC00287CD01598F2F793FE00286F
:1013200077D0159890F86E03C0B3159800F52B7020
:1013300020F07DF800681090109870B3159800F5B3
:101340002B7020F07FF8159800F52B701FF064FBD0
:10135000401E1599C1F8D8021098006840690E9097
:101360000E991098884700210F90F2F770FE1098A0
:1013700030B11098006840680F90DDE90F10884781
:101380001598D0F854020F901598D0F854020068C0
:1013900080680E90DDE90E10884745E0FFE715985C
:1013A00090F86C03B0BB1598D0F85802C0B11598EE
:1013B000D0F8D80201460E90159800F52B7020F059
:1013C0008BF800680F901598D0F858020E900F987F
:1013D0000068406F0D90DDE90D210F98904700BF28
:1013E0001598D0F8D80201460E90159800F52B708C
:1013F00020F072F8006810900068806F0E900E99CF
:10140000109888470F901598D0F854020E900F99B5
:1014100001E01BE008E01BF008F91598D0F8540231
:101420000F901BF0EDF800BF1598D0F8DC020028F3
:101430000CDB0122159901F537711598F2F70CFEB6
:1014400020B14FF0FF311598C0F8DC12002115983B
:1014500080F86C13A1E2C3E200201FE41698042870
:1014600001D100201AE4169803281FD115980DF019
:10147000F3FBA0B11598D0F8D80201461290159848
:1014800000F52B7020F028F8006814900068006CBC
:10149000129012991498884708B1012000E00020AA
:1014A0001390139808B90020B8E476E2169806283D
:1014B0001AD11598D0F8A00313901598D0F8A0036E
:1014C0000068C0691290DDE9121088471599B1F8DB
:1014D000A813884201D0012000E000201490149845
:1014E00008B900209AE458E21698052835D11598D5
:1014F00090EDE90A8DED120AD0F8A003119015982D
:10150000D0F8A0030068406B10909DED120ADDE951
:10151000101088478DED140A1598D0F8A00312908A
:101520001598D0F8A0030068806A1190DDE91110C9
:10153000884700EE100AF8EE400A9DED140AF4EE1A
:10154000400AF1EE10FA01D0012000E000201390D3
:10155000139808B9002061E41FE21698082857D1B3
:10156000159890F8E102022844D106211598F2F767
:101570003CFD00211090F2F73DFD14200EF080F9A3
:101580001490F0B114980C901598D0F83402424998
:101590000D9003C9CDE90E010220109010990C980E
:1015A000F2F75FFD0C903D480C990860DDE90C10E6
:1015B0008860DDE90E120C98C0E903120C981490B3
:1015C00000E0002011901598D0F8340210901FF020
:1015D000CFF812901198139012980068C0684FF0DD
:1015E000FF3213A91090109B1298984708B9002059
:1015F00014E4D2E1159890F8E1020A2806D10020FF
:1016000016900021159880F85C12C6E1002005E4D0
:10161000169807287ED1159890F8E102022826D066
:10162000159890F8E10210B3159890F8E102082897
:101630001DD0159890F8E102012818D0159890F85F
:10164000E1020C2813D0159890F8E10203280ED07F
:10165000159890F8E102042809D0159890F8E10255
:10166000062804D0159890F8E10205287ED1159837
:1016700090F8E102012828D1179888B10020109035
:101680001598D0F8540210AA20210F90F2F767FCA9
:101690001BE00000EC6C041AB46C041A9CF3041BED
:1016A000159890F8E00250B1159890F89C0330B16D
:1016B0001598D0F8480201211090F2F791FC002112
:1016C000159880F8E012002066E400211598C0F813
:1016D00058121598C0F87413159890F8E102012873
:1016E00014D0159890F8E1020C280FD01598D0F876
:1016F000440210901098407F40B91598D0F84402E9
:10170000109001211098017700BF00BF1598D0F804
:10171000F41200E0B1E0C0F8FC1218200EF0B0F8AE
:10172000149078B102200021CDE900101598D0F86E
:1017300034021090AB480CC8109914981BF0C2F8F2
:10174000149000E0002011901598D0F83402109009
:101750001FF00EF812901198139012980068C0684C
:101760004FF0FF3213A91090109B00E077E0129821
:1017700098471598D0F8380210900DF07CFC01289D
:101780003ED018200EF07CF8109018B310980790F7
:101790001598D0F838029449089003C9CDE9090199
:1017A00003200B9004200C900C990798F2F759FC39
:1017B00007908E4807990860DDE907108860DDE929
:1017C00009120798C0E9031207990B980875079842
:1017D000109000E000200D901598D0F838020C9081
:1017E0001EF0C6FF0E900D980F900E980068C0680E
:1017F0004FF0FF320FA90C900C9B0E98984700BF3A
:101800000120F2F7E8FB1598D0F854021090159AD1
:1018100002F26D320121F2F7A2FB0121159880F846
:101820006C13159890F8E102012804D0159890F8EF
:10183000E1020C2803D10121159880F89C130020A7
:10184000109008E01098C0B200210F90FCF76AFBDE
:101850001098401C109010980328F3DB9DE0159819
:1018600090F8E1020A2806D1002016900021159870
:1018700080F85C1291E00020C0E416980A280AD192
:10188000159890F8E102E8B3159890F8E10209285C
:1018900038D00020B2E416980C2878D1159890F82A
:1018A000E10208B10020A9E41598D0F83C029FEDB0
:1018B000500A0E90F2F7B7FBDFED4E0A80EE201AC9
:1018C000BDEEC10A8DED100A07A81599F2F7B0FB1D
:1018D00007A80FC80BAC0FC41598D0F81003191A3D
:1018E0001098081A06901598D0F83C0205900699B1
:1018F000F2F7A3FB0121159880F8B4131598D0F8DE
:10190000380200E049E00E90F2F788FB18200DF055
:10191000B7FF149078B108200221CDE90010159886
:10192000D0F83C020E9034480CC80E9914981AF066
:101930004BFF149000E000200F901598D0F83C0267
:101940000E901EF015FF12900F98139012980068D9
:10195000C0684FF0FF3213A90E900E9B1298984763
:1019600005211598F2F741FB01210E90F2F742FB99
:101970000120F2F730FB012011901598D0F85402A5
:1019800011AA01210E90F2F7EAFA06E0FFE7169895
:101990000D2802D119A0F0F759FF159890F8E1121F
:1019A00080F8E212DDE9151081F8E1021598D0F80F
:1019B00054021390159890F8E1021490139801794D
:1019C0001498814209D0DDE913100871139800685A
:1019D00080681290DDE91210884700BF01200DE4F5
:1019E00000200BE4E46C041ABC6C041A2CF3041BF6
:1019F000E3A59B3DA913503BEC6C041A537570652D
:101A0000727669736F7220696E204552524F522070
:101A100073746174650A0000F0B585B004460D4624
:101A20002868C4F8B00310270C4B0FCB01AE0FC6CB
:101A30002046F2F71BFB064609A30AA210210090DC
:101A400001A8EEF77FFF01AE3046F2F714FB10B1AC
:101A50000648F0F7FBFE00BF05B0F0BD3C6D041A70
:101A600047325F00257325640000000051F9041B14
:101A70000A68C0F8F4220A68C0F8FC22704770B502
:101A800004460D46D4F800032968884209D0286826
:101A9000C4F80003002203212046FFF75DF800B1DF
:101AA00070BD2046F2F779FA00BFF9E70A68C0F87E
:101AB00008237047C0F84812704738B504462046DE
:101AC000FEF72EFF80F00100694600902046FFF7E8
:101AD00015F838BD2DE9F04F2DED028B83B004468B
:101AE0004FF0000AD4F83C02F2F7CAFA18B194F8A1
:101AF000E1020B2804D103B0BDEC028BBDE8F08FEE
:101B0000D4F85482D8F80000416A4046884783469A
:101B10000068816858468847054620460DF09CF8C5
:101B200068B104F52B70D4F8D8121FF0D5FC066804
:101B30003068016C3046884708B1012000E0002081
:101B40000090009818B194F8E10200287ED1D4F8F2
:101B500054020DF009F9012879D182460121D4F807
:101B60005402F2F792FAB0EE408A94F8D40378B9AE
:101B700005F00C0060B9F1F7CCFFB74908609FEDA4
:101B8000B70A84EDBE0AB1EE080A2046FEF7D0FD82
:101B90004FF00008F1F7BDFFAF490968421AB0489D
:101BA0000088B0494843B0490988AE4B594300EB1F
:101BB0002140824208D2B5EE000AB4EEC08AF1EEAE
:101BC00010FA01DD4FF00108B8F1000F25D094F8AC
:101BD000D40310BB012084F8D40305F0040060B1E5
:101BE00094EDBD0AB8EEC00ADFEDA00A30EE200A7F
:101BF000BDEEC00A84EDBF0A41E005F0080038B32D
